:020000040800F2
:10000000000001102D3803085582020871C3000852
:100010003139030831390308313903080000000081
:10002000000000000000000000000000A18802089D
:100030009D8802080000000099880208D58C0008FD
:1000400031390308313903083139030831390308DC
:10005000313903083139030855980008819900089F
:100060004599000809990008CD980008D9B1000801
:10007000C9B10008B9B10008A9B1000899B10008D8
:1000800085B1000871B1000831390308313903081E
:1000900031390308313903083139030891980008D0
:1000A000313903083139030831390308313903087C
:1000B000A1CD00083139030891CD0008313903087A
:1000C000313903083139030831390308313903085C
:1000D0003139030831390308A58D0008098D00085E
:1000E0001998000831390308BD880208313903081E
:1000F00061CD00083139030871CD00085DB10008F9
:10010000313903083139030881CD0008313903083A
:1001100031390308313903080D950108F1940108BC
:1001200049B1000835B1000821B100080DB100083F
:10013000F9B00008313903083139030831390308AF
:100140003139030831390308313903085D82020867
:10015000E5B00008D1B00008BDB00008313903088F
:1001600031390308313903083139030831390308BB
:1001700031390308313903083139030831390308AB
:0801800031390308313903088D
:1001880002020300EC1D0020E81D00200000000012
:1001980000000000F7010600F81D0020F01D0020F7
:1001A800000000008405000816000800001E00205A
:1001B800081E0020000000008A050008270004002F
:1001C800E4210020DC220020000000009205000845
:1001D80008020900902D0020B82D00200000000022
:1001E8002982000802000C009C2D0020C42D00204C
:1001F80000000000000000000A020A009424002009
:10020800D02D002000000000960500081A00080004
:10021800E0350020F835002000000000A0050008A7
:1002280015007000E42F00200036002000000000B8
:100238000000000003000100E02F002070360020BD
:1002480000000000000000002A006000F02E0020DE
:10025800743600200000000085B101082900500014
:100268008C380020D83C002000000000000000006E
:100278001400020088380020283D002000000000FB
:10028800A8050008000205002C3D0020644000205D
:1002980000000000000000001E000400343D0020A3
:1002A8006C40002000000000AA05000822000C0095
:1002B800E03F00207040002000000000AE0500086C
:1002C80026000E006C4700205C470020000000005C
:1002D800492B02080B201000F44500207C47002021
:1002E80000000000BA05000803123300F34800209C
:1002F800C048002000000000CA05000825005A0078
:100308000C480020664800200000000000000000A3
:100318000120080038490020404900200000000062
:10032800FE050008FD012400D44A0020F84A0020F8
:1003380000000000A1810008FB010100A84A00207C
:100348001C4B002000000000D9B20008FC01090085
:1003580074490020204B002000000000A5B20008CE
:100368000A101200484900202C4B00200000000011
:100378000606000804008000285E0020285F002090
:100388000000000000000000F9010400905B00205C
:10039800A85F0020000000001182000818102C003F
:1003A800605B0020AC5F00200000000061D1020803
:1003B80013000400386200204062002000000000A2
:1003C8001806000810000300346200204462002070
:1003D800000000001C06000828000C00286200200D
:1003E80048620020000000002006000823001000DA
:1003F80018620020546200200000000059E3010840
:10040800190005001062002064620020000000004E
:100418002C060008F81101000C6200206C62002014
:1004280000000000320600080001040008620020F5
:100438007062002000000000340600082F00110040
:10044800F4610020746200200000000038060008F3
:10045800060016001C6400205867002000000000F9
:1004680041B1010834001000886200207067002044
:1004780000000000FDB001082C001000A46C002052
:10048800946C0020000000002DC802082B002400F6
:10049800D86C0020B46C002000000000FDC70208E2
:1004A8000D002C00187D0020447D00200000000075
:1004B80051140208FE01080004770020707D002016
:1004C80000000000E1B2000803010600C87D00201A
:1004D800047E0020000000004A0600081F000E00ED
:1004E800E47E0020C08000200000000050060008C4
:1004F80005020100CC7E0020D08000200000000012
:100508005E0600080101040024810020008200200A
:100518000000000000000000050006007E830020A7
:10052800BC83002000000000600600080C002400C6
:1005380046830020C4830020000000008D8C010841
:100548000E20EA003E820020E88300200000000020
:10055800ADB1010812100C001E820020D4840020C6
:10056800000000006606000802010300198200204E
:0C057800E0840020000000004D1103088A
:10058400000001000000C40900001901282820030C
:10059400000000004A01B400D60100007E05EA050F
:1005A400B4053200030000000100C800141E01005D
:1005B40064002C0128002B21231E6400020000008B
:1005C40001000A01290000000000000000000000F2
:1005D4000000000000000000000000000000000017
:1005E4000000000000000000000000000000000007
:1005F40000000000000000000100E8036400040A99
:10060400000100300100005A0000000090012C019C
:10061400C80064000800000000010500000000019B
:100624000000000000000000000028010000040099
:100634009001000000000000000000000000000025
:1006440000000000000004010100000000000000A0
:10065400000001000000000500000000200003006D
:0E0664000100000000010005454C4C30000074
:100672000000803F0000803F0000803F50010000EA
:10068200070000000200000000000000000000005F
:10069200010203040607080901010000CC880308CF
:1006A2005CA303080000000000000000DC880308CF
:1006B200E48803080000000001200000E888030825
:1006C200F08803080000000001400000F4880308DD
:1006D200A09A03080000000001200000008903081E
:1006E2000C890308000000000400000010890308C0
:1006F2001C89030800000000040000002089030890
:1007020064AF0308000000000100000002010000C5
:100712000000803F0000803FFF000000D465030816
:1007220005080400000000004C880308E88703085D
:10073200C0650308000000000066030805080A00FF
:10074200000000004C880308E88703089885030826
:1007520000000000FFFFFFFF010000000001010197
:10076200010000000000803FF1800208A980020819
:10077200F97F020800000000E97C02086D7E020891
:10078200ED7E0208D57D0208000000000000000096
:10079200DD7C0208C17C020859820208BD7C020885
:1007A200B17C0208AD7C0208B97C0208B57C020863
:1007B200D17C0208C57C0208AD7D0208C17D020819
:1007C200997D0208857D0208717D020860A30308F5
:1007D20000000000000000005D110308A086010077
:1007E2000400000000000000000000000000000003
:1007F20000000000000000000000000000000000F7
:1008020088B1030874A003080000000061FD00081D
:100812007D00000006000000000000000000000053
:1008220000000000000000000000000000000000C6
:100832000000000068A303080000000000000000A0
:1008420031B30208E80300000300000000000000CA
:100852000000000000000000000000000000000096
:10086200000000000000000070A303080000000068
:1008720000000000013802081027000003000000F9
:100882000000000000000000000000000000000066
:1008920000000000000000000000000040B6030855
:1008A2000000000089C602081D4B0108204E00000E
:1008B2000500000000000000000000000000000031
:1008C2000000000000000000000000000000000026
:1008D200C8A903080000000000000000EDAD0208F6
:1008E20010270000010000000000000000000000CE
:1008F20000000000000000000000000000000000F6
:10090200000000007CA303080000000000000000BB
:1009120071B20008E80300000500000000000000BA
:1009220000000000000000000000000000000000C5
:10093200000000000000000088A30308000000007F
:100942000000000085130308204E00000300000091
:100952000000000000000000000000000000000095
:1009620000000000000000000000000098A303083F
:1009720000000000000000008D110308204E00005E
:100982000300000000000000000000000000000062
:100992000000000000000000000000000000000055
:1009A200A8A30308000000000000000089AB0208B1
:1009B200400D0300030000000000000000000000E2
:1009C2000000000000000000000000000000000025
:1009D2000000000090A003080000000000000000DA
:1009E200290F020810270000030000000000000089
:1009F20000000000000000000000000000000000F5
:100A02000000000000000000B8A30308000000007E
:100A1200000000009D2C0308A086010001000000D8
:100A220000000000000000000000000000000000C4
:100A3200000000000000000000000000C0A3030846
:100A4200000000000000000015D40008A00F000004
:100A52000100000000000000000000000000000093
:100A62000000000000000000000000000000000084
:100A7200CCA30308000000000000000075F9020882
:100A8200102700000100000000000000000000002C
:100A92000000000000000000000000000000000054
:100AA2000000000068A00308000000000000000031
:100AB20085BB02081A41000001000000000000008E
:100AC2000000000000000000000000000000000024
:100AD2000000000000000000D8A30308000000008E
:100AE200000000002D140208400D03000000000069
:100AF20000000000000000000000000000000000F4
:100B0200000000000000000000000000E0A3030855
:100B12000000000000000000E9130208400D03007D
:100B220000000000000000000000000000000000C3
:100B320000000000000000000000000000000000B3
:100B4200E8A303080000000000000000AD14030841
:100B5200A086010003000000000000000000000069
:100B62000000000000000000000000000000000083
:100B7200000000000000803F01000000040309049F
:100B820012010002020200408304405700020102E7
:100B92000301000009024300020100C032090400FF
:100BA20000010202010005240010010524010001D8
:100BB200042402020524060001070582030800FF3F
:100BC20009040100020A00000007050102400000BA
:100BD2000705810240000000FF000000D9810208E1
:100BE200197F0208510903082D7D02088581020838
:100BF2003D7D0208597D02081D7D02080D7D020817
:100C02000000000000000000303030302D30312D67
:100C120030315430303A30303A3030005CBA030868
:100C22000E000000000000000000000000000000B4
:100C320004130020FFFFFFFFFA0000000100000084
:100C420001000000F4B403080000000000000000EE
:100C52000000000000000000EBB4030804000000E4
:100C6200352303080000000000000000FCB4030864
:100C72000100000000000000000000000000000071
:100C8200000000000D000000000000000000000055
:100C920000000000866800200100C4090000000076
:100CA200846800200100C40900000000826800205E
:100CB2000100C40900000000806800200100C4098E
:100CC200000000007C6800200100C4090000000050
:100CD2007E6800200100C409000000007A6800203C
:100CE2000100C40900000000786800200100C40966
:100CF2000000000020B503080E0000000000000004
:100D02000000000000000000D4050020C47D002087
:100D12009CFF2C0100000000CA1500200A00000000
:100D22009885030804820020E0150C1700000000DB
:100D3200C915002008000000E8870308C815002034
:100D4200050000004C880308068200200200000013
:100D5200B0850308848300200100FF7F01000000AA
:100D62007C83002002000000BC8503082C82002046
:100D720003000000CC8503082B8200200300000042
:100D8200CC850308308300200000F401010000003C
:100D92002E8300200000F401010000002C830020BB
:100DA2000000F401010000002A8300200000F40189
:100DB200010000002883002000FF0100448300207E
:100DC200E803D0070A00000042830020006401000B
:100DD2000A00000043830020006401000A000000B2
:100DE2003C830020006401000A00000041830020CF
:100DF200006401000A00000040830020006401003A
:100E02000A0000003F830020006401000A00000085
:100E12003B83002000FF01000A0000003A8300200B
:100E220000FF01000A0000003A8200200000F401E5
:100E320001000000388200200000F40101000000DF
:100E4200368200200000F4010100000034820020FC
:100E52000000F401010000003783002000C80100F7
:100E62003683002000C801003583002000C801003D
:100E720034830020006401000A0000003383002054
:100E820000FF01000A0000007383002000C8010077
:100E92007283002000C801007183002000C8010095
:100EA2007083002000C801006F83002000C8010089
:100EB2006E83002000C801006D83002000C801007D
:100EC2006C83002000C801006B83002000C8010071
:100ED20028B5030800000000000000000000000028
:100EE2000000000038B503080900000000000000FF
:100EF200780600200400000040B503080900000045
:100F0200000000006C0600200400000008B903087D
:100F1200090000000000000060060020040000003C
:100F220048B5030809000000000000005406002034
:100F3200040000004CB50308090000000000000096
:100F4200480600200400000054B503080900000010
:100F5200000000003C060020040000005CB503080D
:100F6200090000000000000030060020040000001C
:100F720064B50308090000000000000024060020F8
:100F820004000000FCB4030801000000000000009F
:100F92000000000000000000000000000D00000042
:100FA20000000000000000000000000050B603082E
:100FB200000000000000000000000000000000002F
:100FC2005CA303080000000000000000B817002026
:100FD200040000005CB603080C0000007D23030837
:100FE200D806002000000000A0BB03080C0000008F
:100FF2005D1F0308CC0600200000000060B6030855
:101002000C000000291F0308C00600200000000099
:1010120068B603080800000000000000B4060020C3
:101022000400000070B603080C000000151F03083E
:10103200A80600200000000078B60308090000009E
:10104200000000009C0600200400000080B6030897
:101052000300000061BA02088406002000000000BC
:10106200FCB40308010000000000000000000000C2
:1010720000000000000000000D0000000000000061
:10108200000000000000000084B603080000000019
:1010920000000000000000000000000094B60308F9
:1010A2000C00000000000000F0060020000000001C
:1010B2009CB603080A00000000000000958300208F
:1010C20000000000A8B603080A00000000000000AB
:1010D2009D83002000000000B0B603080A00000053
:1010E20000000000A583002000000000B8B603083D
:1010F2000800000000000000E406002000000000DC
:10110200FCB4030801000000000000000000000021
:1011120000000000000000000D00000000000000C0
:101122000000000000000000C0B60308000000003C
:10113200000000000000000000000000D4B6030818
:101142000C00000000000000080700200000000062
:10115200E4B6030804000000312603080000000082
:1011620000000000ECB603080C00000000000000C4
:10117200FC0600200000000000B703080400000085
:10118200152603080000000000000000FCB403085C
:10119200010000000000000000000000000000004C
:1011A200000000000D000000000000000000000030
:1011B2000000000008B70308000000000000000063
:1011C20000000000000000001CB703080700000038
:1011D20000000000440700200000000028B70308B8
:1011E2000800000000000000380700200000000096
:1011F20034B7030808000000000000002C0700209C
:101202000000000040B703080800000000000000D2
:1012120020070020000000004CB70308080000006F
:10122200000000001407002000000000FCB40308C6
:1012320001000000000000000000000000000000AB
:10124200000000000D00000000000000000000008F
:101252000000000058B70308000000000000000072
:10126200B31700200000000064B703080B00000061
:1012720000000000AC070020000000006CB703086B
:101282000B00000000000000A0070020000000008A
:1012920078B703080B00000000000000940700204C
:1012A2000000000084B703080B00000000000000EB
:1012B200880700200000000090B703080B00000020
:1012C200000000007C070020000000009CB703081B
:1012D2000B0000000000000070070020000000006A
:1012E200A4B703080B000000000000006407002000
:1012F20000000000B0B703080B000000000000006F
:101302005807002000000000BCB7030808000000D6
:10131200000000004C07002000000000FCB403089D
:1013220001000000000000000000000000000000BA
:10133200000000000D00000000000000000000009E
:1013420000000000C8B70308000000000000000011
:101352000000000000000000DCB7030808000000E5
:1013620000000000DC07002000000000E8B70308CE
:101372000800000000000000D0070020000000006C
:10138200F4B703080800000000000000C4070020B2
:101392000000000000B80308080000000000000080
:1013A200B807002000000000FCB4030801000000A0
:1013B200000000000000000000000000000000002B
:1013C2000D0000000000000000000000000000000E
:1013D20008B803080000000000000000B017002059
:1013E2000000000018B803080B0000000000000015
:1013F2000C0800200000000024B803080B000000C5
:1014020000000000000800200000000030B80308BF
:101412000700000000000000F807002000000000A4
:101422003CB803080700000000000000F00700209D
:101432000000000048B80308070000000000000098
:10144200E807002000000000FCB4030801000000CF
:10145200000000000000000000000000000000008A
:101462000D0000000000000000000000000000006D
:1014720054B803080000000000000000B01700206C
:101482000000000060B80308070000000000000030
:10149200580800200000000068B803080700000098
:1014A20000000000500800200000000070B803088F
:1014B20007000000000000004808002000000000B3
:1014C20078B8030807000000000000004008002070
:1014D2000000000080B803080700000000000000C0
:1014E200380800200000000088B803080700000048
:1014F20000000000300800200000000090B803083F
:101502000700000000000000280800200000000082
:1015120098B803080700000000000000200800201F
:1015220000000000A0B8030807000000000000004F
:101532001808002000000000FCB4030801000000AD
:101542000000000000000000000000000000000099
:101552000D0000000000000000000000000000007C
:10156200A8B803080E00000000000000E1200308F4
:1015720000000000600800202A82002017000000FE
:10158200DC8503081D8200200A3201001C82002033
:1015920001FA01001882002000C801001682002012
:1015A200E803D00701000000454C4C453000000024
:1015B200B0B803080E000000751E0308000000000A
:1015C200000000003C090020B8B803080E0000002B
:1015D200E52303080D23030809230308180A002042
:1015E200C0B803080E000000F72003080000000046
:1015F20000000000B80A0020C8B803080E0000006E
:10160200812103085121030800000000440B00203F
:10161200D0B803080E000000FD210308452203088C
:1016220000000000E40B00203883002001030100C9
:10163200DCB803080E000000252103080921030875
:1016420000000000D40C0020E4B803080E000000E3
:10165200B12103084D26030800000000600D0020A0
:10166200F0B803080E000000712203089126030857
:1016720000000000000E0020328300200103010060
:10168200F8B803080000000000000000000000009D
:101692000000000004B90308080000000000000078
:1016A2002C0F0020000000000CB903080700000006
:1016B20000000000240F0020000000001CB90308F5
:1016C20007000000000000001C0F002000000000C6
:1016D20028B903080700000000000000140F0020D2
:1016E2000000000034B903080C00000000000000F4
:1016F200080F00200000000040B9030803000000AA
:1017020061BA0208F00E002000000000FCB40308D9
:1017120001000000000000000000000000000000C6
:10172200000000000D0000000000000000000000AA
:101732000000000048B9030800000000000000009B
:10174200000000000000000058B903080A00000071
:1017520000000000608A03080000000060B903086E
:101762000A00000000000000AC880308000000002E
:1017720068B903080A00000000000000748300201A
:101782000000000070B903080A0000000000000019
:10179200380F002000000000FCB403080100000024
:1017A2000000000000000000000000000000000037
:1017B2000D0000000000000000000000000000001A
:1017C20078B90308000000000000000000000000DB
:1017D2000000000034B403080300000061BA0208EC
:1017E200580F0020000000008CB90308030000001D
:1017F20061BA0208CC1500200000000094B9030869
:101802000300000061BA0208400F0020000000003F
:10181200FCB403080100000000000000000000000A
:1018220000000000000000000D00000000000000A9
:1018320000000000000000009CB903080000000046
:10184200000000000000000000000000A8B903082A
:1018520007000000DD260308081000200000000039
:1018620088B103080300000061BA0208F00F0020EB
:1018720000000000B4B903080300000061BA0208C6
:10188200D80F002000000000BCB9030803000000CC
:1018920061BA0208C00F002000000000C4B90308AA
:1018A20007000000C1260308B80F00200000000056
:1018B200C4BB03080300000061BA0208A00F0020A5
:1018C20000000000D0B903080300000061BA02085A
:1018D200880F002000000000DCB9030803000000AC
:1018E20061BA0208700F002000000000FCB4030877
:1018F20001000000000000000000000000000000E5
:10190200000000000D0000000000000000000000C8
:1019120000000000E8B903080E000000AD20030833
:10192200792003080000000010100020F0B903081D
:101932000E000000DD22030800000000000000008D
:10194200C4100020FCB903080E00000000000000D3
:101952000000000000000000501100200CBA030833
:101962000E000000B9220308F92603080000000057
:10197200C811002014BA0308000000000000000093
:10198200000000000000000020BA0308030000006D
:1019920061BA0208EC1200200000000000BA03083D
:1019A2000300000061BA0208D41200200000000007
:1019B20028BA03080300000061BA0208BC12002022
:1019C2000000000034BA03080300000061BA0208F4
:1019D200A4120020000000003CBA0308020000002C
:1019E20069B90208000000000000000044BA0308C0
:1019F2000200000069B902080100000000000000B6
:101A020050BA03080200000069B90208020000008F
:101A120000000000000000000D00000000000000B7
:101A2200000000000000000001010000D9E80108E8
:101A32000000000000000000006002401060024050
:101A420000000000000B0000000020000000000069
:101A52000000000000600240286002400000000018
:101A6200060C000000002000000000000000000042
:101A7200006002404060024000000000100D0000C3
:101A82000000200000000000000000000060024092
:101A92005860024000000000160E00000000200006
:101AA2000000000000000000006002407060024080
:101AB20000000000200F00000000200000000000D5
:101AC2000000000000600240886002400000000048
:101AD20026100000000020000000000000000000AE
:101AE20000600240A06002400000000030110000CF
:101AF2000000200000000000000000000060024022
:101B0200B860024000000000362F000000002000F4
:101B12000000000000000000006402401064024067
:101B2200000000000038000000004000000000003B
:101B3200000000000064024028640240000000002F
:101B42000639000000004000000000000000000014
:101B5200006402404064024000000000103A0000AD
:101B6200000040000000000000000000006402408D
:101B72005864024000000000163B000000004000D4
:101B82000000000000000000006402407064024097
:101B920000000000203C00000000400000000000A7
:101BA200000000000064024088640240000000005F
:101BB2002644000000004000000000000000000079
:101BC20000640240A06402400000000030450000B2
:101BD200000040000000000000000000006402401D
:101BE200B8640240000000003646000000004000D9
:101BF200000000000000000000FFFF0000000000E5
:101C0200AA5505010000AA5507010000AA550300C4
:101C12009FAA550B010000AA55090200000000000E
:101C220001000000C01201000000000001020304D4
:101C320001020304060708090101010048BC030868
:101C42000E000000B11F03080000000000000000A9
:101C52004C1700201CBC030800000000000000001C
:101C620000000000000000005CA303080000000068
:101C720000000000D817002004000000A0BB0308E9
:101C82000C0000006D250308EC1B00200000000082
:101C920060B603080C0000003D250308E01B00208D
:101CA2000000000068B60308080000000000000001
:101CB200D41B00200400000070B603080C000000D2
:101CC20055240308C81B00200000000080B603084A
:101CD2000300000061BA0208B01B002000000000EF
:101CE2002CBC03080300000061BA0208981B002004
:101CF20000000000FCB40308010000000000000026
:101D02000000000000000000000000000D000000C4
:101D12000000000000000000000000001CBC0308DE
:101D220000000000000000000000000000000000B1
:101D32005CA303080000000000000000D817002088
:101D4200040000004CBB030803000000A5230308A5
:101D5200801B00200800000070B603080C00000081
:101D620055240308C81B00200000000080B60308A9
:101D72000300000061BA0208B01B0020000000004E
:101D82002CBC03080300000061BA0208981B002063
:101D920000000000FCB40308010000000000000085
:101DA2000000000000000000000000000D00000024
:101DB20000000000000000000000000034BC030826
:101DC2000000000000000000000000000000000011
:101DD2005CA303080000000000000000D8170020E8
:101DE2000400000054BB03080300000061BA0208AB
:101DF200F81B002000000000FCB4030801000000F2
:101E020000000000000000000000000000000000D0
:101E12000D000000000000000000000000000000B3
:101E220020700020702D72002D202D2D202D2D2DA3
:101E32002D202D2D2D2D000000000000000000009F
:101E420000000000000000002D202D2D202D2D2D42
:101E52002D202D2D2D0000000000000000000000AC
:101E620000000000000000001282002088130C17FE
:101E7200010000001482002088130C1700000000EB
:101E8200A4BA0308000000000000000000000000E7
:101E920000000000B4BA03080800000000000000BF
:101EA2000418002004000000C0BA03080800000063
:101EB20000000000F81700200000000080B60308B0
:101EC20004000000392403080000000000000000A4
:101ED200FCB4030801000000000000000000000044
:101EE20000000000000000000D00000000000000E3
:101EF20000000000000000001082002088130C1770
:101F0200010000000E82002088130C170000000060
:101F1200FCBA03080E0000000920030800000000BC
:101F22000000000010180020AE8300200100000015
:101F32000C8803080D8200200100000018880308A5
:101F4200FA7D00200200000020880308DE5E0020E7
:101F52000000000000000000DC5E00200000000025
:101F620000000000DA5E0020000000000000000017
:101F7200D85E00200000000000000000D65E0020B5
:101F82000000000000000000D45E002000000000FD
:101F920000000000B4150020000000000000000056
:101FA2000C820020020000002C88030804BB0308F6
:101FB200000000000000000000000000000000001F
:101FC200B4BA0308080000000000000094180020C2
:101FD20004000000C0BA030808000000000000006E
:101FE200881800200000000080B6030804000000EA
:101FF200E91F03080000000000000000FCB4030811
:1020020001000000000000000000000000000000CD
:10201200000000000D0000000000000000000000B1
:102022000000000014BB03080000000000000000D4
:10203200000000000000000024BB03080C000000A8
:10204200DD240308D01800200400000030BB030880
:102052000C0000002D200308C4180020040000001A
:102062003CBB03080C0000009D240308B8180020A4
:102072000000000048BB030803000000C52303085A
:10208200A01800200800000054BB03080300000051
:1020920061BA0208F81B002000000000FCB403082B
:1020A200010000000000000000000000000000002D
:1020B200000000000D000000000000000000000011
:1020C20000000000F4B4030800000000000000005B
:1020D20000000000000000005CBB030804000000D8
:1020E2009D2503080000000000000000FCB4030866
:1020F20001000000000000000000000000000000DD
:10210200000000000D0000000000000000000000C0
:1021120000000000A8BB030800000000000000004F
:102122000000000000000000B8BB03080C00000023
:10213200000000003019002004000000C0BB0308AA
:102142000800000000000000241900200400000024
:10215200CCBB030808000000000000001819002092
:1021620004000000D4BB03080800000000000000C7
:102172000C19002004000000DCBB0308080000006A
:10218200000000000019002004000000E4BB030866
:102192000800000000000000F41800200400000005
:1021A200ECBB03080800000000000000E818002053
:1021B20004000000F4BB0308080000000000000057
:1021C200DC18002004000000FCB403080100000039
:1021D20000000000000000000000000000000000FD
:1021E2000D000000000000000000000000000000E0
:1021F200FCBB03080E000000F91F030800000000EA
:10220200000000003C19002004BC03080E0000007E
:10221200000000000000000000000000B4190020CF
:102222000CBC03080E0000000000000000000000CB
:1022320000000000541A0020AD83002004000000BA
:102242003888030808820020E0150C1700000000FF
:102252000B82002008000000E88703080A820020A1
:10226200050000004C88030814BC03080E0000009F
:10227200000000000000000000000000A41A00207E
:102282004300000000000000000000000000000009
:10229200000000000000000000000000000000003C
:1022A20043000000000000000000000000000000E9
:1022B200000000000000000000000000000000001C
:1022C20043000000000000000000000000000000C9
:1022D20000000000000000000000000000000000FC
:1022E20043000000000000000000000000000000A9
:1022F20000000000000000000000000000000000DC
:102302004300000000000000000000000000000088
:1023120000000000000000000000000000000000BB
:102322004300000000000000000000000000000068
:10233200000000000000000000000000000000009B
:102342004300000000000000000000000000000048
:10235200000000000000000000000000000000007B
:102362007D3B0308D53903080000000066BC030862
:10237200E6B40308E6A10308E6A10308E6A1030800
:10238200E6A10308E6A10308E6A10308E6A1030803
:10239200E6A10308E6A10308FFFFFFFFFFFFFFFF1F
:1023A200FFFFFFFFFFFF00000100415343494900C7
:1023B200000000000000000000000000000000001B
:1023C20000000000000000000000415343494900A2
:1023D20000000000000000000000000000000000FB
:1023E200000000000000000000000000801D00202E
:1023F20000000000000000000000000000000000DB
:1024020000000000000000000000000000000000CA
:1024120000000000000000000000000000000000BA
:1024220000000000000000000000000000000000AA
:10243200000000000000000000000000000000009A
:10244200000000000000000000000000000000008A
:042452000100000085
:1080000070B4EFF31186502383F31288436B1A6820
:10801000D20720D45D686DB9446A826A944217D051
:1080200081691144D9600ED9A21A5A608462002273
:1080300080F858201A6842F00102F1B21A6081F308
:10804000118870BC704701698A1A5A608562EEE730
:10805000012380F85830F3B283F3118870BC704765
:10806000436A8269D154436A0169426B01338B428E
:1080700028BF00234362002A2FD0EFF31182502340
:1080800083F31288436B1968C9072CD470B45E68F7
:108090006EB9456A816A8D4217D084690C44DC60F0
:1080A0000ED9691A59608562002180F85810196844
:1080B00041F00101D2B2196082F3118870BC70479F
:1080C0000469611A59608662EEE7012380F858302E
:1080D000D2B282F3118870BC7047426DD36843F00E
:1080E0008003D3607047D2B282F31188704700BF1B
:1080F000026B10B462B1836CC2684469D11A013B4F
:10810000615C5DF8044B08BF13468364C8B27047D6
:10811000016A4369C4685B5C0131A14228BF114612
:1081200001625DF8044BD8B2704700BF436B13B1D6
:1081300090F858007047836A406A181AB0FA80F0C5
:1081400040097047416A836A99420AD3CB1A416B4E
:10815000026961B14968501E0B4483420AD2C01AB9
:10816000704702691144CB1A416B0029F2D1501EAD
:10817000C01A704700207047036B43B1826C5B6884
:1081800093422FBF981AC0689B1AC0187047C269E3
:10819000036A9A422FBFD01AC0688018C01A70476D
:1081A0000A4B30B503F1100493F900205D78072ADB
:1081B000C8BF143A811804330D7313F8025C855458
:1081C00013F8012C0A76A342EED130BD606003089B
:1081D00003682DE9F041DF691FB13B46BDE8F0417E
:1081E0001847002A164611DD04460D460E4400E0ED
:1081F00023689B68204698470028F9D0236815F823
:10820000011B1B6820469847AE42F1D1BDE8F081C2
:1082100010B424211824322200230470417082708B
:10822000C3705DF8044B70472D2343702E230371F8
:108230002F23C371704700BF30B4856815B12B6818
:10824000AC885C83436840F2E93001E0002830D01C
:108250001C89013814F0020F80B2F7D089B29981DD
:1082600040F2E93100E021B31889013910F0010F23
:1082700089B2F8D0998940F2E93100E019B3188940
:10828000013910F0020F89B2F8D092B29A8140F20F
:10829000E93200E0BAB11989013A11F0010F92B246
:1082A000F8D09B8915B12B68AA881A83012030BCAD
:1082B00070470A498B42DED10948418B013189B2AE
:1082C0004183418BD7E7054A9342EBD1044A538B54
:1082D00001339BB25383538BE4E700BF0038004067
:1082E000E4740020002870B51EDB0928044620DD58
:1082F000012303EB83035B00B0FBF3F2092AF8D8F8
:108300007BB10E4EB4FBF3F00928CCBF57223022CC
:10831000A6FB03E5024403FB1044EB0801F8012B24
:10832000F0D100230B7070BD2D230B704042013142
:10833000DBE7303001F8010BF3E700BFCDCCCCCC4C
:10834000884230B44FF001042ED301FB04F4B0FB9B
:10835000F4F58D42F9D284B1AAB901E0B0FBF4F58D
:10836000092DCCBF572230222A4404FB150003F804
:10837000012BB4FBF1F4002CF0D100221A7030BCB8
:108380007047B0FBF4F5092DCCBF372230222A44C8
:1083900004FB150003F8012BB4FBF1F4002CF0D121
:1083A00000221A7030BC70470546002AEBD1D7E78F
:1083B00003685A1C02601970704700BF2DE9F0472E
:1083C000089C2578002B804689460CBF4FF0200A78
:1083D0004FF0300A661C35B3002A29DD334601E030
:1083E000024698B113F8011B501E0029F8D1971EC0
:1083F00060B13D46013D51464046C8476B1C002BCD
:10840000F8DC257827EAE770013055B1041B2946CE
:108410004046C847301916F8015B002DF7D1BDE87A
:10842000F087BDE8F087002A04DC2846BDE8F08725
:108430000020EBE7571EDCE783684268D0ED037A43
:1084400000EB83010133934281ED040A836004BF92
:108450000023836000EB830393ED047A036870EEDE
:10846000277A9A42C0ED037A77EEC77AC0ED037A95
:108470000CDA013307EE103AF8EEC76AB7EE007A6D
:1084800087EEA60A036030EE070A704707EE102A4F
:10849000B8EEC77A87EE870A704700BF90ED057A7D
:1084A00090ED004AD0ED066AD0ED014AD0ED047A95
:1084B00090ED035AD0ED025AA4EE007AB0EE406A75
:1084C000B0EE470AB0EE667AA6EE247A67EEC07A7E
:1084D000A0EE457AE6EE257A80ED057AC0ED067AC3
:1084E000704700BFD0ED057A90ED013AD0ED003A2B
:1084F000D0ED064A90ED024A90ED077A90ED035ACE
:1085000090ED086AD0ED045AC0ED067AF0EE406AAC
:1085100027EE830AC0ED056AA3EEA60A80ED087A6D
:10852000A4EE240AA5EE470AA5EEC60A80ED070AC6
:10853000704700BFD0ED007A90ED017A30EE670A07
:10854000E7EE007AB0EE670AC0ED007A704700BF30
:10855000704700BF0A44914214D030B40139551E0F
:1085600041F2210211F8014F082380EA042004049B
:108570004CBF82EA40004000013B80B2F7D18D42FF
:10858000F0D130BC704700BF4FF400638382704766
:108590004FF400638382704750F8043C012280F856
:1085A0004520103803B11847704700BFBFF34F8F05
:1085B0000549064BCA6802F4E0621343CB60BFF37F
:1085C0004F8F00BFFDE700BF00ED00E00400FA059B
:1085D000F8B5057B466903681F2D29D9A5F120044C
:1085E0005F682021A1400F422A4613D01022A240EA
:1085F000D960DA605A68E240D10703D5012202FA55
:1086000004F4DC6004463046FFF7FAFC227B236862
:108610001F2A20D9A2F1200008215A688140114266
:1086200000D0D9600422596882400A4221D1F8BDA5
:1086300020211C68A9400C422A460CD01022AA40D6
:1086400099609A601A68EA40D207DBD5012202FAE3
:1086500005F59D60D6E7082118689140014200D0D9
:1086600099600421186801FA02F2024203D09A606C
:10867000F8BDDA60F8BDF8BD70B4037B04681F2B49
:1086800008D9203B2021626801FA03F31A421CD169
:1086900070BC70472021226801FA03F31A42F7D018
:1086A00042691449582000FB021251685689CD686E
:1086B0000868296821F001012960828992B222EAC2
:1086C00006028281A36070BC704742690949582044
:1086D00000FB021251685689CD680868296821F0AC
:1086E00001012960828992B222EA06028281E36056
:1086F00070BC70474464002030B4094B1C786CB1E6
:10870000084A002502EBC404116893884D628889E9
:10871000083203439BB2A2428B81F5D130BC704733
:10872000046700200867002070B5044682B014304A
:10873000E56D06236A464321A847B0B19DF80400C1
:108740009DF800609DF801109DF802509DF80320EF
:108750009DF8053041EA062143EA002342EA05225A
:10876000A187E287A4F84030012002B070BD00BFAD
:1087700070B5044682B00830656A06236A463B211C
:10878000A847A8B19DF804009DF800609DF801106D
:108790009DF802509DF803209DF8053041EA06211E
:1087A00043EA002342EA0522E18222836383012017
:1087B00002B070BD30B50446406D61718389A26816
:1087C00023F400531B041B0C838185B0A379009212
:1087D00013F004022ED04FF4805213F00203ADF8D0
:1087E00004203CD1ADF806304FF480630022ADF890
:1087F000083011F00103ADF80C2026D1ADF80A3095
:1088000008238A07694648BFADF80A3026F0D2FB34
:10881000A379626D13F0080F938A1BD123F008032C
:108820001B041B0C938293899BB243F400539381E6
:1088300005B030BD13F00203ADF8042012D04FF4A0
:1088400000551346ADF80650D0E70423ADF80A30C2
:108850000C23D6E79BB243F008039382E3E74FF47F
:108860000053BFE7ADF80630C0E700BF10B50446BF
:10887000406DA160838923F400531B041B0C83818A
:10888000A37984B013F00402009133D04FF48052E6
:1088900013F00203ADF804203CD1ADF806304FF4DC
:1088A00080636279ADF80830D1074FF00003ADF86E
:1088B0000A30ADF80C3045BF0423ADF80A30082368
:1088C0000C236946920748BFADF80A3026F072FBC8
:1088D000A379626D13F0080F938A16D123F0080371
:1088E0001B041B0C938293899BB243F40053938126
:1088F00004B010BD13F00203ADF804200DD04FF406
:1089000000511346ADF80610CBE79BB243F00803C5
:108910009382E8E74FF40053BFE7ADF80630C0E7B5
:1089200000B5002183B00A2025F00AFD0F210A209E
:1089300025F006FD01AA0321102025F029FD9DF94F
:108940000430DFED277ADFED275A06EE103A9DF965
:10895000053006EE903A9DF9063007EE103AB8EE73
:10896000C66AF8EEE66AB8EEC77A76EEE76A36EEE1
:10897000676A37EE677AF7EE007AB0EE675AA6EECE
:10898000255A194B0021B0EE456AB0EE675AA6EEA3
:10899000A55A0A20E7EE257AF3EE0E5A26EE256A4E
:1089A00025EE257A67EEA57A83ED006A83ED017ADC
:1089B000C3ED027A25F0C4FC0DF10302012102206F
:1089C00025F0E6FC0DF103020121092025F0E0FC71
:1089D00001210A2025F0B4FC012003B05DF804FB5E
:1089E000000000430000803B0000002070B582B012
:1089F00004466946143025F0C3FAB0B19DF805006D
:108A00009DF801609DF802109DF803509DF8042028
:108A10009DF8063041EA062143EA002342EA052296
:108A2000A187E287A4F84030012002B070BD00BFEA
:108A30002DE9F04FDFF830C1474A4849484E494DCB
:108A40008046102718F1FF38C0F08480DCF804302D
:108A5000C3F30803002B5CD1EFF31183002B58D133
:108A60000B68946800BF08688342F9D1D6F800907B
:108A70004FF47A7000FB09FEAEEB040EBEFBF9FE6C
:108A800000FB03EEDCF80430C3F308034FF47A7400
:108A90000120FBB9EFF31183E3B90B68D2F808A00A
:108AA00000BFD1F800904B45F7D1D6F800B004FBD9
:108AB0000BF9A9EB0A09B9FBFBF904FB0393A3EB40
:108AC0000E03B3F57A7FBDD2DCF80430C3F308039C
:108AD000002BDFD0EFF3118A87F31288D2F808B0A9
:108AE0001368DB0344BF2860D2F808B00B68D5F8E0
:108AF00000905FFA8AFA8AF31188D6F800A09944A8
:108B000004FB0AF3A3EB0B03B3FBFAF304FB0933F7
:108B1000D5E7EFF3118487F31288D2F80890136831
:108B2000D80303D501232B60D2F808900B6828687E
:108B3000E4B284F31188D6F800A04FF47A7400EB05
:108B4000030E04FB0AF3A3EB0903B3FBFAF304FBE4
:108B50000E3E97E7BDE8F08F10E000E0E8760020D9
:108B6000EC760020E476002000ED00E0204B5B680E
:108B7000C3F3080330B4BBB9EFF31183A3B91D4BA2
:108B80001D4C1868A16800BF1A689042F9D11B4BB0
:108B90001C684FF47A7202FB04F3591AB1FBF4F12A
:108BA00030BC02FB00107047EFF31182102383F3F7
:108BB000128811498C680B6813F4803F104B02D067
:108BC000012018608C680B49D2B20D68186882F3D6
:108BD00011880A4B19684FF47A72284402FB01F39A
:108BE0001B1B30BCB3FBF1F302FB0030704700BF2E
:108BF00000ED00E0E876002010E000E0EC760020D8
:108C0000E47600202DE9F84F8046FFF7AFFF254EB0
:108C10002549DFF8A0E0254A254D844610274FF46A
:108C20007A740120DEF80430C3F30803D3B9EFF3FC
:108C30001183BBB90B68D2F808A000BFD1F800902F
:108C40004B45F7D1D6F800B004FB0BF9A9EB0A09A4
:108C5000B9FBFBF904FB0393A3EB0C034345E1D3FE
:108C6000BDE8F88FEFF3118A87F31288D2F808B0C5
:108C70001368DB0344BF2860D2F808B00B68D5F84E
:108C800000905FFA8AFA8AF31188D6F800A0994416
:108C900004FB0AF3A3EB0B03B3FBFAF304FB093366
:108CA000DAE700BFEC760020E876002010E000E074
:108CB000E476002000ED00E008B5FFF757FF044B15
:108CC0005B68C01AC0F5FA5020EAE07008BD00BF2A
:108CD0001877002030B4EFF31183102282F312884A
:108CE0000649074C0A680748013200250A602560DA
:108CF000DBB2026883F3118830BC7047E87600204D
:108D0000E476002010E000E038B5254B9C68236B2A
:108D100073B1636D626BCAB1998A1A88C90592B240
:108D200001D5D20700D438BD4FF6F7721A8038BD8E
:108D3000636D99891A88890692B2EBD59206E9D5B6
:108D4000E26ACAB1988880B29047E2E799891A88A6
:108D50000D0692B2E0D51006DED5A26A616A8A429B
:108D600019D0A1692569885C98800132B2FBF5F1C0
:108D700005FB1122A262CFE79B88E2696169DBB241
:108D80008B54E269E068636D0132B2FBF0F100FBE5
:108D90001122E261BEE7DA6822F08002DA60BBE706
:108DA000782D002038B5254B5C68236B73B1636D5B
:108DB000626BCAB1998A1A88C90592B201D5D207E5
:108DC00000D438BD4FF6F7721A8038BD636D9989AB
:108DD0001A88890692B2EBD59206E9D5E26ACAB141
:108DE000988880B29047E2E799891A880D0692B276
:108DF000E0D51006DED5A26A616A8A4219D0A1695F
:108E00002569885C98800132B2FBF5F105FB1122DF
:108E1000A262CFE79B88E2696169DBB28B54E269A9
:108E2000E068636D0132B2FBF0F100FB1122E261F8
:108E3000BEE7DA6822F08002DA60BBE7782D002016
:108E400003682DE9F041DF691FB13B46BDE8F04101
:108E50001847002A164611DD04460D460E4400E070
:108E600023689B68204698470028F9D0236815F8A6
:108E7000011B1B6820469847AE42F1D1BDE8F08146
:108E800003689B69184700BF03685B69184700BF08
:108E900003681B69184700BF0368DB68184700BFF9
:108EA00003685B68184700BF03681B68184700BF6A
:108EB000014B1868F8E700BF8067002038B50C4602
:108EC000097849B1054601342B6828461B68984744
:108ED00014F8011B0029F7D138BD00BF064B53F829
:108EE00020302BB11A689B8851690B4201D1138342
:108EF00070475383704700BF4C67002003682DE91B
:108F0000F04F03F13F4404F57E04604EA40A0125AE
:108F1000345D04F01F066409032C05FA06F500F021
:108F2000AF80042C00F0A780022C54D08588B5FABD
:108F300085F0C0F11F0080B2C40803EB840400F088
:108F40000700266A80000F27874026EA0706266268
:108F5000276A01F0030602FA00F0721E3843012A64
:108F6000C1F3810CC1F300182062C1F3411137D95C
:108F70000024224601274FF0030E03E0102A04F1DB
:108F8000020426D007FA02F0A84302F10102F5D14B
:108F9000D3F800C00EFA04F0C04300EA0C0CC3F88A
:108FA00000C0D3F8008006FA04FC4CEA080CC3F8B1
:108FB00000C0D3F80CC000EA0C00D860D3F80CC095
:108FC00001FA04F040EA0C00102AD86004F102040F
:108FD000D8D1BDE8F08F2E4C666C35436564A5E7AB
:108FE000002002464FF0010E4FF0030904E0013269
:108FF000102A00F102003CD00EFA02F737EA05040D
:10900000F5D1D3F800A009FA00F4E4430AEA040A0F
:10901000C3F800A0D3F800B006FA00FA4AEA0B0A37
:10902000C3F800A0D3F808A004EA0A0AC3F808A00D
:10903000D3F808B00CFA00FA4AEA0B0AC3F808A001
:10904000D3F804A02AEA07075F60D3F804A008FA5F
:1090500002F747EA0A075F60DF683C40DC60DF68D0
:1090600001FA00F401323C43102ADC6000F10200F6
:10907000C2D1BDE8F08F064C266B3543256355E71A
:10908000034C266C3543256450E700BF98830308E2
:1090900000380240026802F13F4303F57E032DE9E8
:1090A000F04F9B0A544DEB5C03F01F055B09012454
:1090B000032B04FA05F400F09980042B00F0918052
:1090C000022B3ED001F00306731E012BC1F3810C6D
:1090D000C1F300188588C1F3411137D90024234614
:1090E00001274FF0030E03E0102B04F1020426D0F9
:1090F00007FA03F0A84303F10103F5D1D2F800C049
:109100000EFA04F0C04300EA0C0CC2F800C0D2F81A
:10911000008006FA04FC4CEA080CC2F800C0D2F841
:109120000CC000EA0C00D060D2F80CC001FA04F0C8
:1091300040EA0C00102BD06004F10204D8D1BDE845
:10914000F08F2E4B5D6C2C435C64BBE70020034624
:109150004FF0010E4FF0030904E00133102B00F132
:1091600002003CD00EFA03F737EA0504F5D1D2F835
:1091700000A009FA00F4E4430AEA040AC2F800A0D5
:10918000D2F800B006FA00FA4AEA0B0AC2F800A0C8
:10919000D2F808A004EA0A0AC2F808A0D2F808B077
:1091A0000CFA00FA4AEA0B0AC2F808A0D2F804A0A6
:1091B0002AEA07075760D2F804A008FA03F747EA3B
:1091C0000A075760D7683C40D460D76801FA00F4BA
:1091D00001333C43102BD46000F10200C2D1BDE842
:1091E000F08F064B1D6B2C431C636BE7034B1D6C10
:1091F0002C431C6466E700BF9883030800380240D4
:1092000010B50409013C032C17D80D4B33F814207A
:1092100000F00F0042FA00F313F001030DD0012318
:1092200003FA00F0013810402AF0ECFA054A064B28
:10923000125D104403EBC00010BD002010BD00BF44
:10924000508703084C870308147500202DE9F04F60
:109250004A484B494B4B4C4C4FF0010A4FF0020926
:109260004FF004084FF0080C4FF0100E2027402656
:10927000802530F8022B12F0010F03D01960A3F8FB
:1092800004A0083312F0020F03D01960A3F8049071
:10929000083312F0040F03D01960A3F804800833D8
:1092A00012F0080F03D01960A3F804C0083312F0BD
:1092B000100F03D01960A3F804E0083312F0200F58
:1092C00002D019609F80083312F0400F02D019605D
:1092D0009E80083312F0800F02D019609D80083301
:1092E00012F4807F05D04FF4807B1960A3F804B09E
:1092F000083312F4007F05D04FF4007B1960A3F807
:1093000004B0083312F4806F05D04FF4806B1960FD
:10931000A3F804B0083312F4006F05D04FF4006BCB
:109320001960A3F804B0083312F4805F05D04FF43D
:10933000805B1960A3F804B0083312F4005F05D015
:109340004FF4005B1960A3F804B0083312F4804FA7
:1093500005D04FF4804B1960A3F804B00833D20B4A
:1093600004D04FF4004219609A80083301F58061FF
:10937000A1427FF47EAFBDE8F08F00BF50870308A5
:1093800000000240147500200010024000286AD03E
:1093900003682DE9F04F03F13F4404F57E045F4E6E
:1093A000A40A0125345D04F01F066409032C05FAA4
:1093B00006F559D0042C00F0AC80022C59D08588D9
:1093C000B5FA85F0C0F11F0080B2C40803EB840435
:1093D00000F00700266A80000F27874026EA07066C
:1093E0002662276A01F003068240701E3A43012874
:1093F000C1F3810CC1F300182262C1F341113DD9C0
:109400000024224601274FF0030E03E0102A04F146
:10941000020426D007FA02F0A84302F10102F5D1B6
:10942000D3F800C00EFA04F0C04300EA0C0CC3F8F5
:1094300000C0D3F8008006FA04FC4CEA080CC3F81C
:1094400000C0D3F80CC000EA0C00D860D3F80CC000
:1094500001FA04F040EA0C00102AD86004F102047A
:10946000D8D1BDE8F08F70472D4C266C354325646C
:10947000A5E72B4C666C35436564A0E700200246E7
:109480004FF0010E4FF0030904E00132102A00F101
:1094900002003CD00EFA02F737EA0504F5D1D3F802
:1094A00000A009FA00F4E4430AEA040AC3F800A0A1
:1094B000D3F800B006FA00FA4AEA0B0AC3F800A093
:1094C000D3F808A004EA0A0AC3F808A0D3F808B041
:1094D0000CFA00FA4AEA0B0AC3F808A0D3F804A071
:1094E0002AEA07075F60D3F804A008FA02F747EA00
:1094F0000A075F60DF683C40DC60DF6801FA00F467
:1095000001323C43102ADC6000F10200C2D1BDE808
:10951000F08F034C266B3543256350E7988303088F
:1095200000380240002855D0026802F13F4303F59D
:109530007E032DE9F04F9B0A544DEB5C03F01F05B1
:109540005B090124032B04FA05F444D0042B00F03A
:109550009780022B44D001F00306731E012BC1F348
:10956000810CC1F300188588C1F341113DD9002455
:10957000234601274FF0030E03E0102B04F10204F1
:1095800026D007FA03F0A84303F10103F5D1D2F87E
:1095900000C00EFA04F0C04300EA0C0CC2F800C090
:1095A000D2F8008006FA04FC4CEA080CC2F800C0AD
:1095B000D2F80CC000EA0C00D060D2F80CC001FA5E
:1095C00004F040EA0C00102BD06004F10204D8D162
:1095D000BDE8F08F70472E4B1D6C2C431C64BAE71E
:1095E0002B4B5D6C2C435C64B5E7002003464FF0C9
:1095F000010E4FF0030904E00133102B00F10200CB
:109600003CD00EFA03F737EA0504F5D1D2F800A0F2
:1096100009FA00F4E4430AEA040AC2F800A0D2F806
:1096200000B006FA00FA4AEA0B0AC2F800A0D2F823
:1096300008A004EA0A0AC2F808A0D2F808B00CFA96
:1096400000FA4AEA0B0AC2F808A0D2F804A02AEAF3
:1096500007075760D2F804A008FA03F747EA0A0799
:109660005760D7683C40D460D76801FA00F40133F2
:109670003C43102BD46000F10200C2D1BDE8F08F52
:10968000034B1D6B2C431C6365E700BF98830308E5
:109690000038024038B5044690F8590000285AD1E5
:1096A00004F11405236E80226B212846984764201C
:1096B000FFF7BEF9236E07226821284698476420E9
:1096C000FFF7B6F9236E00226B21284698476420E5
:1096D000FFF7AEF9236E01226B21284698470F2031
:1096E000FFF7A6F994F85320236E032A8CBF1A22A1
:1096F00018221B21284698470F20FFF799F9236E5F
:1097000018221C21284698470F20FFF791F9236E55
:1097100094F852201A21284698470F20FFF788F91D
:10972000236E94F854201921284698476420FFF7A7
:109730007FF9236E10223721284698470F20FFF724
:1097400077F92846236E0122382198470F20BDE87B
:109750003840FFF76DB9FFF753FD0546F0B10368D8
:1097600081881B6919409BD12023C1718371FFF748
:10977000D9FE21460F4B41F8103F284624F094FBB8
:10978000AB88B3FA83F3C3F11F03012212FA03F388
:1097900086D009490A6813430B6081E70146FFF749
:1097A000C1FE2146034B41F8103F284624F07CFBC4
:1097B00076E700BF99850008003C014010B10368BE
:1097C00082885A83704700BF10B1036882881A8369
:1097D000704700BF18B10368828809B95A8370477F
:1097E0001A83704710B40A4B0A4A1C78012383403D
:1097F000234052F8200029B9B3FA83F149095DF8F2
:10980000044BE7E7191C18BF01215DF8044BE1E7A1
:10981000496700204C6700202DE9F0410B4E346869
:1098200073691C400FD0DFF828800127B4FA84F355
:10983000C3F11F0307FA03F558F82300036898479C
:10984000AC437561F2D1BDE8F08100BF003C01403E
:109850009C7600202DE9F0410B4E346873691C4062
:109860000FD0DFF828800127B4FA84F3C3F11F0377
:1098700007FA03F558F8230003689847AC4375616D
:10988000F2D1BDE8F08100BF003C01409C76002091
:109890002DE9F0410B4E346873691C400FD0DFF89E
:1098A00028800127B4FA84F3C3F11F0307FA03F5F4
:1098B00058F8230003689847AC437561F2D1BDE8BE
:1098C000F08100BF003C01409C7600202DE9F04172
:1098D0000B4E346873691C400FD0DFF828800127D5
:1098E000B4FA84F3C3F11F0307FA03F558F8230011
:1098F00003689847AC437561F2D1BDE8F08100BFC1
:10990000003C01409C7600202DE9F0410B4E34686C
:1099100073691C400FD0DFF828800127B4FA84F364
:10992000C3F11F0307FA03F558F8230003689847AB
:10993000AC437561F2D1BDE8F08100BF003C01404D
:109940009C7600202DE9F0410B4E346873691C4071
:109950000FD0DFF828800127B4FA84F3C3F11F0386
:1099600007FA03F558F8230003689847AC4375617C
:10997000F2D1BDE8F08100BF003C01409C760020A0
:109980002DE9F0410B4E346873691C400FD0DFF8AD
:1099900028800127B4FA84F3C3F11F0307FA03F503
:1099A00058F8230003689847AC437561F2D1BDE8CD
:1099B000F08100BF003C01409C760020084A094825
:1099C00008B5536C43F480435364002140222CF0CB
:1099D00093FA054B4FF0FF321A60C3F8032008BD1D
:1099E000003802409C760020DC7600202DE9F04112
:1099F000044618460D461646984629F059FA276837
:109A0000E6722844A07229467D69434632462046C4
:109A1000AC46BDE8F0416047036810B504461B68DA
:109A20009847236820469B689847A37B0133A3731C
:109A300010BD00BF144B984224D003F580639842B8
:109A400020D0028822F040021204120C0280028808
:109A500022F038031B041B0C59B141F4807100291A
:109A600091FAA1F2B2FA82F108BF4FF0FF31013949
:109A7000C9000B439BB2038003889BB243F04003B1
:109A8000038070474908DCE70038004010B58021AA
:109A900004468069FFF7CEFF0120FFF7B3F82046A8
:109AA000FFF7F8FD10226A2104F11400FEF7C4FB51
:109AB0006420FEF7BDFFA0690421FFF7BBFF012072
:109AC000BDE81040FFF79EB8F0B484894FF6FF76EA
:109AD0004FF47A7413B300292FD00F78013101E0CD
:109AE000B44218D00589013CAD07A4B2F8D5BCB288
:109AF00084814FF47A7402E0BCB2B4420BD0058981
:109B0000ED0704F1FF37F7D58589ADB20AB11570BD
:109B10000132013BDEE70A4B984202D00120F0BC43
:109B20007047084A538B01339BB25383508B80B2EA
:109B3000003018BF0120F0BC7047FF27D2E700BFFC
:109B400000380040E474002070B50646806810B10B
:109B500004688088608341F08001706840F2E934D5
:109B600000E0E4B10589013C15F0020FA4B2F8D081
:109B700089B2818140F2E93100E081B10489013983
:109B800014F0010F89B2F8D081890021FFF79CFF02
:109B9000B36813B11A689B881383012070BD05490F
:109BA0008842F2D1044C618B013189B26183618BAF
:109BB000EBE700BF00380040E474002038B50B4CE0
:109BC0002378054653B90A4A6378106849212A4622
:109BD00000252570FFF7B8FF012038BDFFF76CF8AE
:109BE0000028F0D0FFF70EF8EDE700BF187700204F
:109BF00014770020F0B54A4C2578012D83B013D09E
:109C000028D3022D0DD1474B1B780646002B77D168
:109C10006846FFF7D3FF20B19DF8063013F003002C
:109C200022D0002003B0F0BD3E4E3378002B62D12D
:109C30006846FFF7C3FF9DF8003008B1DB0764D426
:109C40000023237033784BB10023013300202370AD
:109C500003B0F0BD334E3378002BF5D10121022043
:109C600024F0C4FB2378F0E79DF801E09DF8001094
:109C70009DF803709DF802209DF805509DF8043072
:109C8000207041EA0E2142EA072243EA052309B285
:109C900012B21BB2494252425B42234806EE901A6E
:109CA00007EE102A07EE903A90ED005AD0ED015AD7
:109CB00090ED026AF8EEE66AB8EEC77AF8EEE77A57
:109CC00066EE856A27EE257A67EE867AFDEEE66A0D
:109CD000BDEEC77AFDEEE77A16EE901A17EE102A5F
:109CE00017EE903A31807280B38001210A2024F06F
:109CF00027FB03B0F0BDFEF7DFFF002898D090E708
:109D0000FEF7DAFF00288CD182E7337823B90721E8
:109D1000032024F06BFB25780135257081E700BF17
:109D2000E41D00201877002000000020427A02B9CC
:109D3000704710B504460368406804F10A0198476B
:109D40000023637210BD00BF437A5A1C0344D2B291
:109D500042729972037A934200D802B9704710B5E3
:109D600004460368406804F10A01984700236372BF
:109D700010BD00BF302827D0312827D0322827D067
:109D8000332827D0342827D0352827D0202827D09B
:109D9000212827D0102827D0112827D0122827D0F3
:109DA000132827D0142827D0152827D0162805D007
:109DB000172808BF0F2202D0002070470E22104B38
:109DC00003EB4203587C70470022F8E70122F6E7D4
:109DD0000222F4E70322F2E70422F0E70522EEE78D
:109DE0000622ECE70722EAE70822E8E70922E6E78D
:109DF0000A22E4E70B22E2E70C22E0E70D22DEE78D
:109E00006060030870B5448806460D46C4F30B0431
:109E10002246002128462CF06FF83369094A934204
:109E200009D3094A934206D2224628461946BDE87C
:109E300070402CF03CB823B121462846BDE8704064
:109E4000184770BD840500087206000838B5054C37
:109E5000054DAC4200D338BD61682046FFF7D2FF04
:109E60001434F6E78801000884050008064B07490A
:109E70008B4202D30023184670471A88C2F30B02A4
:109E80009042F8D01433F3E78801000884050008F5
:109E9000024A136823EA000010607047386200200D
:109EA000F8B5174D2B78A32B28D16B78BE2B25D175
:109EB000022229464FF6FF70FEF74CFB114FAC1CF7
:109EC00022884AB1A618BE4218D2052A16D92146C0
:109ED000FEF740FB3446F3E721460222FEF73AFB49
:109EE0000222A118FEF736FB0634074B641B1C80C8
:109EF00041F60F53C31A58425841F8BD0020F8BD2F
:109F00000040000800800008DE2D00200378202B90
:109F1000024600F10100F9D0092BF7D02D2B2CD0EF
:109F20002B2B03BF5378B7EE000A0246B7EE000AA8
:109F3000A3F13001C8B209289FED467A10D8F2EE9D
:109F4000046A07EE901AF8EEE77A12F8013FE7EE9E
:109F5000267AA3F13001C8B20928B0EE677AF0D9A9
:109F60002E2B4CD003F0DF03452B0BD0F7EE007AFD
:109F700067EE276A20EE260A70475378BFEE000A84
:109F80000246D5E710B451782D2959D02B290ABFA4
:109F90009178501C901C0024A1F13003092B53D858
:109FA000002303EB830301EB430310F8011FA1F12E
:109FB0003002092AA3F13003F3D9B3F59A7F28BF01
:109FC0004FF49A73072B42D9DFED236A1A46F7EE56
:109FD000007A083A072A67EEA67AFAD803F0070350
:109FE0002BB1F2EE046A013B67EEA67AFBD124B3F3
:109FF000C7EE276A5DF8044B20EE260A70475378B7
:10A00000A3F13001C8B2092802F10102AAD8F2EE88
:10A01000046AF0EE665A07EE901AF8EEE77A12F844
:10A02000013F87EEA66AA3F13001C8B2092866EEA7
:10A03000A56A37EE067AEED994E767EE276AD9E784
:10A04000901C91780124A7E7F7EE007ACFE7F7EEAE
:10A05000007AC5E70000000020BCBE4CB5EEC00A87
:10A06000DFED317AF1EE10FACCBF30EE270A30EE98
:10A07000670ADFED2E7A20EE270A30B5FDEEC07AB2
:10A0800087B017EE904A054684EAE470002303A9DE
:10A09000A0EBE4700193009302931CF0E9FA002C0A
:10A0A000ACBF20232D2303A88DF8003028F000FF3B
:10A0B000012803A924D002282DD0032805BF30236E
:10A0C000684668468DF801302BF03CFF684628F062
:10A0D000EFFE0338C4B22246694628462BF090FFB3
:10A0E00000232B55284628F0E3FE2E22431C2A5439
:10A0F0000DEB0401E8182BF042FF284607B030BDF5
:10A10000302368468DF801308DF802308DF8033029
:10A110002BF018FFDAE7302368468DF801308DF810
:10A1200002302BF00FFFD1E76F12033A00007A44A0
:10A130002DE9F041064615460846B6FBF2F43CB957
:10A1400005FB1464124B1B5D00F8013BBDE8F08178
:10A15000B4FBF2F767B90E4B05FB174705FB146418
:10A16000DA5D00F8012B1B5D00F8013BBDE8F081D2
:10A17000B7FBF2F8B8F1000F02D04046FFF7D8FF66
:10A1800005FB1878024B13F8082000F8012BE3E7D1
:10A190006888030830B402681146531C036011F844
:10A1A000024B0160D31C517803609378151D056044
:10A1B0001B0443EA0123D078234343EA006030BC08
:10A1C000704700BF0368591C1A46016012F8021B51
:10A1D0000260587841EA0020704700BF03685A1CAB
:10A1E00002601878704700BF38B50446006815460D
:10A1F0002BF05DFE22682A44226038BD036810B44B
:10A200000A0E5C1C04601A7003680A0C5C1C046073
:10A210001A7003680A0A5C1C04601A7003685A1CEE
:10A22000026019705DF8044B704700BF036810B4FA
:10A230000A0A5C1C04601A7003685A1C02601970D8
:10A240005DF8044B704700BF03685A1C026010B4ED
:10A25000197003680A0A5C1C04601A7003680A0C0F
:10A260005C1C04601A700368090E5A1C02601970A5
:10A270005DF8044B704700BF03685A1C02601970F8
:10A280000368090A5A1C0260197070472DE9F047EB
:10A29000002488B080460F461E46A14605AD531CDB
:10A2A0000393117839B3252933D1931CCDF810903D
:10A2B0000393507830284ED04FF0000AA0F13003BD
:10A2C000DBB2092B42D96C2819D0642800F09380A6
:10A2D00024D825281CD063D9582876D063281BD1D0
:10A2E00031784046B847039A531C039311780436DB
:10A2F00001340029D7D1204608B0BDE8F087039B80
:10A300005A1C03921B78642B7CD02AD8252B54D15D
:10A31000252140460134B847039AC0E7732833D05B
:10A3200044D975284FD106F1040E30682B4600221F
:10A330000A217646FEF704F8049A009553463946FA
:10A340004046FEF73BF8039A0444A8E704AA03A991
:10A350001CF06AF9B7E7D31C039390784FF0010A19
:10A36000ACE7732B10D05BD9752B3AD0782B96D1F4
:10A37000A3F15802B2FA82F2306852092B4610213A
:10A380000436FDF7DDFFD7E73368049A00933946BA
:10A3900000234046FEF712F804360444039A7EE791
:10A3A0000028B9D1204608B0BDE8F0876E28B3D1A7
:10A3B000039A336804361C6071E72AD9582BD7D02A
:10A3C000632B8DD06BE77828A6D1A0F15802B2FAA2
:10A3D00082F2306852092B461021FDF7B1FF043696
:10A3E000AAE706F1040E30682B4600220A217646C1
:10A3F000FDF7A6FFA0E7331D306829461E46FDF78E
:10A4000071FF99E7331D306829461E46FDF76AFF44
:10A4100092E7002B7FF443AF204608B0BDE8F087F9
:10A420006E2BC6D03BE700BF0EB400B584B005ABC1
:10A43000019053F8042B0649039301A8FFF726FF68
:10A44000019B00221A7004B05DF804EB03B0704762
:10A45000B18300080FB430B583B006AB0A490B488E
:10A4600053F8042B096800680193FFF70FFF084CAD
:10A4700005462068FEF708FD0028FAD0284603B0FC
:10A48000BDE8304004B070476C2D0020702D0020D6
:10A4900080670020DFED2B7AB4EEE70AF1EE10FAC8
:10A4A0004ADDDFED296A9FED297A01E0B0EE670A07
:10A4B000B4EEC70AF1EE10FA70EE667AF6DC9FEDA4
:10A4C000247AF4EEC77AF1EE10FA38D5DFED1E6A81
:10A4D0009FED207A01E0F0EE407AF4EEC77AF1EEDB
:10A4E00010FA37EEA60AF6D4DFED1B7AB4EEE70ACF
:10A4F000F1EE10FA14DDDFED137A37EEC00A60EEEC
:10A50000006A9FED166A9FED167ADFED167AA6EEC9
:10A51000867A20EE266AE6EE877AA6EE270A70474C
:10A52000DFED117AB4EEE70AF1EE10FA44BFDFED89
:10A53000087A37EEC00AE2E7F0EE407ABFE7B0EE05
:10A54000670AD1E7DB0F4940DB0FC940E4CB164176
:10A55000DB0F49C0E4CB16C1DB0FC93F92E741B91D
:10A560009730083C15A82ABEDB0FC9BF09B909E01E
:10A57000194690FBF1F301FB13030846002BF7D1BA
:10A58000084670470146FBE7F0EEC07AB0EEE07A8D
:10A59000B4EEE77AF1EE10FAB4BFB0EE676AB0EE4F
:10A5A000476AB5EE406AF1EE10FA46D0B4EEE77AAB
:10A5B000F1EE10FA8CBFF0EE675AF0EE475AC5EE96
:10A5C000866A9FED1F3A9FED1F6A9FED1F4A9FED20
:10A5D0001F5ADFED1F3ADFED1F4ADFED1F5AA6EECF
:10A5E000C36AE6EEA34AA6EE864AB7EE006AA6EE76
:10A5F000845AA6EEA46AE6EE855AC5EE866AB4EEE3
:10A60000E77AF1EE10FA48BFDFED147AF5EEC00AF2
:10A6100048BF77EEE66AF1EE10FA48BFDFED107A38
:10A62000B5EEC00A48BF77EEE66AF1EE10FA48BF11
:10A63000F1EE666AB0EE660A7047DFED076ADEE7A4
:10A6400039094E3DE3B59E3E88FA163E45FE7F3FF2
:10A6500099FB243F69A2163EA7DFA834DB0FC93F50
:10A66000DB0F4940DFED317A30EE277AFDEEC76A25
:10A6700016EE903A2033402B02D99FED2D0A7047F9
:10A68000B4EEE70AF1EE10FA4DDD9FED2A6ADFED38
:10A690002A6A01E0B0EE677AB4EEE67AF1EE10FADB
:10A6A00077EE467AF6DC9FED257AF4EEC77AF1EE86
:10A6B00010FA35D5DFED1F6A9FED217A01E0F0EE4B
:10A6C000407AF4EEC77AF1EE10FA37EEA60AF6D425
:10A6D000DFED167AB4EEE70AF1EE10FA1BDCDFEDDF
:10A6E000197AB4EEE70AF1EE10FA44BFDFED137AFF
:10A6F00037EEC00A60EE006A9FED136A9FED137A91
:10A70000DFED137AA6EE867A20EE266AE6EE877AE9
:10A71000A6EE270A7047DFED0F7A37EEC00AE9E7A9
:10A72000B0EE670AD4E7F0EE477ABCE7DB0FC93F2B
:10A7300000000000DB0FC940E4CB1641DB0F49C02D
:10A74000E4CB16C1DB0FC9BF92E741B99730083C93
:10A7500015A82ABEDB0F4940FDEEC07A17EE903AED
:10A760002033402B51D8DFED2D7AB4EEE70AF1EE1D
:10A7700010FA50DDDFED2A6A9FED2A7A01E0B0EE93
:10A78000670AB4EEC70AF1EE10FA70EE667AF6DCEC
:10A790009FED257AF4EEC77AF1EE10FA38D5DFEDA9
:10A7A000206A9FED227A01E0F0EE407AF4EEC77A5B
:10A7B000F1EE10FA37EEA60AF6D4DFED1D7AB4EE0C
:10A7C000E70AF1EE10FA1BDCDFED1A7AB4EEE70AC5
:10A7D000F1EE10FA44BFDFED147A37EEC00A60EEF6
:10A7E000006A9FED156A9FED157ADFED157AA6EEEA
:10A7F000867A20EE266AE6EE877AA6EE270A70476A
:10A80000DFED067A37EEC00AE9E79FED0E0A7047E2
:10A81000B0EE670AD1E7F0EE407AB9E7DB0F4940C6
:10A82000DB0FC940E4CB1641DB0F49C0E4CB16C1B6
:10A83000DB0FC93FDB0FC9BF92E741B99730083C36
:10A8400015A82ABE0000000010B507EE901A2DEDE5
:10A85000028BB8EE678ADFED217A28EE008A044683
:10A8600028EE278AB0EE480A29F07AFAF0EE408AFC
:10A87000B0EE480A29F0D6F9F7EE007A9FED187A83
:10A88000F0EE675AE8EE875A0023A361B0EE676ADC
:10A89000C7EEA56A63612362E361A8EEC76ABDECF7
:10A8A000028B77EEC07AB6EE007AF8EE005A27EE09
:10A8B000877A20EE250A27EE267A26EE266A67EEAC
:10A8C000A67A20EE260A84ED046AC4ED017A84EDAE
:10A8D000007A84ED027A84ED030A10BD27D4D236C3
:10A8E000F304353F10B44C09012250F8243001F034
:10A8F0001F0102FA01F10B4340F824305DF8044BCC
:10A90000704700BF4B0901F01F0150F823200123BD
:10A9100003FA01F1114214BF18460020704700BF2E
:10A920000C4B984213D0A3F5806398420FD003F5E7
:10A93000804398420BD003F58063984207D003F51B
:10A940008063984203D0044B186840087047024B5C
:10A95000186870470004014058630020F0B5774B39
:10A96000774A87B01968914200AF00F0DB8000237E
:10A97000744A3B607B60136843F48033136003E0E8
:10A980003B68B3F5A04F09D0136803F400337B6034
:10A990003B6801333B607B68002BF1D0694B1B683F
:10A9A00013F4003318BF01237B607B68012B7BD03D
:10A9B000654D644B654AEA606549586F654A0860B1
:10A9C000AA605E6B644C654A654826F080065E634B
:10A9D0005E6F46F080765E67196B0C431C63596BA3
:10A9E0005963996B9963196C41F05B5141F47B1188
:10A9F00041F41F6141F00F011964596C07F118040B
:10AA00000A4348F2FF715A6444F8101D002621469B
:10AA10000123FB733E737E73BE7326F019FA214641
:10AA20004FF6FF734F48BB6026F012FA4FF6FF73E4
:10AA300021464D48BB6026F00BFA21464B4826F0D4
:10AA400007FA21464A4826F003FA2146494826F0EB
:10AA5000FFF92146484826F0FBF92146474826F0F1
:10AA6000F7F92146464826F0F3F9204626F012FB76
:10AA7000444B454C1B68BA6844484549A4FB034312
:10AA80009B09A0FB0202013B920CB3F1807F0A609C
:10AA900007D2404AF0200721536085F823009660D2
:10AAA00011601C37BD46F0BD264B3B4C1A6C3B4930
:10AAB00042F080521A6420680A69CD68496940F4FE
:10AAC00040402060986898609868120640F4004002
:10AAD000986042EA8512986842F48002490842F080
:10AAE0001902013942EA014240F4A05098605A60CC
:10AAF0001A6842F080721A601A689201FCD52849DF
:10AB0000104A40F205700860996821F003019960CD
:10AB1000996841F002019960936803F00C03082BD7
:10AB2000FAD145E700221A6062B61E4B1B6883F318
:10AB300008881D4B1B689847FEE700BFFCFF0120FB
:10AB4000EFBEADDE0038024000ED00E00005FA0582
:10AB50008C5B002000000008FF916700335F070056
:10AB6000000002400004024000080240000C0240C5
:10AB7000001002400014024000180240001C024075
:10AB80000020024058630020D34D621083DE1B4337
:10AB9000EC76002010E000E0007000400000002093
:10ABA000003C02400000FF1F0400FF1F08B5054BDA
:10ABB0001B6803B19847044B044A1A6072B6FDF74C
:10ABC000F5FC00BF10390020FCFF0120EFBEADDE18
:10ABD000F8B50468C4F30D0405460E4604B32F68A7
:10ABE00026F0A0FA092840F08980464C236923F416
:10ABF00040732361236943F400732361236943F0A5
:10AC0000010323613E6026F08DFA2369092823F0B1
:10AC10000103236172D12B6804332B600020F8BD3F
:10AC2000394B3A4A93422CD902F58042934227D9B4
:10AC300002F5804293422BD902F58042934229D9F2
:10AC400002F58032934227D902F50032934225D98A
:10AC500002F50032934223D902F50032934221D902
:10AC600002F5003293421FD902F5802293421DD98A
:10AC7000B3F1016F1CD305201AF0B2F9FFF796FF6C
:10AC8000082426F04FFA092814D04FF0FF30F8BD01
:10AC90001024F6E71824F4E72024F2E72824F0E74C
:10ACA0003024EEE73824ECE74024EAE74824E8E7DC
:10ACB0005824E6E7134F3B6923F440733B613B693B
:10ACC00043F400733B613B6923F0F8033B613B694C
:10ACD00043F002031C433C613B6943F480333B6116
:10ACE00026F020FA3B6923F002033B613B69092807
:10ACF00023F0F8033B613FF472AFC6E76FF0010049
:10AD0000F8BD00BF003C024000400008FF3F0008C3
:10AD1000F8B504460D468E180027B54201D12069CA
:10AD2000F8BDE368591CE160234415F8012B1A7241
:10AD30000429F2D1206918B9A1682046FFF748FF1D
:10AD40002061E760E9E72DE9F04FDFF850914E4FC1
:10AD50008BB00326A7EB09071822002104A82BF0CB
:10AD6000CBF84A4BCDF8109005971A69002A04DAFF
:10AD7000474A5A6002F188325A6001228DF8242035
:10AD8000F322DA60434B444C1B88ADF800300222BA
:10AD9000694604A8FFF7BCFF022269464FF6FF7020
:10ADA000FDF7D8FBDFF8F8A080464FF0000B5445C4
:10ADB0003BD30AAC002524F8245D0222214604A8D6
:10ADC000FFF7A6FF022221464046FDF7C3FB40BA2B
:10ADD000C043ADF80800022202A904A8FFF798FFBB
:10ADE000079878B106ABC0F10402294618442BF04D
:10ADF00083F8089818B9069904A8FFF7E9FE00231C
:10AE0000089007939DF82430089A23B11F490B69D5
:10AE100043F000430B61013E2FD0002A9CD1FFF785
:10AE20003FF860B30BB0BDE8F08F65888DF80DB0CA
:10AE3000C5F30B05AB1DADF808302388C3F30B0237
:10AE4000ADF80A201B0B062202A904A88DF80C30CD
:10AE5000FFF75EFF062202A94046FDF77BFB616813
:10AE600080462A4604A8FFF753FF616840462A46F9
:10AE7000FDF770FB1434804699E7002ACFD00520F7
:10AE80001AF0AEF8FFF792FE00800008003C024086
:10AE9000230167459060030888010008004000080E
:10AEA0008405000808B5034B1B6803B1984772B6C8
:10AEB000FDF77CFB103900202DE9F04F7A4C54F857
:10AEC000204083B0002C00F0EA80D4F85C90B9F107
:10AED000000F00F0E680D9F81050D9F80470734ED6
:10AEE000A16004F162012660616104F262264FF400
:10AEF0000071A661E16021616765A0464DB3DFF88E
:10AF0000B4C14FF0000E61464E68B54201F11C011C
:10AF100006D00EF1010EBEF1100FF5D14FF0000E6C
:10AF2000CEEBCE0E0CEB8E01DFF884C10E69DCF89F
:10AF300030E04FF00C0A4EEA060E461CCCF830E02A
:10AF400081F818A04E76D9F80810A1630437276558
:10AF500025630546D9F80C001F46164600283CD04C
:10AF6000DFF850C1002163465A68904203F11C0388
:10AF700003D001311029F7D10021C1EBC1010CEB45
:10AF800081014B4B0A69186BDFF82CE11043186301
:10AF90000B200876681C4876186B024399F81F004E
:10AFA0001A63830991F80DC08DF805300022012342
:10AFB0004C61C1F808E001A88DF806208DF8073033
:10AFC0008DF804C023F0BEFF636DD9F80810D9F8DE
:10AFD0000C2062630433E163E36494F86100FEF7DC
:10AFE0000FF9824694F86000FEF70AF9834699F853
:10AFF0001C00002850D1380739D4B2070ED5BAF159
:10B00000000F0BD00B226B1C8AF806208AF8073041
:10B01000504699F81D202221FEF7B8F9F30716D4FF
:10B02000A36B83B999F81E208DF8042099F820208D
:10B030008DF8063001A8930901228DF805308DF8AE
:10B04000072023F07FFF404603B0BDE8F08FBBF13F
:10B05000000FE5D001350C238BF807508BF8063034
:10B06000584699F81D202221FEF790F9D8E70135BE
:10B07000EDB2BAF1000F04D00B238AF807508AF81A
:10B08000063017F0100F50460CBF1221022199F81C
:10B090001D20FEF77BF9C3E722F0E4FEABE7A046F4
:10B0A000D1E7C846CFE700BF782D002094600308A1
:10B0B00000380240C8130020D18500080348D0F8AA
:10B0C000AC3113B100F5D27018477047C813002097
:10B0D0000348D0F8903113B100F5C4701847704799
:10B0E000C81300200348D0F8743113B100F5B670CE
:10B0F00018477047C81300200348D0F8583113B1DF
:10B1000000F5A87018477047C81300200348D0F80E
:10B110003C3113B100F59A7018477047C8130020EE
:10B120000348D0F8203113B100F58C7018477047F0
:10B13000C81300200348D0F804310BB1FC30184785
:10B14000704700BFC81300200348D0F8E8300BB1A7
:10B15000E0301847704700BFC81300200348D0F8FC
:10B16000CC300BB1C4301847704700BFC813002063
:10B170000348D0F8B0300BB1A8301847704700BF73
:10B18000C81300200348D0F894300BB18C30184716
:10B19000704700BFC81300200248836F0BB17030A6
:10B1A00018477047C81300200248C36D0BB15430D4
:10B1B00018477047C81300200248036C0BB13830A1
:10B1C00018477047C81300200248436A0BB11C306F
:10B1D00018477047C81300200248836803B1184716
:10B1E000704700BFC81300201549164B1648CA689F
:10B1F00010B44C691549B2FBF4F203FB02F303608F
:10B20000D1F88820124B134C42F47002C1F8882008
:10B210001A68002042F001021A6098601A6822F051
:10B22000847222F480321A605C601A684FF0006405
:10B2300022F480221A60D8608C605DF8044B70475D
:10B240000000002040420F005863002000ED00E0A5
:10B250000038024010300024044B4FF4F0700221FB
:10B260000A22D86059611A61FFF7BEBF00000020B2
:10B2700038B50B4C23688BB15A68821A002A0546F0
:10B2800004DA0CE05A68AA1A002A07DB9A682260DE
:10B2900018461A6890472368002BF3D138BD38BD93
:10B2A000446A00200B4B002210B4027203F1C00468
:10B2B000032102E0072A09DC9979890702D5197967
:10B2C000815401329C4203F11803F3D15DF8044B21
:10B2D000704700BF7486030812230370704700BFD5
:10B2E000012334213522417042710370037170478C
:10B2F00008B511F0D1F8FFF7D5FD00BF038A2DE99D
:10B30000F0478589ADB21D4029D00F4606464FF063
:10B3100000484FF00009B5FA85F328FA03F2D2434A
:10B3200091B21B3B15403182042B16D8DFE803F0A5
:10B330003129211903007B6A002B32D003F1FF3A37
:10B340001FFA8AFAC7F824903C6A34B12368204671
:10B35000514698476468002CF8D1002DDBD1BDE838
:10B36000F0873868716B036889B29847002DD2D195
:10B37000F5E77868B16B036889B29847002DCAD1A8
:10B38000EDE7B868F16B036889B29847002DC2D128
:10B39000E5E7F868316C036889B29847002DBAD1A7
:10B3A000DDE7F36A1FFA83FACEE700BF2DE9F04F1D
:10B3B0002DED028BA0F10A0389B00C46E72B00F2B9
:10B3C0007586DFE813F01C017306730673067306B7
:10B3D00073067306730673067306730673067306A5
:10B3E0007306730673067306730673067306730695
:10B3F0007306730673068D017306730673067E016A
:10B40000730673067306710173062D0173067306C6
:10B410007306730673062702730602027306EE01B3
:10B42000730673067306E801E1017306DA01730619
:10B430007306D3017306AB017306730673066304C8
:10B44000730673067306730644047306FC007306E2
:10B450004F061905730673067306730673067306A3
:10B460007306D7047306A9047306750473065B0597
:10B4700073065E067306730673067306EC02E9052F
:10B48000E105B005E8000F0370025902E2027306FD
:10B49000AB028F027306730673067306840273068B
:10B4A0007306930373067306730684036D035903CF
:10B4B00073067306730673064A03330335041504D3
:10B4C00073067306730673067306730673067306B4
:10B4D0007306730673067306730673067306EC022F
:10B4E0007306730673067306730673067306730694
:10B4F00073067306730673067306DD03730673061D
:10B500007306730673067306730673067306730673
:10B510007306730673067306730673067306730663
:10B520007306730673067306730673067306730653
:10B530007306730673067306730673067306730643
:10B540007306730673067306730673067306730633
:10B550007306730673067306730673067306730623
:10B560007306730673067306730673067306730613
:10B570007306730673067306730673067306730603
:10B5800073067306730673067306730673067306F3
:10B5900073062F022406A94E337853B1A84F002515
:10B5A00037F8021F2046FEF767FE33780135AB42BD
:10B5B000F6DC012009B0BDEC028BBDE8F08F9F4E98
:10B5C0003378002BF5D09F4F0025B846236817F835
:10B5D0001520591C21601A7098F8011001EB8101A7
:10B5E00001EB810101F2EE2189B22046FEF744FE13
:10B5F00033780135AB4208F10208E7DCD9E7924D18
:10B60000284627F055FC0028D3DD2B460544226848
:10B6100013F8011B501C9D4220601170F7D1C8E740
:10B620008A4D0B682A7A591C21601A70A98B204612
:10B63000FEF722FE298B2046FEF71EFE698B204670
:10B64000FEF71AFE2368EA7C591C21601A70A98C47
:10B650002046FEF711FEE98C2046FEF70DFE23681A
:10B66000AA7F591C21601A70236895F82020591C64
:10B6700021601A70698C2046FEF7FEFD2368EA7A85
:10B68000591C21601A70E9682046FEF7DDFD236829
:10B690002A7C591C21601A70236895F82120591CB6
:10B6A000216001201A7085E70B68694A581C1178DF
:10B6B0002060197023685278591C216001201A708B
:10B6C00078E7644D08462988FEF7D6FDA98820460C
:10B6D000FEF7D2FD20462989FEF7CEFD012069E75D
:10B6E0005D4D05F15006287820F0C6F82368027AEF
:10B6F000591C21601A7023686A78591C21601A70DD
:10B700002368AA78591C21601A702368EA780435E6
:10B71000591CAE4221601A70E5D14AE70B684C4AC9
:10B720004C4D11784D4A581C206019701168204604
:10B73000FEF78AFD2368454A591C127A21601A7067
:10B7400029882046FEF798FDA9882046FEF794FD3B
:10B7500029892046FEF790FD00212046FEF78CFD4A
:10B7600020460021FEF788FD012023E70846082235
:10B770003649FEF739FD01201CE70B68384A581C92
:10B7800091782060197095E70B6801229918216063
:10B7900010461A700EE708460021FEF755FD0120FD
:10B7A00008E7304D304E05F1280795F902102F4B70
:10B7B00093F906208A4203F1080300F07A84B34229
:10B7C000F6D10835AF42F0D1F3E6294B03F15A0523
:10B7D00022685979501C2060117022681978501C19
:10B7E0002060117022685978501C20601170226806
:10B7F0009978501C206011702268D978501C206004
:10B800001170226819790633501C9D422060117016
:10B81000DED1CEE60B680D4A591C527D2160012015
:10B820001A70C7E6134D0846E989FEF725FD204644
:10B83000A989FEF721FD0120BCE600BF8869002030
:10B8400076680020D86C0020F4610020605B002046
:10B85000883800209C2D00208C3800203862002081
:10B8600034620020187D0020D44A0020AC4A002019
:10B870000C48002018620020AD4D08462988FEF7CC
:10B88000FBFC69882046FEF7F7FCB5F90430A94AAD
:10B89000D91782FB0323C1EBA301204689B2FEF72F
:10B8A000EBFC012086E6A44B08461988FEF7E4FC71
:10B8B000A24B20461988FEF7DFFCA14B22681B78BB
:10B8C000511C03F0010321600120137072E69D49B1
:10B8D00052232268501C2060137011F8013F002B86
:10B8E000F7D166E6984800232268056803EB430118
:10B8F000561C6D5C26601570026825680A446E1C33
:10B90000527826602A70026825680A4401339278CA
:10B91000691C0A2B21602A70E6D14AE68B4D0B6820
:10B920002A68591C127821601A702B68226899784D
:10B93000531C2360002311702A6821681A440133C4
:10B940005279481C032B20600A70F5D123682A68BD
:10B95000591C127A21601A7023682A68591CD278FF
:10B9600021601A7023682A68591C127921601A70A4
:10B970002B6820465989FEF77FFC2A682368527A93
:10B98000591C21601A702A6894E600212046FEF7AF
:10B990005BFC20460021FEF76FFC01200AE6002533
:10B9A0008146DFF8D481DFF8D4B10595049506957A
:10B9B000079501214FF6FF7A05E001350B2D00F0C8
:10B9C000968318F9011F4F1C4AFA05F3F5D0DE07DC
:10B9D000F3D5BBF800302B41D807EED506A8FEF70B
:10B9E00081FFEAE75A4B0A681B785A4D511C03F055
:10B9F00002032160137023682A7D591C21601A708C
:10BA000029682046FEF720FC69682046FEF71CFCEA
:10BA100029892046FEF730FCE9892046FEF72CFCF8
:10BA20002046298AFEF728FC0120C3E50A684A4B14
:10BA3000501C19782060117022685978501C2060C1
:10BA4000117022689978501C206011702268DB7890
:10BA5000511C216001201370ACE5404D0846298A35
:10BA6000FEF70AFC698A2046FEF706FC2046A98AF2
:10BA7000FEF702FC01209DE50B68394A3949107830
:10BA8000394A5D1C2560187023688978581C20602D
:10BA9000197023689278591C216001201A7089E579
:10BAA0000A68324B32491878551C2560107022689C
:10BAB0005878551C2560107022689B78501C2060B7
:10BAC00013702046C988FEF7D7FB012072E5284D88
:10BAD00008462988FEF7D0FB69882046FEF7CCFB94
:10BAE0002046A988FEF7C8FB012063E5214D05F13A
:10BAF0006006A9882046FEF7BFFBE9882046FEF7CE
:10BB0000BBFB29892046FEF7B7FB2368AA7A591C9C
:10BB100021601A702368EA7A591C21601A7055F85E
:10BB20000C1B2046FEF790FBB542E2D141E500BF79
:10BB3000EC450020676666668C3F00208E3F002043
:10BB4000463F0020BC6003083082002008480020E7
:10BB50000C46002010460020343D00201C640020CC
:10BB6000484900201862002028620020106200204E
:10BB7000E0350020F02E0020EC600308A43F0020F8
:10BB80000B68DFF8F4C2591C9CF8002021601A7081
:10BB90009CF80030002B3FF40CADA94EA94DAA48EB
:10BBA000AA490023226816F8017F02F1010EC4F8A9
:10BBB00000E01770226815F8017F02F1010EC4F849
:10BBC00000E01770226810F8017F02F1010EC4F83E
:10BBD00000E01770226811F8017F02F1010EC4F82D
:10BBE00000E017709CF8002001339A42DADCE0E4B0
:10BBF0000B68974F591C3A7821601A703B78002BDC
:10BC00003FF4D7AC0025EEB2304624F011F923689A
:10BC10004278591C216030461A7024F009F90189D4
:10BC20002046FEF729FB3B780135AB42EBDCC0E454
:10BC3000884B8949B3F9003081FB0321DB17C3EB43
:10BC4000A101204689B2FEF717FB0120B2E40B6880
:10BC5000824D591C2A7921601A7023686A79591C0F
:10BC600021601A7029882046FEF706FB2368AA790E
:10BC7000591C21601A7069882046FEF7FDFA236876
:10BC8000EA79591C216001201A7093E40B680025A1
:10BC90005A1C0A60204629461D70FEF7D5FA29462F
:10BCA0002046FEF7D1FA29462046FEF7CDFA80E479
:10BCB0006B4E0B6872796B4D591C21601A702B68A2
:10BCC0002046198CFEF7D8FA2B682046D98BFEF750
:10BCD000D3FA71892046FEF7CFFAB1892046FEF7E4
:10BCE000CBFA2B682046598CFEF7C6FA2B68204603
:10BCF000998CFEF7C1FAF1892046FEF7BDFA318A28
:10BD00002046FEF7B9FA2A68236892F82620591CC3
:10BD1000216001201A704DE4514EF378002B00F0A1
:10BD2000B9820B680822591C21601A70236801220D
:10BD3000991821601A7023684B4D591C2A7921608B
:10BD40001A702368AA78591C21601A702988204625
:10BD5000FEF792FAE9892046FEF78EFA2368F27917
:10BD6000591C21601A702368EA78591C216001204F
:10BD70001A701FE415F02CFBFF28064600F096828F
:10BD800008A9002501F8125D0DF10D008DF80D5088
:10BD90001AF0D8FD08A800F8115D1AF0C7FD08A830
:10BDA00000F8105D1AF0B6FD08A820F8085D15F03F
:10BDB000EFFA23685A1C22601E7023689DF80D203C
:10BDC000591C21601A7023689DF80E20591C2160AF
:10BDD0001A7023689DF80F20591C21601A7023687F
:10BDE0009DF81020591C21601A702046BDF81810CB
:10BDF000FEF742FAFFF7DDBB0B681C4E01255A1C0B
:10BE00000A601D700B68B278591921601A701CF015
:10BE10000FFE2368164A17495F1927601870B1F999
:10BE20000010B2F90000FEF7A1FB23685A19226046
:10BE3000187031882046FEF71FFA2846FFF7BABB74
:10BE40004F3D00205F3D00207F3D00206F3D0020E2
:10BE5000A85E0020286200206766666638490020D8
:10BE600048490020308200201C6400207E8300208E
:10BE700050600020526000204D3D002000212046EF
:10BE8000FEF7FAF900212046FEF7F6F900212046D8
:10BE9000FEF7F2F92368B54D00265A1C22601E7089
:10BEA00023682A68591C92F82C2021601A70236894
:10BEB0002A68591C92F8362021601A7023682A6873
:10BEC000591C92F8372021601A7023685A1C22608E
:10BED0001E7023685A1C22601E7023685A1C226040
:10BEE0001E702B682046598FFEF7C6F92B68204636
:10BEF000198FFEF7C1F923682A68591C92F82E2081
:10BF000021601A7023685A1C22601E702B6820461C
:10BF1000598EFEF7B1F92B682046998EFEF7ACF9E1
:10BF20000120FFF747BB924D924E9FED938ADFF8B9
:10BF30008882DFED928A05F120070EE0FCEEE77AB9
:10BF4000CDED017ABDF8041020460435FEF794F9D2
:10BF5000AF4206F118063FF42CAB717C0029F3D0F8
:10BF6000874BD5ED007A1B78012BE7D1854B1B68F9
:10BF7000DB0440F18581F5EE407AF1EE10FA40F0F5
:10BF8000AE8140F2DC51DFE7084610227E49FEF721
:10BF90002BF90120FFF70EBB7C4B9B8AB3F5006F9A
:10BFA00000F27681B3F5806F00F29781B3F5007FE0
:10BFB00034BF01270227764D05F10C0655F8041B06
:10BFC00091FBF7F1204689B2FEF756F9AE42F5D162
:10BFD000704D714F05F10C06B5EC010AD7ED087AEA
:10BFE00080EE270A27F070FE81B22046FEF744F962
:10BFF000AE42F1D1694D05F10C0655F8041B2046FF
:10C0000089B2FEF739F9AE42F7D1FFF7D2BA644BE5
:10C0100003F1700522681978501C206011702268A5
:10C020005978501C2060117022689978501C20604B
:10C0300011702268D978501C20601170226819791B
:10C04000501C2060117022685979501C20601170BA
:10C05000226899790733501C9D4220601170D9D114
:10C06000FFF7A7BA0B6800255A1C0A601D700B6801
:10C070005A1C0A601D700B685A1C0A6029461D7004
:10C080000EE60B68474A4849D078484A5D1C25604F
:10C09000187023684979581C206019702368D27879
:10C0A000591C216001201A70FFF784BA0020FFF7A5
:10C0B00081BA23685A1C2260197029882046FEF72D
:10C0C000DBF82368EA78591C21601A7023682A7902
:10C0D000591C21601A702368AA79591C21601A70B2
:10C0E00023686A79591C21601A70FFF76ABBDFF870
:10C0F000CCA000254FF008080135C5F1200208FA50
:10C1000002F2A5F120032AFA05F6164328FA03F3F2
:10C110001E43252D06F001024FF000030BD0134300
:10C12000EAD0E8B211F0BCFE0028E5D0294606A806
:10C13000FEF7D8FBE0E71E4B1B78DA0700F1BD8065
:10C1400000251C4E2F4602E00135252D38D029460A
:10C150003046FEF7D7FB0028F6D0294606A8FEF7A2
:10C16000D1FB002840F087800137EDE730820020C6
:10C17000603800205C6300200000404200E0824400
:10C18000406400206C490020503800209C4500206D
:10C19000D445002060490020FC6C00203C38002081
:10C1A000E42F0020186200206C4700202862002045
:10C1B0008D7D0020F8670020DB9B914190E33FF4E8
:10C1C000654B664DB3F850102046FEF755F8002138
:10C1D0002046FEF751F8624B19684B0103F020022C
:10C1E000C1F340031343C1F3800243EA4203C1F3A6
:10C1F000C00243EA8203C1F3401243EAC20301F0E2
:10C20000100119432046FEF737F804A904222046FE
:10C21000FDF7EAFF23682978524A581C20601970FC
:10C2200011886429A8BF64212046FEF725F8B9F1DA
:10C23000960F47D000212046FEF71EF82168B7F17F
:10C24000190348BFA7F11203A3F3C4034A1C2260D9
:10C2500020461A460B7005A9FDF7C6FF2368424A1F
:10C26000581C10212060197020461188FDF7ECFF42
:10C270000120FFF79FB9394604A8FEF733FB73E7A7
:10C28000F4EEC87AF1EE10FA45DA4FF47A715BE613
:10C29000082790E60B68B178344A581C2060197062
:10C2A00023681278591C21601A7044E523685A1CCF
:10C2B000226001201E70FFF77DB9069B43F0010349
:10C2C00006933DE723680322591C21601A702368F6
:10C2D0006A78591C21601A70B0E704276BE6F4EE07
:10C2E000C87AF1EE10FA3FF54CAEF4EEE87AFDEEC6
:10C2F000E77AF1EE10FA17EE901A1ED86FF4F97380
:10C30000303903FB01F140F2E73391FBF3F101F225
:10C31000DB5189B218E6FDEEE77A40F2E73217EE1C
:10C32000903A303B02FB03F388FB0312D917C1EBB1
:10C33000622101F2E93189B206E640F2F313A1F578
:10C34000836103FB01F140F2E73391FBF3F101F26A
:10C35000DD5189B2F8E500BF5C0100201E8200209B
:10C3600008460020E02D0020066800200C62002016
:10C3700008B501210220FDF735FA094B1B7803F0BF
:10C380000503052B08D000210120FDF72BFA002121
:10C390000846FDF727FAFEE710F010F9F3E700BFB3
:10C3A000742D0020022810B428BF0220064C074B31
:10C3B000207000EB8001064A5DF8044BC0EBC10021
:10C3C00003EB4000106070471E8200203E82002078
:10C3D0003082002010B5FDF739FD094A094B0A49A2
:10C3E0000A4C0B48146000221A705A70086021F041
:10C3F000F5F8FEF7A8FCBDE8104021F0D7B800BF63
:10C40000308200201E820020084800203E8200204A
:10C410004683002008B521F0E1F8FEF794FCBDE862
:10C42000084021F0C3B800BF38B5484B5A899989F4
:10C43000914224BF00225A81198ADA89914224BF8D
:10C440000022DA81DA78CAB1072A41496AD091F824
:10C450005700404D012400210A282C709C70D9718E
:10C460005DD00C2807D0002A6CD0DFED3B7A072A7C
:10C470000ED00A2862D0DFED397A09E0344A92F80A
:10C4800057000A2856D00C285BD1D979DFED347AD1
:10C49000344C9FED350AA278002918BFF0EE407A9F
:10C4A000062A04D8314901EB820191ED0F0A217966
:10C4B00079B1013A032A0BD8F7EE007A87EE800AA9
:10C4C00027F002FC2388984228BF1846208038BDF8
:10C4D00038BD9B781F4A07EE103A1178B8EEC77A3C
:10C4E00067EE277A07EE101AB8EEC77A27EE277A9A
:10C4F000B4EEC70AF1EE10FAEADD80EE277AFDEE1F
:10C50000C77A17EE903A102BA8BF1023012BB8BFA3
:10C510000123DBB28B4238BF0B46137038BDDFED11
:10C52000147AA4E791F857000A2803D00C28ACD05D
:10C53000D9799AE7D979DFED0E7AA9E7DFED0D7A9F
:10C54000A6E7D979DFED047AA2E700BF48490020C9
:10C55000FC6C00200C6200206F1203396F12833ACA
:10C560000AD7A3391C6400206F120338BC6003088B
:10C570005304E9380F506E3A2DE9F047B24FB34EED
:10C5800021F02CF8BE421ED2DFF84C83DFF84C932A
:10C590004446258862197DB14A450DD2052D0BD937
:10C5A00033886188C3F30B03994200F0FA80144684
:10C5B00025886219002DEFD1716830461436FDF7D9
:10C5C00021FCBE42E4D3A24A1378A3F11701022949
:10C5D0000FD9A04911F83300002840F02781D80076
:10C5E0000144497829B19C4911F833300BB918231B
:10C5F00013709A4C6378022B84BF002363702378F6
:10C60000022B84BF00232370954B9A78042A00F0F4
:10C61000048132B91A88B2F5F07F84BF4FF4F0720A
:10C620001A80904D904A2B681A40002A00F007812A
:10C63000D80700F1ED80590400F1E5801A0700F1F8
:10C64000DD809B0400F1D380884D2B685A8C998C37
:10C65000914224BF00225A84FFF7E6FE19F0ECFB5A
:10C66000002800F0C0804FF40070FDF711FC4FF47B
:10C670008030FDF70DFC4FF40030FDF709FC4FF45E
:10C680008020FDF705FC4FF40010FDF701FC4FF092
:10C690000070FDF7FDFB4FF08060FDF7F9FB63785C
:10C6A000022B06D8724A734903EB430302EB830360
:10C6B0000B602378022B07D803EB83016E4AC3EB90
:10C6C000C10302EB43032B6011F062FC0021302216
:10C6D0006A4829F011FC28680FF090FB684B2D6820
:10C6E00003F1500102E0043399427AD01A78002A0B
:10C6F000F9D19C78D8788442F5D26249624B0A70AD
:10C7000028461D6014F0E2FD604B614A1E796149C4
:10C710006148624B1160C825642212FB0652604CCE
:10C72000406B31F8061C5A60002221809A60DA6062
:10C730001A615A619A61DA6183F8202083F8212016
:10C7400008B113F0CBF8574B9FED575A1B88574A47
:10C750009FED576A5579574C57495848086006EE7F
:10C76000903AF8EEE66A1388C5EE265A07EE103ABC
:10C7700053881279C4ED005A07EE903AB8EEC77AA2
:10C780004F4BF8EEE77A1D725A7227EE067A67EE83
:10C79000867ABDE8F04783ED017AC3ED007A20F098
:10C7A00005BF63799B077FF402AF716894F804A01A
:10C7B0003046FDF727FB3388BAEB133F04D014361D
:10C7C000BE42FFF4E5AEFEE673887068AA1FC3F3AD
:10C7D0000B039A4204F10601A8BF1A4629F067FB31
:10C7E000EDE7012289E7374814F032FE3BE736488F
:10C7F000FDF74EFB4020FDF74BFB25E73348FDF7E7
:10C8000047FB2B681DE73248FDF742FB2B6815E715
:10C810003048FDF73DFB2B680DE79A8AB2F57A7F29
:10C82000BFF4FFAE4FF47A729A82FAE6D8000C1881
:10C830006468002C7FF4D4AE17241470D0E643F063
:10C8400008032B60F4E600BF840500088801000897
:10C8500088380020987D0308C07403081E820020D9
:10C860001C64002038620020096000023082002031
:10C8700046830020084800203E82002094230020A8
:10C880008C380020E8000020C82300203849002010
:10C89000D06700201E6200209C450020E838002060
:10C8A000683C0020E4210020C0C9FB48001E002095
:10C8B00017B7D138E8210020EC4700203661023D4F
:10C8C000C8470020187D00200940000201600002D6
:10C8D00009200002086000020240000800800008F1
:10C8E00008B520F07BFEFEF72EFA20F05FFEBDE8D3
:10C8F000084041E6F0B50C2934D8DFE801F089336F
:10C9000033335E333333343333330700048C968947
:10C91000B2F802E01788734D24F480542404240CE8
:10C920000484038C8488818B23F4005321F4E64132
:10C930001B0409041B0C46EA0E06090C43EA0633E5
:10C9400041EA0721A8429BB2A4B289B200F09E80BE
:10C9500005F58065A84200F0998092688480818303
:10C9600002640384F0BD048C9589B2F802C0B2F869
:10C9700000E05C4F24F480742404240C0484038CB1
:10C980008688818B23F400731B0421F073011B0C38
:10C9900045EA0C04090443EA0423090CB8429BB29B
:10C9A000B6B241EA0E015CD04F4CA04259D0926819
:10C9B00086808183C2630384F0BD048C9589B2F8BC
:10C9C00002C0B2F800E0474E24F010042404240C06
:10C9D0000484038C8788018B23F0200321F4E64133
:10C9E0001B0409041B0C45EA0C04090C43EA04135C
:10C9F00041EA0E21B0429BB2BFB289B25DD03A4C3F
:10CA0000A0425AD092688780018382630384F0BD7C
:10CA1000048C9789B2F802E01688324D24F00104A4
:10CA20002404240C0484038C8488018B23F00203E7
:10CA30001B0421F073011B0C47EA0E0709043B435A
:10CA4000090CA8429BB2A4B241EA060125D005F523
:10CA50008065A84221D09268848001834263038468
:10CA6000F0BDD589148A578A23F4006343EA05256B
:10CA70004FF6FF332B40958826F440563C4343EA5B
:10CA8000052346EA04169BB2B6B290E7158A24F451
:10CA9000804444EA8514A4B25FE7D689158A578A90
:10CAA00023F00803334324F4407496883D4323F075
:10CAB00004032C433343A4B2CDE7D489158A568AA4
:10CAC00023F0800343EA04134FF6BF741C4093889D
:10CAD00027F44067354344EA031347EA85079BB2CE
:10CAE000BFB28FE700000140000401402DE9F04F84
:10CAF000A022002183B08A488A4CDFF84C928A4DEC
:10CB00008A4E8B4FDFF8448229F0F6F989488A492A
:10CB1000DFF83CE2DFF83CC200221359834200F008
:10CB2000D580B3F1804F00F0E580AB4200F0E480A7
:10CB3000B34200F0E380BB4200F0E280734500F0B6
:10CB4000E180634500F0E080434500F0DF80DFF8DE
:10CB500008A2534500F0DC800AF5806A534500F0D6
:10CB6000D9800AF5806A534500F0D680AAF5983A34
:10CB7000534500F0D3800AF5806A534500F0848065
:10CB80000AF5806A534508BF0D237ED01832D82A93
:10CB9000C3D1644C694E6A4F6A4D04F1D80802E073
:10CBA0001834A0456DD0A379002BF9D023794FEA32
:10CBB000131909F1FF39B9F1030F03F00F03EFD88F
:10CBC00036F8190040FA03F2D207E9D54FF0010A0E
:10CBD0000AFA03F3013B184026F014FE17F8093057
:10CBE000184415EBC002DBD055F83000DFF86CE1DB
:10CBF000217A00F13F4303F57E039B0A1EF80330C0
:10CC000003F01F0E5B09032B0AFA0EFA60D0042B07
:10CC100067D0022B07D1DFF820E1DEF844304AEA82
:10CC20000303CEF8443093880093B3FA83F3C3F13F
:10CC30001F039BB2DA0800EB820203F00703D2F86D
:10CC400020E09B004FF00F0C0CFA03FC2EEA0C0EB8
:10CC5000C2F820E0D2F820E001FA03F343EA0E0321
:10CC6000136269460023022218348DF804208DF8DF
:10CC700005308DF806308DF8073024F0E9F8A0452E
:10CC800091D103B0BDE8F08F0C2309EBC3034FF043
:10CC9000010A93F85C3003F01F0B5B09032B0AFABF
:10CCA0000BFA09D0042B0CD0022B7FF46FAF4B6C26
:10CCB0004AEA03034B6469E70B6C4AEA03030B641B
:10CCC00064E70B6B4AEA03030B635FE70023DCE7CF
:10CCD000DFF864E0DEF840304AEA0303CEF8403083
:10CCE000A1E7DFF854E0DEF830304AEA0303CEF87B
:10CCF000303098E70123C8E70223C6E70323C4E7DF
:10CD00000423C2E70523C0E70623BEE70723BCE7E9
:10CD10000823BAE70923B8E70A23B6E70B23B4E7E9
:10CD2000E02300207486030800040040000800404F
:10CD3000000C00400000014000380240508703080A
:10CD40004C87030814750020BC60030800040140F0
:10CD50000010004000140040004001409883030888
:10CD600001490248FEF7CABA5824002000040140D5
:10CD700001490248FEF7C2BA5824002000040140CD
:10CD800001490248FEF7BABA30240020000C0040E6
:10CD900001490248FEF7B2BA08240020000800400A
:10CDA00002494FF08040FEF7A9BA00BFE0230020FF
:10CDB000F0B50468434DA30AAB4269D05BD9424D3C
:10CDC000AB4251D03E35AB4266D14FF0980E0326B0
:10CDD0004779B0004FEA970C00295FD063460227DD
:10CDE000A5899F4083190CEB43032F4303F1040CE7
:10CDF000364DBFB245F8231045F82C20A781EFF33C
:10CE00001181502282F31288821905EBC202136944
:10CE100073B313620433821905EBC202576917B169
:10CE20001F6053690433821905EBC202976917B179
:10CE30001F6093690433821905EBC202D76917B1E9
:10CE40001F60D36904330027CAB21F6082F31188C0
:10CE5000304405EBC000036AA3B9A38923F00103A2
:10CE60001B041B0CA381F0BD4FF0700E0226AFE730
:10CE700005EB0E03CFE7B3F5801F0ED14FF0200E68
:10CE80000026A5E7A3899BB243F00103A381F0BD6F
:10CE90004FF0480E01269BE7F0BDF0BD0223BF080E
:10CEA00003FA07F7A389094D9BB223EA0703871901
:10CEB0000CEB470CA3810CF1040345F82C1045F84A
:10CEC00023209CE70200100003001000E023002054
:10CED00010B5036883480139834282B089B200F0FB
:10CEE000CB80A0F58060834200F0C68000F58040D2
:10CEF000834200F0B88000F58060834200F0B38088
:10CF000000F58060834200F0AE80774C188824687A
:10CF10006408B4FBF2F4013CA4B282B2B3F1804FD6
:10CF20000AD07248834207D000F58060834203D064
:10CF300000F58060834202D122F0700292B26C4808
:10CF4000834200F0A28000F58060834200F0A78059
:10CF500022F4407200F56C4092B283421A80D9628A
:10CF60001C854FD05F4A93424CD001229A821A8886
:10CF700092B242F001021A80B3F1804F00F0998022
:10CF80005A4A934200F0978002F58062934200F083
:10CF9000948002F58062934200F0918002F58062F5
:10CFA000934200F08E8002F58062934200F08B8005
:10CFB00002F57042934200F0888002F5705293426D
:10CFC00000F0858002F58062934200F0828002F5D5
:10CFD000806293427FD0A2F5983293427DD002F5D1
:10CFE000806293427BD002F58062934208BF0D229B
:10CFF00015D002A84FF0012340F8043D21F0A2FF14
:10D0000002B010BD0122002119869A821A8839487F
:10D0100092B242F0010283421A80ADD10A46364BE9
:10D0200003EBC20301A893F85D408DF8044001238F
:10D0300000228DF805308DF807308DF8062021F09C
:10D0400081FF1B2C08D02E2CDAD12C4B019301A888
:10D0500021F078FF02B010BD294B019301A821F007
:10D0600071FF02B010BD204C18882468B4FBF2F4A4
:10D07000013CA4B282B251E71B4C18882468B4FB6F
:10D08000F2F4013CA4B282B256E701201A80D962C0
:10D090001C8598821A8892B202431A8070E7012098
:10D0A0001A80D9621C8598821A8892B202431A802B
:10D0B00062E70122B3E70222B1E70322AFE70422CD
:10D0C000ADE70522ABE70622A9E70722A7E708227A
:10D0D000A5E70922A3E70A22A1E70B229FE70C227A
:10D0E0009DE700BF00040140586300200004004099
:10D0F0000010004000000140BC6003082C0100014A
:10D10000190100012C4B98423DD0B0F1804F3CD02A
:10D11000A3F57C4398423AD003F58063984238D017
:10D1200003F58063984236D003F58063984234D08B
:10D1300003F58063984232D003F57043984230D0B3
:10D1400003F5705398422ED003F5806398422CD09B
:10D1500003F5806398422AD0A3F59833984228D0EB
:10D1600003F58063984207D003F58063984208BFB7
:10D170000D2202D0002070470C22104B03EBC2039B
:10D1800093F85C0070470022F7E70122F5E70222DE
:10D19000F3E70322F1E70422EFE70522EDE7062299
:10D1A000EBE70722E9E70822E7E70922E5E70A2299
:10D1B000E3E70B22E1E700BF00000140BC60030889
:10D1C0002DE9F04F013085B0C3B203930B460291B5
:10D1D0008B4C8C4E002B00F099808B4D8B4FDFF8E1
:10D1E000309217F0A9FD4FF4FA7A4FF0100C4FF47B
:10D1F0007A70D9F80430C3F30803002B40F0DE80C6
:10D20000EFF31183002B40F0D9802968A26800BF9A
:10D210002B689942F9D1D7F800E000FB0EF39B1A76
:10D22000B3FBFEF300FB01314FF0010E0191D9F881
:10D230000430C3F30803002B40F08780EFF3118321
:10D24000002B40F082802B68A16800BF2A689342BF
:10D25000F9D1D7F800B000FB0BF2521AB2FBFBF287
:10D2600000FB0323019A9B1AB3F57A7FDFD3BAF14F
:10D27000010ABED1039B002B40F0BD804FF47A7AA7
:10D28000DFF88C9150464FF0100CD9F80430C3F3FE
:10D290000803002B75D1EFF31183002B71D129689E
:10D2A000A26800BF2B689942F9D1D7F800E000FBD3
:10D2B0000EF39B1AB3FBFEF300FB01314FF0010E9E
:10D2C0000191D9F80430C3F3080313BBEFF31183C2
:10D2D000FBB92B68A16800BF2A689342F9D1D7F83F
:10D2E00000B000FB0BF2521AB2FBFBF200FB03236F
:10D2F000019A9B1AB3F57A7FE3D3BAF1010AC4D13C
:10D30000029B013B0293002B7FF467AF05B0BDE8A1
:10D31000F08FEFF311888CF31288A1682368DB0388
:10D3200044BFC6F800E0A1682B6832685FFA88F84D
:10D3300088F31188D7F800801A4400FB08F35B1AC1
:10D34000B3FBF8F300FB0233D2E7EFF311888CF361
:10D350001288A1682368DB0344BFC6F800E0A16817
:10D360002B6832685FFA88F888F31188D7F8008054
:10D370001A4400FB08F35B1AB3FBF8F300FB02331B
:10D3800070E7EFF311828CF31288D4F808E0236879
:10D39000D90303D501233360D4F808E02B68316842
:10D3A000D2B282F311883A68194400FB02F3A3EB6E
:10D3B0000E03B3FBF2F300FB01317FE7EFF31182C1
:10D3C0008CF31288D4F808E02368D90303D501232D
:10D3D0003360D4F808E02B683168D2B282F3118848
:10D3E0003A68194400FB02F3A3EB0E03B3FBF2F31C
:10D3F00000FB013118E718461DF05EFA3EE700BF5A
:10D4000010E000E0E4760020E8760020EC760020D2
:10D4100000ED00E02DE9F04F2DED028B93B0834637
:10D4200015F00CFF914B1D7825B113B0BDEC028BAC
:10D43000BDE8F08F8E4B1B685905F6D58D4B8E4E8F
:10D440001B6863B18D4A31681368CB1A7C2B06D9EF
:10D450008B48116003780133037015F0ABFB894BE7
:10D460001B78002B72D0884C884AD4F81031ABEB73
:10D470000303934201F2548394F81891B9F1000F19
:10D4800035D1DFF83C82D8F80000FBF709FDC0B2C7
:10D4900001280FD902287E4F42F066803B78002B8E
:10D4A00042F0B181D4F81C31ABEB0303B3F57A6FD2
:10D4B00082F0EF82D4F82031002B47D094F8183155
:10D4C000C3B9744B1B689B7801211E3B00228B4221
:10D4D00084F8181184F82C2142F29682D8F80000C2
:10D4E0000221043022F0F0FF94F8243111E0D4F846
:10D4F00020315BB3D4F8283140F6B732ABEB0303ED
:10D50000934223D994F82431002B01F0F986DFF8F7
:10D51000B081013BDBB284F82431002B01F026847A
:10D52000D4F8207194F82C2117F8011B94F82D31B0
:10D53000D8F80000C4F820710A44013384F82C2183
:10D5400084F82D31FBF7B0FCC4F828B1524B376892
:10D550001B7853B1DFF86C81D8F8000028B14F4B2D
:10D560001B78013B012B41F211844D4B1B7873B1A9
:10D57000DFF85481D8F800304BB13368424C029345
:10D580001A46D4F84431D31A632B01F2B281DFF882
:10D590003C8198F80030022B01F08A863C4F97F8C6
:10D5A0007430032B01F0CC833E4B1B7873B13E4D9E
:10D5B0002B685BB1344CFBF7D9FAD4F850310290A8
:10D5C00044F61F62C31A934200F23081374B1B7836
:10D5D000002B7DD1364B1B7843B12B4CD4F8A032B5
:10D5E00003F5C333A0339B4581F03E82314B1B785A
:10D5F000002B3FF41AAF244E2F4C304D06F2C127BA
:10D600002068FBF74DFC00283FF40FAF2068FBF7C4
:10D6100043FC2B7880465A1E33B120682A70FBF7F2
:10D620003FFC0028F2D100E703223946781E28F09B
:10D6300049FC96F8C03296F8C12286F8C38283F47A
:10D640007F4383F0FF039B1A1FFA88F89BB2B8EB65
:10D65000132FD5D196F8C222DBB29A42D0D1781ED0
:10D6600022F064FC2B7818442870C9E7373F00206B
:10D670006C49002084450020E8760020E845002021
:10D68000E4450020BA460020101E00203F0D030094
:10D6900028000020BC800020BC460020C44600209A
:10D6A000CC460020D4460020D84600204447002025
:10D6B00055470020DE460020E4460020E8460020D2
:10D6C000B8800020A87E0020B08000200E6B0020D3
:10D6D000484C2278A2B1484B9B7A53B1FBF746FAEB
:10D6E000464B1B68C31AA3F57A73B3F5FA6F07D8D4
:10D6F0002278434B43491868FBF7A2FB00232370B1
:10D70000414CD4F8983203F5C333A0339B45FFF462
:10D7100061AF3E4DC4F898B22B78002B41F03587AD
:10D720003B4D2B78002B41F08D8694F89C22394993
:10D730008D5CEA0701F1E787AF0701F1A78768076A
:10D7400002F12B802A0748D5334B344F0B9312AA92
:10D750001146A3F13D0241F8202D0020A3F1400223
:10D760000D4603F8400C0391022311215170937070
:10D7700028463968FCF742FD28467968FCF73EFDEB
:10D78000FB89274903EBC3039B00053381FB03217E
:10D79000DB17C3EBA101284689B2FCF747FD3B8AA2
:10D7A00003EB8303590089B22846FCF73FFD1D4B6C
:10D7B000039D1B789B0743BF398901F57A7189B2B4
:10D7C0004FF47A712846FCF731FD0A9B3A7D591CCB
:10D7D0000A9128461A7015F0C1FC134A94F89C323D
:10D7E0001178013393FBF1F201FB123384F89C3280
:10D7F000F0E600BFAC460020605B00207C6A0020A1
:10D80000484700206C460020101E00204C47002096
:10D810004D470020504700206C4600201046002055
:10D82000676666660C4600205447002094F856311F
:10D83000002B41F08A85DB4B1A6802F00803002BAD
:10D840004AF60B4048F603414BF60F4349F60747AB
:10D8500004BF03460F4612F0040F4FF0190118BF22
:10D860001F46900684F8561103D547F4804747F0C9
:10D870002007CD4B5A79C7F30909002A42F03181BC
:10D880009B79002B42F03D82984664204FF0FF3A8E
:10D890004FF0000C0A970B97ADF834C0CDF83AC0A2
:10D8A000CDF83EC0CDF842C0CDF83090ADF836800E
:10D8B000ADF838A08DF846000AAF0FCFDFF800E3CF
:10D8C00084F805C0AEE80F0097E80F00AEE8070047
:10D8D0002EF8023B71464FF0010C1B0CFE271F2057
:10D8E000C82201F81E39A770A27184F807C0E07041
:10D8F00094F86601207180F0F10383EA0313DAB231
:10D90000130983F0E70343EA022383EAC2031BB24D
:10D9100083EA0312D2B2C3F3072383EA121343EA62
:10D92000022383EAC2031BB283F0C80282EA021216
:10D93000D2B2C3F3072383EA121343EA022383EA32
:10D94000C2031BB283EA0C0787EA0717FFB2C3F3CF
:10D95000072282EA171242EA072200EB0C0382EA4E
:10D96000C7070EEB0C0084F86631278011F8013BE5
:10D970007B4083EA0313DBB21A0982EA172242EAE8
:10D98000032282EAC3031BB29FB281422780EDD1FA
:10D9900083F07C0383EA0313DBB24FEA131E8EEAA3
:10D9A000172E8EEA032E8EEAC30E0FFA8EFE1FFA92
:10D9B0008EF9DFF810C2A4F800905FFA8EFE4FEAED
:10D9C000192984F8289084F827E00CF5C77804F129
:10D9D000220ADCF80000DCF80410DCF80820DCF88F
:10D9E0000C3047460FC70CF1100CD445B846F0D1A7
:10D9F000DCF8000038606D4F9CF8043088F8043083
:10DA000007F1270884F8B5E184F8B69117F8011FEB
:10DA10002868FBF749FAB845F8D194F85731002B3C
:10DA200041F08E846249326809780A2084F85701EF
:10DA3000002901F021865F4F01293888069042F2C3
:10DA400057810229B7F802E002F06580B888059096
:10DA5000032902F05D81F8880490042902F06E81A8
:10DA60000529388902F065810629B7F80A9002F085
:10DA70005C810729B7F80C8002F05481FB8903937D
:10DA800094F866110A920B4683F0300282EA021281
:10DA9000D2B217094849079387F07A0747EA022765
:10DAA0000988237187EAC202444FC1EB012187FB39
:10DAB000013A069B4FF0000C63F30F0C059B6EF3CD
:10DAC0001F4C4FF0000E63F30F0E049BCDF82CC0DB
:10DAD00012B28A440027C91763F31F4EC1EB6A2AAA
:10DAE000039BCDF830E082EA021160F30F070020BB
:10DAF000C9B268F30F00C2F3072269F31F4782EA35
:10DB0000111263F31F404FF000090D978DF83DA0EF
:10DB10000E908DF83C9042EA01220DF1280C82EA29
:10DB2000C107BCE80F003FB287F0C80888EA0818B0
:10DB3000DFF88CE084F805905FFA88F8C7F30727D0
:10DB4000AEE80F0087EA181747EA08239CE80300AD
:10DB500083EAC8031BB283F023024EF8040B82EA67
:10DB60000212D2B2C3F30723079F83EA121370464F
:10DB700043EA022383EAC20207F1010C20F81419D8
:10DB80004FF023081621FE27C82384F866C122809F
:10DB900084F807800EF1020EA770E170A3711146A0
:10DBA00012E000BF08460020F44500209F1F00201F
:10DBB00088690020786800204C3800200308208005
:10DBC000181E0020121E002010F8013B4B4083EA73
:10DBD0000313DBB21A0982EA112242EA032282EA23
:10DBE000C3031BB299B270452180EDD183F0F403D9
:10DBF00083EA0313DBB24FEA131E8EEA112E8EEA7C
:10DC0000032E8EEAC30E0FFA8EFE1FFA8EF8CA4F4D
:10DC1000A4F800804FEA182C5FFA8EFE84F81EE00C
:10DC200084F81FC07968BA683868FB6807F5C77858
:10DC3000A8E80F0038697969BA6904F28F17A8E873
:10DC4000070004F2AD1884F8ADC184F8ACE117F810
:10DC5000011F2868FBF728F9B845F8D194F85A3124
:10DC6000002B41F07783B54B1B681922990684F885
:10DC70005A2140F1FC82B24BB24F1B789A0741F116
:10DC800028873B7D042B8CBF4FF003084FF0020820
:10DC9000FAF76CFF3B8A3A890A9003EB83035B0037
:10DCA000ADF842304FF47A703B680C93F98997F8DD
:10DCB00014E07B688DF8448000FB02F24FF0000C0A
:10DCC0000AA84FF0FF398DF845E0CDF82CC0CDF80B
:10DCD0003C900E920D93ADF8401080460390B8E84A
:10DCE0000F00DFF870E2AEE80F0098E80F00AEE832
:10DCF00007007246182122F81C39E17194F8661168
:10DD000084F805C081F0780383EA0313D8B20309CD
:10DD100083F0F60343EA002383EAC0031BB283EADD
:10DD20000310C0B2C3F3072383EA101343EA0023AE
:10DD300083EAC0031BB283F0C80080EA001C5FFACC
:10DD40008CFCC3F3072080EA1C1040EA0C2080EA18
:10DD5000CC0000B280F0180383EA0313DBB2C0F3F7
:10DD6000072080EA131040EA032080EAC30301F190
:10DD700001081E204FF0FE0C4FF0C809E0700EF1B4
:10DD8000020E217184F86681238084F802C084F831
:10DD90000690184612F8011B414081EA0111C9B2F0
:10DDA0000B0983EA102343EA012383EAC10109B284
:10DDB00088B272452080EDD181F0180181EA01110D
:10DDC000C9B20A0982EA102383EA012383EAC10364
:10DDD0001BB29AB2DFF860A12280DBB2120A059270
:10DDE000049384F8272084F82630D6460AF5C779AC
:10DDF00004F12208DEF80000DEF80410DEF8082046
:10DE0000DEF80C30CC46ACE80F000EF1100EC64523
:10DE1000E146EFD1DEF80000CCF800009DF81030AC
:10DE2000DFF8348184F8B4319DF8143084F8B531CA
:10DE3000C14619F8011F2868FBF736F8424B4B45DD
:10DE4000F7D1FAF793FE414B414AB3F90410B7F802
:10DE500008E03B680B930A907B680C9382FB0127D8
:10DE60004FF47A70C9174FF0000C00FB0EF0C1EBB5
:10DE7000A701DDF80CE0ADF83CC0ADF83EC0ADF850
:10DE800040C0ADF842100D900E90BEE80F00314F2B
:10DE900084F805C00FC79EE807004FF0210C87E803
:10DEA00007001C23C8224FF0FE0EE37084F807C061
:10DEB00084F802E0A27194F86611217181F06A037E
:10DEC00083EA0313DAB2130983F0D50343EA02238A
:10DED00083EAC2031BB283EA0312D2B2C3F307235D
:10DEE00083EA121343EA022383EAC2031BB283F0DC
:10DEF000C80282EA0212D2B2C3F3072383EA1213E2
:10DF000043EA022383EAC2031BB283EA0C0282EAD9
:10DF10000210C0B2C3F3072282EA101242EA0022C2
:10DF2000013182EAC0020C3784F866112280A7F121
:10DF30001C01104612E000BF121E002008460020FF
:10DF40000C46002010460020C51F0020EC45002094
:10DF500067666666181E00209F1F002011F8013BAF
:10DF6000434083EA0313DBB21A0982EA102242EA31
:10DF7000032282EAC3031BB298B2B9422080EDD1DA
:10DF800083F0680383EA0313DBB2190981EA1022E4
:10DF900082EA032282EAC3031BB29AB2DB4F2280D9
:10DFA000DBB24FEA122C049384F8243004F12203EC
:10DFB00084F825C007F5C7790593FB683868796848
:10DFC000BA68CE46AEE80F00059B10379F42F14677
:10DFD000F3D13B88AEF800309DF81030CC4F84F878
:10DFE000B231C14684F8B3C119F8011F2868FAF7A5
:10DFF0005BFF4F45F8D194F866C1C64AC64F84F816
:10E0000004C08CF0EB0383EA0313D9B20B0983F04D
:10E01000C50343EA012383EAC1031BB283EA031069
:10E02000C0B2C3F3072181EA101141EA002181EA5D
:10E03000C0010CCA09B281F0C80E8EEA0E1E5FFA4A
:10E040008EFE4FF000090A92C1F30721039A0B9349
:10E05000CDF8309081EA1E1343EA0E2307CA83EA03
:10E06000CE031BB283F0310E87E807008EEA0E1E46
:10E070005FFA8EFEC3F3072383EA1E1343EA0E23DF
:10E0800083EACE0394F808E0607AA17AE27A277BEB
:10E0900084F805901BB28EEA030E8EEA0E1E5FFA1C
:10E0A0008EFEC3F3072383EA1E1343EA0E2383EA9B
:10E0B000CE031BB2584080EA0010C0B2C3F307235E
:10E0C00083EA101343EA002383EAC0031BB25940DA
:10E0D00081EA0110C0B2C3F3072181EA101141EABD
:10E0E000002181EAC00109B24A4082EA0212D2B29A
:10E0F000C1F3072383EA121343EA022383EAC2032C
:10E100001BB25F4087EA0717FFB2C3F3072383EA16
:10E11000171343EA0723607BA17BE27B94F810E0AE
:10E1200094F8119083EAC7031BB2584080EA0010AC
:10E13000C0B2C3F3072383EA101343EA002383EA40
:10E14000C0031BB2594081EA0111C9B2C3F30723CE
:10E1500083EA111343EA012383EAC1031BB25A4045
:10E1600082EA0212D2B2C3F3072383EA121343EA0C
:10E17000022383EAC2031BB28EEA030E8EEA0E1E4E
:10E180005FFA8EFEC3F3072383EA1E1343EA0E23CE
:10E1900083EACE031BB289EA030989EA09195FFA07
:10E1A00089F9C3F3072383EA191343EA092383EAAE
:10E1B000C903A17CE27C594F1BB2594081EA01118D
:10E1C000C9B2C3F3072383EA111343EA012383EAA5
:10E1D000C1031BB25A4082EA0212D2B2C3F3072330
:10E1E00083EA121343EA022383EAC2031BB283F0D9
:10E1F000270989EA0912D2B2C3F3072989EA121959
:10E2000049EA022989EAC2090FFA89F91FFA89F253
:10E210000CF101034FEA122E5FFA89F931204FF019
:10E22000FE0C0C2184F86631C8232280E07184F84A
:10E2300002C0E170A37184F8149084F815E0DAF854
:10E240000410DAF80820DAF80C30DAF80000BAF82E
:10E2500010C00FC727F803CB84F8A3E184F8A2917C
:10E2600018F8011F2868FAF71FFE4745F8D194F8FF
:10E270005EC1BCF1000F41F07880294B94F866E153
:10E28000B3F90010B3F90220B3F904309FED256A09
:10E29000214F84F805C007EE103A33680A938EF0D8
:10E2A0006A0383EA031306EE901AD9B20B0983F0CE
:10E2B000D50343EA012383EAC1031BB283EA0311B6
:10E2C0005242C9B207EE902AC3F3072383EA11131F
:10E2D00043EA0123F8EEE77AF8EEE66AB8EEC77A89
:10E2E00083EAC1031BB267EE867A66EE866A27EE82
:10E2F000067A002083F0C808CDED0C7ACDED0B6ACC
:10E300008DED0D7A0E900F900EE000BF121E0020D2
:10E31000C31F00203C3F0020181E0020A01F00202B
:10E32000EC45002088C3E43A109088EA08160DF105
:10E330002809F6B2C3F30728B9E80F0088EA1618CF
:10E3400048EA062888EAC6080FFA88F80FC788F056
:10E350001E0699E8070086EA0616F6B2C8F30723F8
:10E3600083EA161343EA062387E8070083EAC60612
:10E37000C8214FF005084FF01E0CFE231C200EF1A3
:10E380000102A17184F85E8184F807C0A370E07077
:10E39000A7F1100184F804E00C37268084F8662188
:10E3A00011F8013B734083EA0313DBB21A0982EAD6
:10E3B000162242EA032282EAC3031BB29EB2B9428A
:10E3C0002680EDD183F0270383EA0313DBB24FEA03
:10E3D000131E8EEA162E8EEA032E8EEAC30E0FFA55
:10E3E0008EFE1FFA8EFCD94FA4F800C05FFA8EFE95
:10E3F0004FEA1C2C84F825C084F824E007F5C77880
:10E4000004F1220938687968BA68FB6846460FC685
:10E4100010374F45B046F5D1CD4E3B88A8F80030B7
:10E4200006F1240784F8B2E184F8B3C116F8011F9D
:10E430002868FAF739FDB742F8D194F85F81B8F14E
:10E44000000F40F08C87C34B1B6805229B0684F8A5
:10E450005F2141F10B81C04BDFEDC06ADA891B8976
:10E4600007EE902A07EE103AF8EEE77AB8EE477A10
:10E4700067EEA67A94F866C1B94BBA4AB3F90410AC
:10E48000B2F90620B84EB948CDED0B7A8CF02203D4
:10E4900083EA0313DFB23B0983F0590343EA0723FE
:10E4A00083EAC703B2F5FA6F1BB2A8BF4FF4FA6252
:10E4B00083EA0317FFB2B2F57A7FC3F3072383EA37
:10E4C0001713B8BF4FF47A724FF0640E43EA072374
:10E4D000A2F57A720EFB02F283EAC70786FB02E618
:10E4E00080FB01E03FB2C917D217C2EBA612C1EB05
:10E4F000A0034FF000090AA987F0C8068DED0C7A39
:10E50000ADF83A20ADF83830CDF82890CDF83490F9
:10E510008E4686EA0616F6B20391C7F30727BEE8D1
:10E520000F0087EA161747EA062787EAC606904FC4
:10E53000DEF800E084F804C00FC736B286F04A0364
:10E5400083EA0313DBB2C6F3072181EA13113A46CB
:10E5500041EA03210CF1010C81EAC303142042F8C3
:10E5600010E9FE264FF04A0E002184F866C14FF0F4
:10E57000C80CE0702380043784F807E0A67061714E
:10E5800084F806C0184612F8011B414081EA0111C7
:10E59000C9B20B0983EA102343EA012383EAC101CC
:10E5A00009B288B2BA422080EDD181F0140181EA2B
:10E5B0000111C9B24FEA111E8EEA102E8EEA012E09
:10E5C0008EEAC10E0FFA8EFE1FFA8EF6DFF87CA1DE
:10E5D00026804FEA162C5FFA8EFE84F81CE084F841
:10E5E0001DC0DAF80410DAF80000DAF80820DAF8CA
:10E5F0000C30BAF818900AF5C7770FC7DAF8100090
:10E60000DAF8141003C704F28F16A7F80090374603
:10E6100084F8ABC184F8AAE104F2AB1917F8011F22
:10E620002868FAF741FCB945F8D1524B524A1B7899
:10E630001278013B12F00100DBB214BFC02140216F
:10E64000172B03D84D4A134493F830804C4B1A884B
:10E6500097071ABF002341F01001012312F4027F33
:10E6600018BF022312F0100F18BF062312F0200F5C
:10E6700018BF1023002841F002824FF0030C94F8D9
:10E6800066E10A938EF0460383EA0313DAB21309B4
:10E6900083F0920343EA022383EAC2031BB283EAB4
:10E6A0000310C0B2C3F3072282EA101242EA00222A
:10E6B00082EAC00212B282F0C80787EA0717FFB2E7
:10E6C000C2F3072282EA171200238DF82FC003201D
:10E6D00042EA072C039A8DF82C808DF82D308DF8A6
:10E6E0002E108DF8300007CA8CEAC70C0FFA8CFC8C
:10E6F0001F4FE3718CEA0C1803C75FFA88F8CCF35C
:10E70000072C8CEA181C4CEA082181EAC80894F806
:10E7100008C03A700FFA88F88CEA080C8CEA0C1CD6
:10E720005FFA8CFCC8F3072282EA1C1242EA0C2230
:10E73000607AA17A94F80B80637182EACC0212B2FB
:10E74000504080EA001C5FFA8CFC1BE0121E002087
:10E750009F1F002008460020104600200AD7233CB7
:10E76000EC45002078680020D34D6210676666662D
:10E77000181E0020883800208D7D00208461030849
:10E78000A43F0020C2F3072080EA1C1040EA0C20BE
:10E7900080EACC0000B2414081EA0111C9B2C0F365
:10E7A000072282EA111242EA012282EAC10212B26F
:10E7B00088EA020888EA08185FFA88F8C2F3072294
:10E7C00082EA181242EA082294F80CC0607BA17B0E
:10E7D00084F804E082EAC80212B28CEA020C8CEAE5
:10E7E0000C1C5FFA8CFCC2F3072282EA1C1242EA7C
:10E7F0000C2282EACC0212B2504080EA0010C0B271
:10E80000C2F3072282EA101242EA002282EAC00220
:10E8100012B2514081EA0111C9B2C2F3072282EA61
:10E82000111242EA012282EAC102E17B94F81080CF
:10E8300013B281EA030282EA0212D2B2C3F30723BF
:10E8400083EA121343EA022383EAC2031BB288EA73
:10E85000030282EA0212D2B2C3F3072383EA12133D
:10E8600043EA022383EAC2031BB283F0320282EA44
:10E870000212D2B2C3F3072383EA121343EA02233C
:10E8800083EAC2031BB29AB24FF0FE0C0920C821E2
:10E890000EF1010EDBB284F802C04FEA122CE070D8
:10E8A000A17184F866E1228084F812C06374DAF8FA
:10E8B0000000DAF80410DAF80820BAF80C9007F52E
:10E8C000C07EAEE8070007F5C8778EF80280AEF884
:10E8D000009084F8A0C184F89F3116F8011F2868C1
:10E8E000FAF7E2FAB742F8D1029BC4F85031FEF7CA
:10E8F0006DBEDFF824A27C4FDFF82092412021F08A
:10E900008FFDBAF9023087FB0320DB17C3EBA000B1
:10E9100080B221F069FDBAF9003087FB0320DB17D4
:10E92000C3EBA00080B221F05FFDBAF9043087FB91
:10E930000320DB17C3EBA00080B221F055FD99F84E
:10E940000010D8F80000FAF7AFFA94F848A11AF0CE
:10E95000010700F01085654B1B689A0672D5644B61
:10E96000644F1B789B0741F14B803B7D042B8CBF90
:10E970004FF0030A4FF0020A472021F051FD38689A
:10E9800021F0FEFC786821F0FBFCFB895A4AD8F89C
:10E990000000A2FB0323C3F3471319460393FAF7BE
:10E9A00083FA3A8999F80010039B64204B4000FBDE
:10E9B00002F089F8003021F0E3FC3F7DD8F8000038
:10E9C0004AEA8707FFB23946FAF76EFA99F800303B
:10E9D000D8F800005F40394689F80070FAF764FA09
:10E9E00094F848A1BAF1000F2CD1444F4F2021F0E8
:10E9F00017FD386821F0C4FC786821F0C1FC50464E
:10EA000021F0BEFC0121D8F80000FAF74DFA384A8F
:10EA100099F800301778D8F8000007F00107394658
:10EA200083F0010389F80030FAF73EFA99F80030D4
:10EA3000D8F800005F40394689F80070FAF734FAD8
:10EA400094F848A1029B2E4AC4F844310AF101030C
:10EA5000DBB2A2FB0312D20802EB8202A3EB420359
:10EA600084F84831FEF793BD94F8A432254AC4F8DF
:10EA7000A0B202EB8302926C42B312AD04F2AB235C
:10EA8000214E45F8203D002104F2BD2331800B9337
:10EA900080211523A52784F8AA32284684F8A912D4
:10EAA00084F8A872904728463188FBF7E5FB0A9D59
:10EAB000164804F52A716D1A152DA8BF15252A468A
:10EAC00027F0F5F9124A94F8A4321570114A01336F
:10EAD00082FB0312A2EBE37202EB42029B1A84F860
:10EAE000A432FEF783BD00BF676666660846002055
:10EAF0000C460020104600201F85EB513C3F0020B3
:10EB0000CDCCCCCC8461030888450020B8370020E8
:10EB1000CD37002056555555EC450020B4800020D7
:10EB2000C24AC34BD4F8141130681B8892F80BE02A
:10EB3000C04A401A4FF47A71DFB201FB0EF11B0A92
:10EB40009777177588424FF00007D3775375977002
:10EB5000177180F0F784B849DFF808C30B6889683B
:10EB6000B648B74F007897F814A08CFB03E8DB1782
:10EB70008CFB01EC4FEAE17EC3EBA801117709128F
:10EB8000CEEBAC0E5177F4214FEA2E2C82F820E028
:10EB900091764FF0010E302182F81BE082F82210AE
:10EBA000A84B82F821C04FF0750E782182F823E03F
:10EBB00082F82410820783F81AA040F1BF84D7F8A6
:10EBC00000C0A14AD7F804E0A04882FB0C194FEA24
:10EBD000EC7182FB0E82C1EBA9514FEAEE79C9EBD1
:10EBE000A25200FB01C9029200FB02E009EB4909B5
:10EBF000974A4FEA490982FB0982049200EB4000E0
:10EC0000934A4000039082FB0008049A9014029AF1
:10EC10000490F8893F8902EB820200EBC00002EB0E
:10EC2000820207F5FA770692BAF1050F4FEA8002E1
:10EC30001FFA87FA0398049F029201EB81014FEAC1
:10EC4000E97201EB810105914FEAE071A7EB020047
:10EC5000804F83F815A0024607FB1292059F4FEAEA
:10EC6000A84840B200EB8709A8EB0100794F03994F
:10EC7000804607FB1010069F77494FFA88F84FEA45
:10EC8000DC7C4FEADE7E83F809C083F80EE0DFF813
:10EC9000D8C108EB870E029F81FB07814FEAE77816
:10ECA000BCF800700397C8EBA1116C4F029187FB71
:10ECB000021887FB00170299DFF8B0C11FFA89F923
:10ECC0001FFA8EFE4FEAE2724FEAE070C2EB68185C
:10ECD00083F80A90C0EB671283F80FE04FEA192718
:10ECE0004FEA1E29C1F3072E0399BCF80000DF721A
:10ECF00083F810904FEA222783F80C805A749DF80D
:10ED00000820DA714FEA282C4FEA1A2A4FEA112913
:10ED100034BF4FF032084FF033089DF80C2083F8D1
:10ED20000DC09F7483F816A083F808E0DA7483F8A6
:10ED3000149083F81B801877C4F810B1FEF79CBBC1
:10ED4000DFF82C91D9F80000FAF79EF800283EF47D
:10ED50002BACD9F800000121FAF792F80222002327
:10ED600087F8742088F80030FEF71EBC94F82C1148
:10ED700094F82D31D8F800004A1C013384F82C2176
:10ED800084F82D31FAF790F8FEF7DEBB344CDFF84B
:10ED9000E4904FF0000A0BE01B2B00F09F820D2B3C
:10EDA00000F079814FF0010389F80130D8F80000B4
:10EDB000FAF776F800285FD0D8F80000FAF76CF878
:10EDC00083B27E2B32682AD099F801100029EDD148
:10EDD00094F82E21002ADFD07D2B00F0648294F875
:10EDE0003CE1BEF1000F04D080F02003DBB284F8D8
:10EDF0003C11511CC9B22244092984F82E1182F811
:10EE0000303100F044820829D0D8B4F83A211344B4
:10EE100003EB132303F0FF03A4F83A31C6E784F8A9
:10EE20002EA184F82FA189F801A0BFE7E47E00207D
:10EE3000DC7E0020EC4600208C4500200C460020A3
:10EE400010460020184700206BCA5F6B806967FF7F
:10EE500083DE1B4340420F00D34D62101F85EB51F0
:10EE6000101E0020676666668C3F00208E3F0020E3
:10EE70006C6B00202800002094F83D3133B194F8E9
:10EE8000313184F83D01302B00F0D78594F82F21E3
:10EE9000BA4BBB49DFF818A3DFF8189302954FF07F
:10EEA000010E90464246002A00F05B833268D21B76
:10EEB000012A00F21F8294F83E21002A40F0348299
:10EEC00094F83FC133F81C00F0B984F83FE10A68B8
:10EED0009506E7D59AF800209007E3D5A94FAA49EF
:10EEE000FA89029D4FF4F36303FB02F381FB0321D4
:10EEF000DB17C3EB61114FF4036021F0CBFA002361
:10EF000084F82F31FEF731BB0CF1010C5FFA8CFC59
:10EF1000B0F5E06F84F83FC100F09A801BD8B0F5DF
:10EF2000047F00F0498136D8B0F5887F00F0D380A7
:10EF3000B0F5007F00F0B880B0F5807FB2D10A68EC
:10EF40005207AFD50021029D21F0A4FA002384F8D6
:10EF50002F31FEF70ABBB0F5026F00F05E816CD86E
:10EF6000B0F5E46F00F08480B0F5006F00F0DD8054
:10EF7000B0F5E26F96D1854B029DDA6B998A6423D6
:10EF800003FB02F393FBF1F121F084FA002384F8F0
:10EF90002F31FEF7EABAB0F5826F00F05581B0F577
:10EFA000C06F00F02981B0F5806F7FF47BAF94F8DB
:10EFB0004031029D0133DBB2032B00F2AF8142F2FC
:10EFC000107184F8403101FB03F1714B1B88002B59
:10EFD00040F0A28101316F4B1B78DB076E4B1B8821
:10EFE00048BF0431DF0748BF0A31980748BF1431D2
:10EFF0001A0648BF2831DF0548BF2831580748BFE7
:10F0000064311A0748BFC8319F0548BF01F5C87170
:10F01000980648BF01F57A71DA0648BF01F5FA6132
:10F020005F0648BF01F57A614FF4806021F032FA43
:10F03000002384F82F31FEF798BAB0F5046F1CD086
:10F04000B0F5116F56D0B0F5036F7FF42BAF3EE7EC
:10F050004E4B029D90469A6B998A642303FB02F300
:10F0600093FBF1F121F016FA84F82F81FEF77DBAB7
:10F07000464B029D90461A6CEEE7484B029DB3F951
:10F08000041001EB81019046490021F003FA84F855
:10F090002F81FEF76ABA4FF0010184F82E1184F82F
:10F0A0003031A4F83A2181E699F80620002A3FF48D
:10F0B000F9AE3B4B3B491B68029D81FB0321DB17EB
:10F0C000C3EBA1014FF4007021F0E4F9002384F8B0
:10F0D0002F31FEF74ABA0A6852077FF5E3AE0021E6
:10F0E0004FF48870029D21F0D5F9002384F82F3168
:10F0F000FEF73BBA99F80520002A3FF4D3AE2A4A1E
:10F10000107800283FF4CEAE284B029D1B8803EBFD
:10F110008303590091FBF0F14FF4116021F0BAF92B
:10F12000002384F82F31FEF720BA0A6895067FF590
:10F13000B9AE9AF8002090077FF5B4AE1CF0010F2D
:10F14000029D104F104900F068847A6882EAE273E9
:10F15000A3EBE27303EB5303A1FB0331C908002ABD
:10F16000ACBF41F0004141F040414FF4006021F05C
:10F1700091F9002384F82F31FEF7F7B98461030871
:10F1800008460020104600201F85EB519C450020BA
:10F19000066800208D7D0020A43F0020EC45002063
:10F1A0008C45002067666666F27E0020DC7E0020CB
:10F1B0000C460020F445002099F80520002A3FF471
:10F1C00071AEC64A107800283FF46CAEC44B029D65
:10F1D0005B7B002B00F08184C24B1B8893FBF0F01B
:10F1E00000EB800041004FF4047021F053F900233C
:10F1F00084F82F31FEF7B9B999F80620002A3FF4B8
:10F2000051AEB94B029D99684FF4C06021F042F9AC
:10F21000002384F82F31FEF7A8B90D68AD067FF5FD
:10F2200041AE9AF800C01CF0020F3FF43BAEAF4F66
:10F23000029D3B896421904601FB03F121F02AF9EC
:10F2400084F82F81FEF791B90A68900640F1018198
:10F25000A74BA64F1878397D029D00F00203002BC2
:10F260000CBF00234FF47A7340F6B83208BF4FF456
:10F27000FA6210F0010F18BF134619444FF4826070
:10F2800021F008F9002384F82F31FEF76EB9B4F8A5
:10F290003A21C2F1FF0293427FF484AD4FF00103A3
:10F2A00084F83D317EE54FF0010384F83C317DE583
:10F2B000F9F75CFC8F4B1B68C01A40F6B8339842D4
:10F2C00000F25881DFF858A29AF804303A2B00F087
:10F2D000C782002388F80030FEF766B9D8F800002E
:10F2E000F9F7DEFD00287FF45DAD4FF0010384F8EF
:10F2F0002F315BE50023029D84F82F31FEF735B9ED
:10F30000C4F8203184F81831DFF8188221F010F9A0
:10F3100094F82431FEF7FDB802315CE6012384F84D
:10F32000403142F2107150E67349029D062020F0F0
:10F3300083FE002384F83E0184F82F31FEF715B9CF
:10F34000013B84F85731FEF789BC013B84F8563104
:10F35000FEF763BB013B84F85A31FEF788BF08F122
:10F36000FF3884F85F81FFF7BFBA0CF1FF3C84F8E7
:10F370005EC1FFF762B8614B1B88D80513D4D9066C
:10F3800000F17B839A0600F1DA83580600F1DC83F2
:10F39000190700F1DB83DA0700F1EC8313F0020FA9
:10F3A0000CBF04270C27564B564A1B78D27803F023
:10F3B00001030AB143F002035320039321F030F814
:10F3C000484A128802EB820202EB8202900080B26D
:10F3D00021F00AF8002021F007F84B4A4B49128827
:10F3E000D8F80000C2EBC212520081FB0231114476
:10F3F0004FEAE27ACAEB612A5FFA8AFA5146F9F7D4
:10F4000053FD99F80020039BD8F800001F438AEAB7
:10F41000020A002189F800A0F9F746FD3946D8F81C
:10F420000000F9F741FD99F80030D8F800007B4062
:10F43000DBB2194689F80030F9F736FD94F848A197
:10F44000FFF7D0BA32493A2020F0F6FD2870FEF7D7
:10F45000C1B8304A1268120600F1F782204A127BC6
:10F46000002A3FF41FAD94F84111029D032900F2D8
:10F470008383DFE801F059281902274B1B6859796B
:10F480009A79DB7901F1407101EB022101EB034133
:10F49000002384F841314FF4826020F0FBFF002309
:10F4A00084F82F31FEF761B81C4B1A68137A507933
:10F4B00092781B0403EB002313444A1C84F8412177
:10F4C00003EB0161E7E7154B1A68D379107952789D
:10F4D0001B0403EB00231344EFE700BFF27E002080
:10F4E000E47E0020DC7E00208C45002010460020B9
:10F4F0000C460020146B00208D040308A43F00205C
:10F500008D7D0020E83800204C3800200308208042
:10F51000BD3102086C4900200848002030820020DC
:10F52000FC6A0020B8800020BA4B1A689379D07822
:10F5300012781B0403EB00231344BEE72D22DA7676
:10F54000FFF7FABBB44B31681B78C4F81411013BC8
:10F55000012B3FF600AB1021022391701371FFF7CE
:10F56000FABA029DFEF701B820F0D2FF01233B70EA
:10F57000FDF7A0BFA94AB2F84A3100210133A2F831
:10F580004A3188F80010FEF70FB8A54EA54B00933E
:10F590000024A6F13F01A44BA44A089106F8404C70
:10F5A000A34909960AA8FAF73FFF089E731C08931F
:10F5B0003470089B2922591C08911A70089BEA2272
:10F5C000591C08911A70089BC822591C08910AA856
:10F5D0001A7023F06DFC471C0AA93A46089826F0D9
:10F5E00066FC089AD31901330893D455089B5A1C1A
:10F5F00008921C70089B5A1C08921C70089B5A1C8D
:10F6000008921C70089B5A1C08921C70089B5A1C7C
:10F6100008921C70089B5A1C08921C70089B5A1C6C
:10F6200008921C70089B5A1C08921C70089B5A1C5C
:10F6300008921C70089B5A1C08921C70089B5A1C4C
:10F6400008921C70089BFF22591C08911A70089B95
:10F650000122991812A808911A7050F8283D9B1B96
:10F66000337013F07BFD2C70FDF7B4BFDFED717AC2
:10F67000B0EE677AFEF7FEBE8846894608460491DA
:10F6800005918E4606910391FEF7FAB9644A6A4BDA
:10F690000B9212AEA2F13D0046F8200D1988674F7B
:10F6A000A2F1400300204FF00A0E02F8400C08229D
:10F6B00083F801E030469A70FAF7B8FD3B6860497C
:10F6C000DA1781FB0313C2EBA30399B23046FAF7B2
:10F6D000ADFD21F051FFBF680A9B3A0C591C0A91FD
:10F6E0001A700A9B3A0A591C0A911A700A9B5A1CF2
:10F6F0000A921F700A9B5A1C0A921870304613F027
:10F700002DFDFEF71CB84F4F9FED4F8AB7F9022031
:10F7100043480B9007EE902AF8EEE77A12AE67EEB8
:10F72000887AA0F13D01FDEEE77A46F8201D00F849
:10F73000403C0823CDED027A00F83F3C1E23BDF883
:10F74000081000F83E3C3046FAF770FDB7F900307B
:10F7500007EE903AF8EEE77A304667EE887AFDEEEB
:10F76000E77ACDED027ABDF80810FAF75FFDB7F938
:10F77000043007EE903AF8EEE77A304667EE887A82
:10F78000FDEEE77ACDED027ABDF80810FAF74EFDEE
:10F79000304613F0E3FCFDF7CFBF2C4A204B126834
:10F7A0000B93A3F14007002103F8401C2123D10053
:10F7B000BB7040F1B88126490326264B1B885A05A9
:10F7C00000F1A681D80700F1BC8103F00203224AB0
:10F7D000002B1CBF03261146DFF8808032464046CE
:10F7E00026F065FB06EB080312A80133A8F102011D
:10F7F00040F8203D00225B1A06F808207B7013F0C9
:10F80000ADFCFDF79FBFC4F81CB187F80090FDF771
:10F8100051BE00BF30820020DC2D0020101E0020D1
:10F820006C46002024820020AC880308B4880308BA
:10F83000C088030800000000DC7E00208C4500200A
:10F8400067666666EC45002058A08B41CC610020BD
:10F8500098880308A43F0020A88803082F460020AA
:10F860009AF80240C4B1013CE4B201345444514618
:10F87000002211F8013B534083EA0313DBB2120A62
:10F88000DF0042EA03228C4287EA131382EA030272
:10F89000EFD1002A7FF41DADBC4ABD4FBD4B12888D
:10F8A000BD4CFA61DFF824931A68FA629B68B4F8D9
:10F8B0004A21F8660021FB64D9F80000F963FA6573
:10F8C000F8F75AFC029000287DF469AE0221D9F8BD
:10F8D0000000F9F7D5FA94F84C319AF80320039216
:10F8E000642B4FF0040287F8742040F0738194F881
:10F8F0004D31072B04BF9DF8083084F84D3194F842
:10F900004D31069307EB031ADAF80410029108460A
:10F9100023F0CEFADAF8081005915FFA80FA08466B
:10F9200023F0C6FAC0B204900AEB0002069B9B4883
:10F93000029902900832C27123F00F028646827249
:10F94000049803F00F0300EBCA008EF80D30524606
:10F950008EF80E000EF10F0026F0A9FA904B049AD3
:10F9600005990AF10900184426F0A1FA0298C37912
:10F9700003F1010ACBB1013B5FFA83FC0CF1080CE7
:10F98000DFF84CE284440023073010F8011B594093
:10F990008B00CA0883EA410302F018024B404EFA7A
:10F9A00002F253408445DBB2EFD17D4A03980AF856
:10F9B000023017F077F894F84D310022013384F8C3
:10F9C0004D3184F84C21029BDDF808A09B785BB197
:10F9D0001AF80510D9F80000F9F766FA01359AF817
:10F9E0000230EDB2AB42F3D894F84C31032201332C
:10F9F00084F84C3187F8742088F80020FFF7A2B90A
:10FA00004FF0010AFEF7B8BF0221D8F80000F9F75D
:10FA100037FA94F82431FDF77CBD3A6882EAE27344
:10FA2000A3EBE27303EB5303A1FB0331C908002AE4
:10FA3000B8BF41F08041FFF798BB5A49881F20F0BA
:10FA40009FFB84F83E01FFF721BA10230027042210
:10FA500018460AA9029D8DF828308DF829208DF8C6
:10FA60002A708DF82B708DF82C708DF82D7020F089
:10FA7000F1FC84F82F71FDF778BD342793E44A4AEE
:10FA8000D278002A0CBF4FF0040C4FF0050CFEF7A3
:10FA9000F6BD0123D8F800003B70F9F7FDF90746E1
:10FAA000D8F80000F9F7F8F97B067DF403AD8A2851
:10FAB0004ED08E287DF4FEAC94F81831002B7DF4E6
:10FAC00016AD3A4BC4F820312D2384F82431FDF7CC
:10FAD000F8BC4FF00108FEF7DBB82C4B1888FFF795
:10FAE0007FBB2A499A790B8803EB830303EB8303DB
:10FAF0004FEA83081FFA88F8002A00F01081254B8E
:10FB00001B680FFA83FA21F037FD40B2FDF7C0BE43
:10FB10000326274960E698469946184604930593BC
:10FB20000393FDF7ADBF234B234A1B68234903F41E
:10FB30008003002B16BF1146042603263DE624272A
:10FB400031E41F49042647E610272CE420272AE445
:10FB50001C4B1B689F067DF5ADAC94F81831002B4B
:10FB60007DF4C5AC184BC4F820312D2384F8243122
:10FB7000FDF7A7BC082716E44B1CDBB2042B84F866
:10FB800041314FEA01613FF483AC84E4DC7E002024
:10FB9000280000208C450020101E00209C5B0020C7
:10FBA000A25B0020481F0020E8380020EC4600201F
:10FBB0009C8803086C4900209888030890880308F3
:10FBC000A088030808460020184700206C6B00201E
:10FBD0000007090E97F875A05B4904951AF00F0FFE
:10FBE00004BF0AF1010A5FFA8AFABAF1070F28BFC7
:10FBF0004FF0010A4FEA0A1C07EB0C03187C534B29
:10FC000002930A18002392F82410504A93725FFA64
:10FC10008CF31A464E4B964607EB0C024EEA000058
:10FC200001291870D26803F101000CD90239C9B258
:10FC30008D1C1D44034603F8012BAB424FEA1222F0
:10FC4000F9D101310844BC4422F060030AF1010AF1
:10FC50009CF811205FFA8AFA1343BAF1080F037077
:10FC600000F1010340D04FEA0A1C07EB0C01384AAF
:10FC7000087C354901449A1A91F8241055180EF160
:10FC8000100E132D5FFA8EFEC6DD049D0298DFF87C
:10FC9000CCE0D2B2931DDBB243F04001C17103F15D
:10FCA000010CCBB10532D3B20833C31804930EF163
:10FCB0000100002310F8011B59408B0083EA410327
:10FCC000CA084B40234902F0180241FA02F253409D
:10FCD000049A8242DBB2EDD103980CF80E3087F81B
:10FCE00075A016F0DFFE6EE6194A049D9A1ACDE75C
:10FCF000984699461846049305939E460393FDF74C
:10FD0000BFBE154B9046B3F900A06420FDF7C0BDFF
:10FD100098469946184604930393FDF7B1BE4FF0F9
:10FD2000FF33EEE60393FDF7ABBE98460393FDF772
:10FD3000A7BE984699460393FDF7A2BE98469946FA
:10FD400018460393FDF79CBE846103089C5B00206A
:10FD5000A95B00200007090E8C450020A25B002053
:10FD60002DE9F04F2DED0A8B3C4B1B7895B0012B04
:10FD7000089001F089863A4C94F80021002A41F05D
:10FD8000C180072B374D01F07A864FF0000B6B686E
:10FD900034489847002800F06881B5F8B470002214
:10FDA00085F85520002F40F03B87B5F93E00AA6A40
:10FDB000B5F93C60696AB5F94030DFF8B4A0821A41
:10FDC000E86A6A63711A1B1A2963274895F8561066
:10FDD000AB630FF005FDDAF80030990040F1F080D8
:10FDE00095ED0D7AD5ED0C7A204A94ED676A94ED85
:10FDF000688AD4ED698AD4F8A8311268F8EEC76A27
:10FE000095ED0E7AF8EEE77AB8EEC77A013377EE21
:10FE1000867A36EE888A77EE288A9342C4ED677A2E
:10FE200084ED688AC4ED698AC4F8A83101F063835F
:10FE30000A4B1F78142F02F06B870023D4F8B061AF
:10FE40000493062E00F2AF80DFE816F01E16E316CC
:10FE5000C214F71614008E15261500BF2C7E002044
:10FE6000D4200020FC6C00202C6D002014390020D0
:10FE70006C490020D84B1A78D4F8B4E1DFF8C4C339
:10FE80009FEDD67A4FEACE000CEB000383ED007AAB
:10FE9000002A7DD0D249B0EE476AF0EE476A0023CF
:10FEA000F1EC017A013367EEA77A05EE903AB4EEF1
:10FEB000E77AF1EE10FAF8EEE55AB8BFB0EE677ADD
:10FEC0009A4276EEA76AA7EEA56AE9D1F5EEC06A76
:10FED0000CEB0003F1EE10FA83ED007A58DDC6EE6C
:10FEE000265AC04BC04A1288F7EE007A75EEE75AE0
:10FEF000D3ED007A65EEA77AFDEEE77A17EE903A39
:10FF0000812B43F3C5859342A8BF134607EE903A71
:10FF1000F8EEE77AB54B00EB0E0103EB810393EDAE
:10FF2000057AD3ED003A93ED066A93ED014AD3EDDD
:10FF3000046AD3ED034A93ED025AA3EEA77AA4EE26
:10FF4000276A66EEC76AA7EE646ABDEEC77AE5EE79
:10FF5000276A17EE101A812983ED056AC3ED066A38
:10FF600043F393858A42A8BF0A4607EE902AF8EE2B
:10FF7000E77AFCEEE77ACDED057ABDF814300CEBAC
:10FF800000029380BEF1000F02D1132F04F0F9811B
:10FF9000152F42F072846044DFF86482838828F869
:10FFA0001E30D4F8B061924B013683FB06239A19B8
:10FFB000F317C3EBA203C3EBC303F61AC4F8B06193
:10FFC0008C4B1B78002B01F09D808B4EDFF87892D4
:10FFD00006F2DC680027894BD5ED087A1B78172BD1
:10FFE00001F0808396ED007AB8EEC78A082B28EEE0
:10FFF000278A08D1B0EE480A049323F065FE804BAF
:020000040801F1
:1000000023F81700049BDAF8002092000BD5002F8C
:1000100004F01885B0EE480AD5F8783708F170007A
:100020009847B0EE408AB0EE480AD5F89836A8F165
:1000300070009847D5F80837404698476F4B1B78B3
:10004000032BB0EE408A01F05B83D6F85C06D5F84E
:10005000B830B0EE480A98470137032F08F124085A
:10006000A9EC010A06F10406B5D1644B93F800909F
:10007000B9F1070F00F08F8694F8B831002B40F0EB
:100080009786604B5B79002B40F0C48501235B4A67
:1000900084F8B8311278072A02F0748000230B9399
:1000A000594B94ED709A93ED007A584BDFF89C8190
:1000B0001B680493F7EE007A37EEC9BA544B0593E8
:1000C0002BEE07BA534B0793534B0993B4EEE7BAA1
:1000D000524B06930025F1EE10FA08F16803D4EDB7
:1000E0006FBADFF86CB1DFED4E8A9FED4EAADFEDFF
:1000F0003BAADFED4D9ADFF85C91DFF85CA14B4F36
:100100000A9388BFB0EE67BA2E46494B98ED008A35
:100110002B44D3ED007AF5EE407AF1EE10FA17D0C9
:10012000444B2B44D3ED006A38EE667AB0EEC76AD2
:10013000F4EEC67AF1EE10FA08D5B5EEC07AF1EE1B
:1001400010FACCBF37EEA68A36EEE78A83ED008A36
:10015000059B1A88930700F08680022E00F08380AA
:10016000049B93F82E10344B33F9163007EE103AF7
:100170000A9B07EE901A2B44F8EEE76AB8EEC77AAE
:10018000D3ED007A4B42A6EEA77A700007EE903AC4
:10019000F8EEE77AB4EEE77AF1EE10FA0AD407EE59
:1001A000901AF8EE677AF4EEC77AF1EE10FA88BF8B
:1001B000F0EE477A214B22490344085EB3F90C3034
:1001C000C01A07EE100AB8EEC77AD007E7EE687AD1
:1001D00040F1F68542E000BF1A390020000000001F
:1001E000D42000201C39002018390020503B00206A
:1001F000932449920E3900202C6D00202C7E002083
:10020000307E002048490020043500203082002044
:10021000A43F0020A00000208D7D00205C4900202C
:10022000CDCCCC3DAE47813F0000C84224380020F1
:10023000F834002098220020642200201862002058
:10024000EC450020383B002060490020D8210020E8
:10025000583000203038002018380020D34B93ED60
:10026000008A27EE888A069B94F8D0212B44D3ED90
:1002700001CA38EE6CCA002A38D0CD4BD4F8D4214C
:1002800008991B688A1A9A4230DD022E04F02383F3
:10029000C84B1B68990740F12987C74BC749DFF84E
:1002A0000CE331F916C09EED008ADFF878E3C7ED64
:1002B00000AA03EB460028EE288AB0F90C00A0EB58
:1002C0000C0007EE900AF8EEE77ADEF8000027EE61
:1002D000888A824238EE6CCA01F3E181F7EE007A37
:1002E000B4EEE79AF1EE10FA01F1B081B44B2B4471
:1002F00093ED000A2BEE800A022E20EE0C0AAAECE7
:10030000010A04F01683079BDBED007A93ED007A77
:10031000AC4BD7ED006A93ED006AAB4B67EE277AE2
:100320002B4427EE8B7AD3ED007A67EE277AF0EE36
:10033000665AE7EE8C5AB1EE467AF4EEC75AF1EE01
:1003400010FA08D4B4EEE56AF1EE10FA8CBFB0EE04
:10035000657AB0EE467A94ED706AF7EE007AB4EE04
:10036000E76AF1EE10FAACBF0123002343B1F0EECF
:10037000E66AF0EEC77AF4EEE67AF1EE10FA01D50D
:1003800087ED007A022E04F07E82904A904B52F85C
:1003900026001B68B0EE6C0A98478E4A8E4B52F8C6
:1003A00026001B689847049B93F8373023B1059BC0
:1003B0001B88002B00F06E85B0EE6A8A874B9BEDA0
:1003C000007A38EE400A2B4493ED008A83ED000A50
:1003D000049B30EE480A93F84830C0EE077A2BB3FE
:1003E000099B1B78DB0721D5B7EE007AB4EEC79ADC
:1003F000F1EE10FA04DB94F8D031002B00F05487B2
:10040000D4F8D431089AD31A694A12689A420DDD99
:10041000734B93ED007AB0EECCCAB4EEC7CAF1EEDE
:1004200010FA41F15980002384F8D0316D4B94F8D3
:10043000E0212B4493ED007A2BEE877A67EE277A42
:10044000C9ED007A2AB94AED01AAC7ED00AAC9EDA3
:1004500000AA0136032E08F1040809F1040907F186
:10046000040705F104057FF450AE5F4B1B78072BA2
:1004700001F02F83012B01F08A86002794F8E831E0
:10048000002B40F0FD85594A594B10681B6810F449
:10049000805A93F82C3040F05E86564A564992EDC9
:1004A000006A498B554A84ED7E6A92ED007A544A7F
:1004B00084ED7F7A07EE901AF8EEE76AD2ED037AC0
:1004C000504A84ED7C6A37EE467A77EEE67AD2EDD2
:1004D000006A84ED7B7A012284F80022C7EEA65AD6
:1004E00049494A4A91ED005A49499FED4A6A91EDBE
:1004F000004A4949DFED496AD1ED004A92ED007AA0
:1005000035EE045AF7EE007AF4EEE75A35EE245A47
:10051000F1EE10FA88BFF0EE675A25EE065AF4EEB7
:10052000E65AB1EE476AF1EE10FAB4EEC65AB8BF19
:10053000F0EE665AF1EE10FAC4ED815A01F1CB806B
:10054000B4EEC75AF1EE10FA88BFB0EE475A2E4A01
:10055000DFED306AD2ED017A2D4A92ED014A2E4A42
:1005600077EE847AD2ED014A77EEA47A67EEA67A26
:10057000B4EEE76AF1EE10FA08DCB4EEE77AF1EED9
:1005800010FA8CBFB0EE676AB0EE476A1E4ADFED24
:10059000216AD2ED027A1E4AD2ED024A204A77EE53
:1005A000A47A92ED007A67EEA67A3DE0E03400206E
:1005B0000C3500200846002018620020EC45002081
:1005C000B434002028350020C034002060300020E2
:1005D0005C300020B4300020B0300020AC2200207D
:1005E00018350020CC3400202C7E00206C490020DF
:1005F000308200206C600020605B0020E8610020F9
:10060000F47E0020E8350020183800202C3500202A
:10061000243800206F12833A303800200000000098
:100620003035002008350020B1EE473AF4EEC37AA9
:10063000F1EE10FA08D4F4EEC77AF1EE10FA8CBF9E
:10064000B0EE473AB0EE673AEF4A52780AB9B1EEE7
:10065000433A002B41F05E83F7EE003AEB4D2A78E7
:10066000002A02F09986EA4BDFEDEA7AD3ED024ADE
:10067000D3ED016A93ED037A66EE244AE5EE264A4D
:10068000E3EE074A63EEA44AF4EEE74AF1EE10FA0D
:10069000B4BFB0EE674AB0EE644A98BFF0EE647A39
:1006A000012ACDED0C4A02F09C8693ED067AD3ED3B
:1006B000052AD3ED076A26EE077AA5EE227AA3EE85
:1006C000267A23EE877AB4EEE77AF1EE10FAB4EEEA
:1006D000C47A8CBFF0EE676AF0EE476AF1EE10FA6A
:1006E00088BFF0EE676AB4BFF0EE447AF0EE477A66
:1006F000022A8DED0D7A00F0DE8093ED0A7AD3EDBB
:10070000092A93ED0B4A26EE077AA5EE227AA3EE8C
:10071000047A23EE877AB4EEE67AF1EE10FAB4EEBC
:10072000E77A8CBFB0EE664AB0EE474AF1EE10FAB7
:1007300098BFF0EE446AA8BFF0EE477A032A8DED29
:100740000E7A00F0B88093ED0E7AD3ED0D2A93ED7A
:100750000F4A26EE077AA5EE227AA3EE047A23EE5C
:10076000877AB4EEE67AF1EE10FAB4EEE77A8CBF4F
:10077000B0EE664AB0EE474AF1EE10FA98BFF0EEDE
:10078000446AA8BFF0EE477A042A8DED0F7A00F094
:10079000928093ED124AD3ED112A93ED137A26EE4F
:1007A000044AA5EE224AA3EE074A23EE844AB4EE99
:1007B000E64AF1EE10FAB4EEE74A8CBFB0EE667A84
:1007C000B0EE447AF1EE10FA98BFF0EE476AA8BF97
:1007D000F0EE447A052A8DED104A6CD093ED164A5E
:1007E000D3ED152A93ED177A26EE044AA5EE224A98
:1007F000A3EE074A23EE844AB4EEE64AF1EE10FA7D
:10080000B4EEE74A8CBFB0EE667AB0EE447AF1EE11
:1008100010FA98BFF0EE476AA8BFF0EE447A062AB5
:100820008DED114A47D093ED1A4AD3ED192A93ED75
:100830001B7A26EE044AA5EE224AA3EE074A23EECF
:10084000844AB4EEE64AF1EE10FAB4EEE74A8CBF01
:10085000B0EE667AB0EE447AF1EE10FA98BFF0EEA0
:10086000476AA8BFF0EE447A072A8DED124A22D0DB
:1008700093ED1E7AD3ED1D2A93ED1F4A26EE077ADB
:10088000A5EE227AA4EE037A27EE237AB4EEE67A76
:10089000F1EE10FAB4EEE77A8CBFB0EE666AB0EE15
:1008A000476AF1EE10FA8DED137A98BFF0EE466AC2
:1008B000A8BFF0EE477A77EEE67AF7EE006AF4EE3C
:1008C000E67AF1EE10FAC4ED707A43F3478586EECE
:1008D000A77A022ADDED0D7A67EE244A67EE877A61
:1008E000CDED0C4ACDED0D7A2DD0DDED0E7A67EE13
:1008F000877A032ACDED0E7A25D0DDED0F7A67EEEB
:10090000877A042ACDED0F7A1DD0DDED107A67EEDF
:10091000877A052ACDED107A15D0DDED117A67EED4
:10092000877A062ACDED117A0DD0DDED127A67EEC9
:10093000877A072ACDED127A05D0DDED137A27EEFE
:10094000877A8DED137A344B1E6816F0805601F0CD
:10095000B480F6EE005AC4ED815A002A02F01185E7
:100960002E4BD4ED7F4A93F8038094F90032099915
:10097000D4ED7E6A91F800E0DFF8ACC02849DFF8DA
:10098000AC90B1F906109CED007A049106EE103A95
:10099000FDEEE44A234B99F80090B3F81AB094EDB9
:1009A0007B5AD4ED7C7A14EE903AFDEEE64A00F0E4
:1009B000100C00F480000EF0010EB8EEC66A14EEC2
:1009C000901A0590B8F1000F41F0FA81DFF84080ED
:1009D000BCF1000F41F0928098ED007ADDED0C6AD9
:1009E000DFF84CC025EE877AA6EE267AF0EE676A2D
:1009F000E5EE076ABDEEE67A17EE106A17EE100A0A
:100A00009E42A8BF184615E088380020A85E002046
:100A10005835002000000000CC610020E83800209C
:100A200078680020605B002034350020406400209E
:100A300060380020B142C8BF084607EE100AB8EE81
:100A4000C77A012A8CED007A00F0DC8098ED047AF8
:100A5000DDED0D6A25EE877AA6EE267AF0EE676A5E
:100A6000E5EE076ABDEEE67A17EE106A17EE100A99
:100A70009E42A8BF1846B142C8BF084607EE100AFA
:100A8000B8EEC77A022A8CED017A00F0BB8098EDAF
:100A9000087ADDED0E6A25EE877AA6EE267AF0EE6C
:100AA000676AE5EE076ABDEEE67A17EE106A17EEA2
:100AB000100A9E42A8BF1846B142C8BF084607EEBA
:100AC000100AB8EEC77A032A8CED027A00F09A80F9
:100AD00098ED0C7ADDED0F6A25EE877AA6EE867A20
:100AE000F0EE676AE7EE056ABDEEE67A17EE106A89
:100AF00017EE100A9E42A8BF1846B142C8BF08466A
:100B000007EE100AB8EEC77A042A8CED037A79D082
:100B100098ED107ADDED106A25EE877AA6EE867ADA
:100B2000F0EE676AE7EE056ABDEEE67A17EE106A48
:100B300017EE100A9E42A8BF1846B142C8BF084629
:100B400007EE100AB8EEC77A052A8CED047A59D060
:100B500098ED147ADDED116A25EE877AA6EE867A95
:100B6000F0EE676AE7EE056ABDEEE67A17EE106A08
:100B700017EE100A9E42A8BF1846B142C8BF0846E9
:100B800007EE100AB8EEC77A062A8CED057A39D03E
:100B900098ED187ADDED126A25EE877AA6EE867A50
:100BA000F0EE676AE7EE056ABDEEE67A17EE106AC8
:100BB00017EE100A9E42A8BF1846B142C8BF0846A9
:100BC00007EE100AB8EEC77A072A8CED067A19D01C
:100BD00098ED1C7ADDED136A65EE875AE6EE265A2B
:100BE000E5EE257AFDEEE77A17EE900A8342A8BF7C
:100BF00003468142C8BF0B4607EE903AF8EEE77A0B
:100C0000CCED077ABEF1000F40F04782002A40F099
:100C10003F8242E2AD4B1B78013BDBB2FFF737BAB4
:100C2000AB4B06934FF47A761B68B6FBF3F3C3EB3A
:100C30004316A849DFF8C88291F801A0A649B8F97F
:100C4000060091F8009003EB8603DE00B6B2B742CF
:100C500002F02681D5F88810B5F93CE0EB6E4A1C0D
:100C600007EE90EA7344012AC5F88820EB66F8EE97
:100C7000E77A02F02081D5ED1E5AD5ED206A07EE05
:100C8000102A37EEE56AB8EEC75A012F86EE057ACC
:100C900037EE257A77EEC77A85ED1F7AE7EE866A1A
:100CA00085ED1E7AF0EE667AC5ED216AC5ED206A03
:100CB00002F0D084D5F89C10B5F93EE02B6F4A1CA9
:100CC00007EE90EA7344012AC5F89C202B67F8EEE2
:100CD000E77A02F00981D5ED235AD5ED256A07EEB2
:100CE000102A37EEE56AB8EEC75A012F86EE057A6C
:100CF00037EE257A77EEC77A85ED247AE7EE866AB5
:100D000085ED237AF0EE667AC5ED266AC5ED256A93
:100D100002F0D484D5F8B010B5F940E06B6F4A1CEE
:100D200007EE90EA7344012AC5F8B0206B67F8EE2D
:100D3000E77A02F0F280D5ED285AD5ED2A6A07EE5F
:100D4000102A37EEE56AB8EEC75A012F86EE057A0B
:100D500037EE257A77EEC77A85ED297AE6EE276AAF
:100D600085ED287AF0EE667AC5ED2B6AC5ED2A6A24
:100D700002F09884A8F80600574B013F93F80090C2
:100D8000A5F8B47006990023B9F1070F4B608B608A
:100D9000CB607FF471A9F7F7E9FEDFF8648194F87E
:100DA000B831A0EB0B00A8F80000002B3FF469A9B4
:100DB000013B84F8B83115B0BDEC0A8BBDE8F08F6B
:100DC000B1F9002094ED5E7AB1F90200D4ED5F6ACA
:100DD000424982EAE273A3EBE273F4EEC76A80EA67
:100DE000E072F1EE10FAA2EBE072B4BFB0EE476A27
:100DF000B0EE666A9342B8BF134607EE103A0B781E
:100E0000B8EEC77A27EE287A002B40F0E781344B02
:100E1000D3ED005AF4EECA5AF1EE10FA41F1EC802B
:100E2000B7EE005A75EE654ADFED2E6A9FED2E5A39
:100E30002E4B36EEC77A24EE855AD3ED006AE5EEE6
:100E4000075A65EEA65AF5EEC05AF1EE10FA40F2D6
:100E50003086C9EEA56AB7EE007AF0EE475AE6EEA4
:100E6000665AF0EE656AF4EEC76AF1EE10FA88BFD2
:100E7000F0EE476AF5EEC06AF1EE10FAB8BFF0EE98
:100E80006A6A1B4B93ED007A67EE877AA7EEA68A13
:100E9000FFF7E9B9174B184A2B4493ED007AD2EDCE
:100EA000007A164B67EE277AF7EE006AF4EEE67AE0
:100EB000F1EE10FA93ED007A88BFF0EE667A67EEF5
:100EC000877A27EE888AFFF779BA00BF0C62002084
:100ED0005C490020484900202C7E0020EC34002092
:100EE000F434002000003443610BB63BE8340020AA
:100EF000E43400204C220020DC340020D8340020D0
:100F0000307E0020072B02F067824FF00009DFF8E7
:100F10008CA3CA4DDAF800305A0501F12981C84B7B
:100F200019680B0701F16D80C64B1B78002B40F050
:100F3000E681DFF848B394F8126126B1C24B1B88F2
:100F40009F0742F03E8094F81831002B41F0B480A6
:100F50009BF81E60002E00F0DA83022E02F02A8039
:100F6000032E01F00583B94A52889BF81F7002379F
:100F7000FFB2002B02F01280002A02F00F80B44969
:100F80000E68B2FBF6F216B2A4F84861002F03F027
:100F9000ED8107EE906AF8EEE77AF7EE006A86EEEA
:100FA000A77AAC4A012FD4ED576AD2ED007A77EEDA
:100FB000E67A67EE877AC4ED537A21D0D2ED017AD2
:100FC000D4ED586A77EEE67A022F67EE877AC4EDA1
:100FD000547A15D0D2ED027AD4ED596A77EEE67ADA
:100FE000032F67EE877AC4ED557A09D0D2ED037AE4
:100FF000D4ED5A6A77EEE67A67EE877AC4ED567AD0
:1010000095490978092903F04482002E40F385832D
:1010100097B394ED577AD4ED537A77EE877A012F10
:10102000C4ED577AC2ED007A21D094ED587AD4ED10
:10103000547A77EE877A022FC4ED587AC2ED017A9E
:1010400015D094ED597AD4ED557A77EE877A032F3F
:10105000C4ED597AC2ED027A09D0D4ED5A7A94EDF2
:10106000567A77EE877AC4ED5A7AC2ED037A013F59
:10107000022FB8BF0227FFB2002B18BF02274DE393
:10108000099B764D1B78DE0700F157812A7822B143
:1010900092007349734824F00AFF734B1B68002BBE
:1010A00040F01D83714B1B789BB1287870B1DFF83D
:1010B000B481DFF8EC910026F0B2D9F80030B8EC3A
:1010C000010A9847287801368642F5DB684B1B6891
:1010D0009847614B1B78072B00F0F484012384F8B8
:1010E000003115B0BDEC0A8BBDE8F08F614BC7ED48
:1010F00000AA1B689A427FF7F1A8002384F8D03138
:10110000FFF7F4B85C4FDFF89C9107F24C7607F5D7
:10111000F768F7EC017A95ED080AD5F87837F8EE1C
:10112000E77A304627EE800A9847A6F1E000D5F826
:1011300098369847A6F17000D5F808379847D7F841
:101140005806D5F8B83098472436B045A9EC010ABE
:10115000DFD1FEF78ABF099A1278D50703D4474A30
:10116000128BA4F8F421464A3A49128891ED037A89
:1011700007EE902AF8EEE77AB4EEE77AF1EE10FA8D
:1011800041F210813F49098807EE901AF8EEE77A9C
:10119000B4EEE77AF1EE10FAC1F252803A493B4AD6
:1011A000D1ED006A92ED006A3949C4ED7E6ABCEE69
:1011B000C75A76EE665A15EE102AC4ED7C6AC4ED65
:1011C0007B5A84ED7F6AA4F8F4210122D1ED006AF4
:1011D00084F8002277EE677AFFF780B92D4B93ED04
:1011E000005AB5EEC05AF1EE10FA40F362842A4B71
:1011F000D3ED006AF5EEC06AF1EE10FA40F35984BF
:1012000036EEC77A66EE695A87EE266AC5EE856ABB
:10121000B7EE007AB4EEC76AF1EE10FA88BFB0EE0E
:10122000476AB5EEC06AF1EE10FA76EE876AB8BF8B
:10123000B0EE6A6A66EE266A15E600BFFC6C002016
:1012400008460020E8000020A43F00208869002014
:1012500084380020F47E00202C7E0020A85E002030
:1012600038350020603800205430002048670020C6
:101270003C640020083500202C6D0020605B0020BD
:10128000EC350020EE350020D8350020E861002044
:10129000F4350020E8340020F03400206C490020B0
:1012A0003464002060490020DA4A92ED007AF0EEC2
:1012B000E76AF4EEC76AF1EE10FA7FF7A1A8D64A02
:1012C00092ED007AF0EECC6AF4EEC76AF1EE10FA15
:1012D0007FF796A8D14A98ED007AD2ED006AB0EE79
:1012E000C77AB4EEE67AF1EE10FA7FF589A801220A
:1012F0000899C4F8D41184F8D021FFF785B8C84BF9
:10130000DFF838B3B3F90620BBF81A309A423FF73A
:1013100012AEC44B1B78012B01F02B86192B01F068
:1013200028860E2B3FF407AE082B3FF404AEBE4ACE
:1013300000239360C4F80C31FDE52B78002B3FF4BB
:10134000ACAED4ED5F3A94ED5E6AD4ED7C7AB74AE8
:1013500094ED7B7AD2ED005A94ED5C4AD4ED5B4A71
:10136000DFF8DC82DFF8DCC2F4EEC63AF3EE046AA2
:10137000F1EE10FA37EEA65A01F14B8098ED026AB1
:1013800026EE446AF0EE674AE6EE074AF4EEC54AF6
:1013900034EEE66AF1EE10FA48BFB0EE656A012B52
:1013A0008CED006A3FF479AE98ED066A26EE446A49
:1013B000F0EE674AE6EE074AB4EEE45A34EEE66A27
:1013C000F1EE10FA88BFB0EE656A022B8CED016A6F
:1013D0003FF463AE98ED0A6A26EE446AF0EE674A7F
:1013E000E6EE074AF4EEC54A34EEE66AF1EE10FA8C
:1013F00048BFB0EE656A032B8CED026A3FF44DAE38
:1014000098ED0E6A26EE446AF0EE674AE6EE074A69
:10141000F4EEC54A34EEE66AF1EE10FA48BFB0EEDB
:10142000656A042B8CED036A3FF437AE98ED126ABF
:1014300026EE446AF0EE674AE6EE074AB4EEE45A56
:1014400034EEE66AF1EE10FAC8BFB0EE656A052B1D
:101450008CED046A3FF421AE98ED166A26EE446ADC
:10146000F0EE674AE6EE074AF4EEC54A74EEE66A25
:10147000F1EE10FAB8BFF0EE656A062BCCED056A06
:101480003FF40BAED8ED1A6A66EEC46AF0EE674A16
:10149000E6EE874AB3EE046AB4EEE45A74EEC66A26
:1014A000F1EE10FAC8BFF0EE656A072BCCED066AC4
:1014B0003FF4F3ADD8ED1E6A26EEC44AE4EE077A97
:1014C000F4EEC57A77EEC67AF1EE10FA48BFF0EE88
:1014D000657ACCED077AE0E5504B98ED007AD3EDD4
:1014E000006AB0EEC77AB4EEE67AF1EE10FA7EF753
:1014F0009DAFFEF798BF07EE103A4D4BDFF84881DD
:101500001B78C4F8A871B8EEC77AF7EE006A132BFF
:1015100086EE879AB8F90400B4F8AC6195ED080A34
:1015200001F02C84434B444AD3ED000A93ED053A75
:1015300093ED091A93ED0E4AD3ED121AD3ED172A43
:10154000D3ED015AD3ED063A93ED0A7A93ED0F5A93
:1015500093ED132A93ED186AD3ED044A93ED030A31
:1015600067EE897A69EE086A69EE288AA0EEA73AE2
:1015700002EB86070021A1EE264AC4F89C11C4F8AC
:10158000A011E1EEA82AE5EEA73AA7EE265AD3ED80
:101590000D5A93ED167AD3ED020AD3ED0B1A93EDA3
:1015A0000C1A87ED003AA2EE286A64EEC34A65EE93
:1015B000C45A27EE627A93ED152A87ED204AE0EEB1
:1015C000433A93ED143AC3ED053AE0EEA74AE1EE53
:1015D000A65AF0EE477AF0EE466AA1EE445AE2EEE1
:1015E000626AE3EE287AC3ED064A83ED0E5AC3ED34
:1015F0000F5AC7ED402AC3ED176AC3ED187AC4F835
:10160000A411731C03F01F03A4F8AC31A8F8040064
:10161000FEF70EBC1C3500201835002020350020B8
:101620007868002088380020F47E002034350020BF
:101630002C7E0020BC3B002038390020605B00205D
:101640005835002060380020307E00200699D64BA7
:10165000D1ED017A93ED007AF0EEE77AF4EEC77AF5
:10166000F1EE10FA7EF542AED1ED027AF0EEE77AB5
:10167000B4EEE77AF1EE10FA7EF738AED1ED037AE8
:10168000F0EEE77AB4EEE77AF1EE10FA7EF72EAEDE
:10169000C64B1B689A077FF530ADC549C54BB3F9FA
:1016A0000C20B1F900E0C448AEEB020E00688EEAEF
:1016B000EE72A2EBEE728242BEF618AEB3F90E30B5
:1016C000B1F90220D21A82EAE273A3EBE2739842E4
:1016D0007EF70CAE11E5B0EE465AFEF738BF09F0C2
:1016E00075FDDFE496ED007AB44905EB4702B8EEEC
:1016F000C78A928F21F8172028EE278AFEF783BC2D
:1017000022F0E2FAAD4B23F81700FEF79EBCA4F8D6
:101710004861002B00F09481A94A0227A94BDFED14
:10172000AA6A1968A94B887893F800E00B7807EE4D
:10173000903AF8EEE77AB0EE007A67EEA67AF4EE29
:10174000C77AF1EE10FA40F3168337EEC77ADFED71
:10175000A06AB0EE676AA7EE266AB0EE467A9FED01
:101760009D6AD2ED006A66EE866AB0EEE66AC4ED66
:101770005B6A84ED5E6A98B105EE900AB8EEE55AB0
:10178000DFED915A66EEA64A25EE255AF7EE005A8D
:1017900075EEC55A64EE864AE4EE855A66EEA56A91
:1017A000DFED8D5A4B7927EE257A27EE267ACBB1DD
:1017B000DFED856ADFED895A26EE266A06EE903A5D
:1017C000F8EEE66A26EE266AB4EEE56AF1EE10FA65
:1017D00000F31B86F7EE005A35EEC66AC5EE866A40
:1017E00027EE267ABEF10C0F9FED7E8ADFED7E6A32
:1017F00000F07285B4EEC87AF1EE10FA98BFB0EE40
:10180000478AB4EEE68AF1EE10FAB8BFB0EE668A07
:1018100084ED418A002F00F00581B0EE007AF4EEED
:10182000C77AF1EE10FA05DD37EEC77ADFED686AA8
:10183000E7EE267A92ED017ADFED666A27EE267AE8
:10184000B0EEC76A84ED5C7A84ED5F6A98B106EE0B
:10185000900ADFED5D5AF8EEE66A27EE075A66EE6B
:10186000A56AF7EE005A75EEE65A25EE065AE5EE41
:10187000265A27EE257ADFED586A8B7967EEA67A2D
:1018800067EE877AABB107EE103AB8EEC77ADFEDB4
:101890004E5ADFED526A27EE067A27EE257AB4EE2D
:1018A000E67AF1EE10FA40F3A285DFED4D6A67EEBD
:1018B000A67ABEF10C0F00F0EE84DFED4A6A9FEDD0
:1018C0004A7AF4EEE67AF1EE10FA88BFF0EE667A24
:1018D000F4EEC77AF1EE10FAB8BFF0EE477A012FB6
:1018E000C4ED427A40F39E804B78DFED376A07EE15
:1018F000903AF8EEE77AB0EE007A67EEA67A4B7A85
:10190000F4EEC77AF1EE10FA05DD37EEC77ADFEDB7
:10191000306AE7EE267A92ED027ADFED2E6A27EE44
:10192000267AB0EEC76A84ED5D7A84ED606A9BB179
:1019300006EE903ADFED245AF8EEE66A27EE075AF3
:1019400066EEA56AF7EE005A75EEE65A25EE065ADF
:10195000E6EE855A27EE257ADFED1F6ACB7967EE32
:10196000A67A67EE877A002B44D007EE103AB8EEDD
:10197000C77ADFED155ADFED196A27EE067A27EEF2
:10198000257AB4EEE67AF1EE10FA2FDCB5EEC07AE5
:10199000F1EE10FA01F1F882B7EE006A36EE477AFE
:1019A000C6EE076A24E000BF143500200846002078
:1019B000EC4500201862002010350020307E002009
:1019C000F47E0020084800200AD7233C2C7E00200B
:1019D000D7A368416F12033B00004843A4707D3FCA
:1019E0000000C84200C0F94400C0F9C45FED046AB9
:1019F00067EEA67ABEF10C0F00F08B845FED076AEC
:101A00001FED077AF4EEE67AF1EE10FA88BFF0EEF9
:101A1000667AF4EEC77AF1EE10FAB8BFF0EE477AC4
:101A2000C4ED437ABEF1090F00F029849BF82160D0
:101A3000002E40F0BF83D14B1968002384F8183181
:101A4000890609D5CE4B1B8803F0300323B1CD4B5B
:101A50001B78DA0701F1A487CB4B1B7823B9CB4E57
:101A6000B378002B41F0EE82C94B1B78072B00F0B6
:101A70005A840022072B84F800217EF486A9F7F708
:101A800075F88346FEF783B9C24BC34C1A68C34B43
:101A9000DFF8148394F80001D2691B88A8F80020AD
:101AA000A8F8023000287FF430AA8346BC4DFEF728
:101AB0006EB9DFEDBC6AFFF7E4B941023EF549AF0C
:101AC000FEF74BBFF7F752F8B74BC01BD880FFF7B4
:101AD00005BBF7F74BF8AE4B0B9A1B78DFF8C882C3
:101AE000801A012BA8F8020000F05383072B7EF424
:101AF000C4ACF7F73BF80746FEF7C0BCBEF1000FD9
:101B000041F0818498ED007ADDED0C6ADFF8ACC21B
:101B100025EE877AA6EE867AF0EE676AE7EE056A2A
:101B2000BDEEE67A17EE106A17EE100A9E42A8BFC5
:101B30001846B142C8BF084607EE100AB8EEC77A89
:101B4000012A8CED007A3FF4A3AA98ED047ADDED2A
:101B50000D6A25EE877AA6EE867AF0EE676AE7EEE2
:101B6000056ABDEEE67A17EE106A17EE100A9E427D
:101B7000A8BF1846B142C8BF084607EE100AB8EE23
:101B8000C77A022A8CED017A3FF482AA98ED087A8E
:101B9000DDED0E6A25EE877AA6EE867AF0EE676AAC
:101BA000E7EE056ABDEEE67A17EE106A17EE100A48
:101BB0009E42A8BF1846B142C8BF084607EE100AA9
:101BC000B8EEC77A032A8CED027A3FF461AA98ED49
:101BD0000C7ADDED0F6A25EE877AA6EE867AF0EEB6
:101BE000676AE7EE056ABDEEE67A17EE106A17EE51
:101BF000100A9E42A8BF1846B142C8BF084607EE69
:101C0000100AB8EEC77A042A8CED037A3FF440AA92
:101C100098ED107ADDED106A25EE877AA6EE867AC9
:101C2000F0EE676AE7EE056ABDEEE67A17EE106A37
:101C300017EE100A9E42A8BF1846B142C8BF084618
:101C400007EE100AB8EEC77A052A8CED047A3FF445
:101C50001FAA98ED147ADDED116A25EE877AA6EEBB
:101C6000867AF0EE676AE7EE056ABDEEE67A17EE71
:101C7000106A17EE100A9E42A8BF1846B142C8BFAC
:101C8000084607EE100AB8EEC77A062A8CED057AE8
:101C90003FF4FEA998ED187ADDED126A25EE877AF9
:101CA000A6EE867AF0EE676AE7EE056ABDEEE67AA2
:101CB00017EE106A17EE100A9E42A8BF1846B142EE
:101CC000C8BF084607EE100AB8EEC77A072A8CED9F
:101CD000067A3FF4DDA998ED1C7ADDED136A65EE16
:101CE000875AE6EE265AE5EE257AFDEEE77A17EEFC
:101CF000900A8342A8BF03468142C8BF0B4607EE45
:101D0000903AF8EEE77ACCED077A002A7FF4C0A982
:101D1000FFF7C3B9254B5A79002A3EF49DAC244AFB
:101D20001278002A3EF498AC1B78DFED224A07EEC9
:101D3000903A214BB8EE677A1B8807EE902A06EEA0
:101D4000903AF8EEE77AF8EE666A67EE277AB7EE31
:101D5000007AC7EEA63AF4EEE43AF1EE10FA88BF44
:101D6000F0EE643AF4EEC73AF1EE10FAB8BFF0EED6
:101D7000473AFEF773BCB0EE677AF0E408460020FD
:101D8000A43F00200C460020373F00207E83002027
:101D90002C7E002090470020D4200020E02D002041
:101DA000FC6C002000000000307E0020F445002084
:101DB000F27E0020713DAA3FDC7E002060380020CA
:101DC000BCF1000F00F0E883BEF1000F42F01B8071
:101DD000DFF8C485B9F1000F41F06A86D8ED006ADA
:101DE000DDED0C4ADFF8B4C565EEA66ABDEEC77A34
:101DF00017EE101AB0EE667AA4EE867AF0EE676AF5
:101E0000E7EE056ABDEEE67A17EE106A17EE100AE5
:101E10009E42A8BF1846B142C8BF084607EE100A46
:101E2000B8EEC77A012A8CED007A3FF431A998ED1B
:101E3000047ADDED0D6A25EE877AA6EE867AF0EE5D
:101E4000676AE7EE056ABDEEE67A17EE106A17EEEE
:101E5000100A9E42A8BF18468E42B8BF084607EE39
:101E6000100AB8EEC77A022A8CED017A3FF410A965
:101E700098ED087ADDED0E6A25EE877AA6EE867A71
:101E8000F0EE676AE7EE056ABDEEE67A17EE106AD5
:101E900017EE100A9E42A8BF18468E42B8BF0846E9
:101EA00007EE100AB8EEC77A032A8CED027A3FF4E7
:101EB000EFA898ED0C7ADDED0F6A25EE877AA6EE95
:101EC000867AF0EE676AE7EE056ABDEEE67A17EE0F
:101ED000106A17EE100A9E42A8BF18468E42B8BF7D
:101EE000084607EE100AB8EEC77A042A8CED037A8A
:101EF0003FF4CEA898ED107ADDED106A25EE877AD2
:101F0000A6EE867AF0EE676AE7EE056ABDEEE67A3F
:101F100017EE106A17EE100A9E42A8BF18468E42AE
:101F2000B8BF084607EE100AB8EEC77A052A8CED4E
:101F3000047A3FF4ADA898ED147ADDED116A25EE30
:101F4000877AA6EE867AF0EE676AE7EE056ABDEE5E
:101F5000E67A17EE106A17EE100A9E42A8BF1846DE
:101F60008E42B8BF084607EE100AB8EEC77A062AB6
:101F70008CED057A3FF48CA898ED187ADDED126AA5
:101F800025EE877AA6EE867AF0EE676AE7EE056AB6
:101F9000BDEEE67A17EE106A17EE100A9E42A8BF51
:101FA00018468E42B8BF084607EE100AB8EEC77A48
:101FB000072A8CED067A3FF46BA898ED1C7ADDEDCC
:101FC000136A65EE875AE6EE265AE5EE257AFDEEAF
:101FD000E77A17EE900A8342A8BF03468142D8BF32
:101FE000194607EE901AF8EEE77ACCED077A002A48
:101FF0007FF44EA8FFF751B8D14BD3ED005AFEF74E
:1020000022BFD04AD2ED027AB2EE0E7AF0EEE76A43
:10201000F4EEC76AF1EE10FA41D5CB4B1B885F078F
:102020003DD5CA4BCA48B3F90430CA4E80FB037091
:102030003688DB17C3EBA0039B1B9BB218B210F1D1
:10204000B30FBCBF03F5B47318B2B328C4BFA0F577
:10205000B47318B2C04BC14E1B793678002B4FF6C3
:10206000FF7318BF012336077EF55EAFBC4E36689E
:1020700010FB03F3307EBB4E9BB210FB03F386FBD9
:1020800003601844DB17C3EB201307EE103AB8EED9
:10209000C77A77EEC77AC2ED027AFEF745BFAB4B3F
:1020A000AB4AB3F90430AB4882FB0362DB17C3EBE6
:1020B000A2030380FEF738BFAB48AC4AD0F8EC006F
:1020C000126844F62066B042A8BF3046B0F57A7F69
:1020D000B8BF4FF47A7080B212F0100FA4F81A0152
:1020E000DAF8002001F09882D20400F16A839C4A59
:1020F0001768B7F932C0934A9D4ED2ED037AD4F8EF
:102100001C21A6FB0006B609642090FBF6F01428FB
:10211000BDEEE77A04EB420EA8BF142001329042D4
:10212000C4F81C2117EE108ADCBF0022C4F81C2161
:1021300004EB4202AEF82081B2F9202107EE102A0A
:10214000B8EEC77A77EEC77AFDEEE77ACDED047A7E
:10215000BDF9100080EAE072A2EBE072624502F382
:10216000EF80844A10464FF07E520260FEF7F0BEC8
:10217000AB68002B3EF4D3AE05F1500128469847DA
:10218000FEF7CDBEF6F7F2FC0B90FDF789BFDFF846
:102190001082F6F7EBFC784AD4F8E4311268C4F800
:1021A000E401C31A9A1A0746A8F80430A8F80620D2
:1021B000FEF764B91E216D48F8F7A4FB00283FF430
:1021C0003AAC614B1B8858063FF535AC94F8843126
:1021D000B34242F0EF80674BD4ED627AD3ED016AEF
:1021E00094ED435ADFED655A9FED656A27EEC57A97
:1021F00068EE277AA8EE267AE5EE267AB4EEE57A3E
:10220000F1EE10FA88BFB0EE657AB4EEC67AF1EE60
:1022100010FAF4EEE57AB8BFB0EE467AF1EE10FAB5
:1022200088BFF0EE657AF4EEC67AF1EE10FAB8BF28
:10223000F0EE467A84ED417AC4ED437AFFF7FBBBBA
:10224000B4F8F411914240F27A854E494E4AD1EDEC
:10225000007A92ED007A4D49C4ED7E7A77EE676A96
:10226000C4ED7C7A0122C4ED7B6A84ED7F7AD1EDE6
:10227000006ADFED477A84F80022FEF72FB9FDEE01
:10228000C87ADFF81C8117EE903AA8F80460A8F825
:102290000630FFF7CBBB9FED397ADFED396ADFF807
:1022A0000081F4EEC77AF1EE10FA98BFB0EE677ACB
:1022B000FDEEE77AB4EEE67AF1EE10FA17EE903A18
:1022C000B8BFB0EE667A012F84ED427AA8F80230EA
:1022D0003FF70AABFFF7AABBB4EEC87AF1EE10FAEB
:1022E00098BFB0EE478ABDEEC77AB4EEE68ADFF853
:1022F000B080F1EE10FA17EE103AB8BFB0EE668A71
:1023000084ED418AA8F80030002F7FF486AAFFF7F9
:102310008DBBBDEEE77ADFF8888017EE103AA8F89B
:102320000430FFF76BBBF6F721FCDFF87480194B24
:10233000A0EB09001B78A8F80400FFF79ABB00BFC8
:10234000E8340020F47E0020A43F0020EC4500206B
:10235000676666665C400020106200200C46002024
:1023600030820020898888885C010020CC610020B0
:10237000D34D6210A00000208438002000C0F94432
:1023800000C0F9C4D8350020E8610020F4350020F1
:10239000000000002C7E002058350020603800200E
:1023A000307E0020774A7849D2ED006A774A91ED75
:1023B000006A1278C4ED7E6A84ED7F6A002A00F01C
:1023C000B88476EE665ABCEEC76A7149C4ED7B5A92
:1023D00016EE102AC4ED7C6AA4F8F421FF22D1ED98
:1023E000006A84F8002277EEC77AFEF777B8B5EE78
:1023F000C07AF1EE10FA00F1C385B7EE006A36EE4E
:10240000477AC6EE076AFFF752BADFED626AFFF756
:10241000E7B998ED016A26EE646AB0EE674AA6EE67
:10242000074AB4EEC45A34EE666AF1EE10FAC8BF39
:10243000B0EE656A012B8CED006A3EF42EAE98ED8D
:10244000056A26EE646AB0EE674AA6EE074AB4EE65
:10245000C45A34EE666AF1EE10FAC8BFB0EE656A8F
:10246000022B8CED016A3EF418AE98ED096A26EE57
:10247000646AB0EE674AA6EE074AB4EEC45A34EE78
:10248000666AF1EE10FAC8BFB0EE656A032B8CEDF8
:10249000026A3EF402AE98ED0D6A26EE646AB0EE72
:1024A000674AA6EE074AB4EEC45A34EE666AF1EE05
:1024B00010FAC8BFB0EE656A042B8CED036A3EF4D7
:1024C000ECAD98ED116A26EE646AB0EE674AA6EEAE
:1024D000074AB4EEC45A34EE666AF1EE10FAC8BF89
:1024E000B0EE656A052B8CED046A3EF4D6AD98ED2E
:1024F000156A26EE646AB0EE674AA6EE074AB4EEA5
:10250000C45A74EE666AF1EE10FAC8BFF0EE656A5E
:10251000062BCCED056A3EF4C0ADD8ED196A66EE27
:10252000E46AB0EE674AA6EE874AB3EE046AB4EEF8
:10253000C45A74EE466AF1EE10FAC8BFF0EE656A4E
:10254000072BCCED066A3EF4A8ADD8ED1D6A66EE09
:10255000E44AE4EE877AF4EEC57A77EEC67AF1EED5
:1025600010FAB8BFF0EE657ACCED077AFEF795BDAC
:102570009BF82020C2EB421002EB8002D20092B204
:10258000FEF7F3BC6C600020DC35002040640020C6
:10259000F03500200000C842DFF8DC84B9F1000FFC
:1025A00041F0BF80D8ED006ADDED0C4ADFF8CCC405
:1025B00065EEA66ABDEEC77A17EE101AB0EE667A1F
:1025C000A4EE867AF0EE676AE7EE056ABDEEE67A7B
:1025D00017EE106A17EE100A9E42A8BF1846B142C5
:1025E000C8BF084607EE100AB8EEC77A012A8CED7C
:1025F000007A3EF407AB98ED047ADDED0D6A25EE26
:10260000877AA6EE867AF0EE676AE7EE056ABDEE97
:10261000E67A17EE106A17EE100A9E42A8BF184617
:102620008E42B8BF084607EE100AB8EEC77A022AF3
:102630008CED017A3EF4E6AA98ED087ADDED0E6A9B
:1026400025EE877AA6EE867AF0EE676AE7EE056AEF
:10265000BDEEE67A17EE106A17EE100A9E42A8BF8A
:1026600018468E42B8BF084607EE100AB8EEC77A81
:10267000032A8CED027A3EF4C5AA98ED0C7ADDEDC2
:102680000F6A25EE877AA6EE867AF0EE676AE7EEA5
:10269000056ABDEEE67A17EE106A17EE100A9E4242
:1026A000A8BF18468E42B8BF084607EE100AB8EE1B
:1026B000C77A042A8CED037A3EF4A4AA98ED107A26
:1026C000DDED106A25EE877AA6EE867AF0EE676A6F
:1026D000E7EE056ABDEEE67A17EE106A17EE100A0D
:1026E0009E42A8BF18468E42B8BF084607EE100AA1
:1026F000B8EEC77A052A8CED047A3EF483AA98EDE9
:10270000147ADDED116A25EE877AA6EE867AF0EE70
:10271000676AE7EE056ABDEEE67A17EE106A17EE15
:10272000100A9E42A8BF18468E42B8BF084607EE60
:10273000100AB8EEC77A062A8CED057A3EF462AA32
:1027400098ED187ADDED126A25EE877AA6EE867A84
:10275000F0EE676AE7EE056ABDEEE67A17EE106AFC
:1027600017EE100A9E42A8BF18468E42B8BF084610
:1027700007EE100AB8EEC77A072A8CED067A3EF407
:1027800041AA98ED1C7ADDED136A65EE875AE6EEF4
:10279000265AE5EE257AFDEEE77A17EE900A834297
:1027A000A8BF03468142D8BF194607EE901AF8EE3B
:1027B000E77ACCED077ABEF1000F7EF46EACFEF73F
:1027C00025BAA14A1768B7F832C04FEA5C0C92E408
:1027D000DFF8AC92D4ED017A94ED006AB9F800000C
:1027E000D9F8143077EEA77AF0EE006AB0EE677A87
:1027F000A6EE267A013804EBC002D6EE267A083A15
:102800001033F6EE003A27EE237A67EEA37A84EDD2
:10281000207AC4ED217A8D4CA64604F1800192ED18
:10282000027A92ED036ADEED036ADEED027A53ED81
:10283000014A13ED025A37EE674A76EEC65A77EE32
:10284000277AE4EE845A0138A2F10802E5EE047A10
:102850000EF1080E03F1080336EE267A01F10801A5
:10286000E4EE877AE5EE475A67EEA37A25EEA37A7F
:10287000C1ED007A81ED017AD1D1142F7DF493ABB3
:10288000F6F774F9049BDFF8FC81C01AA8F802007F
:10289000D4F8B061FDF787BBD4F8B481B4F8AC319B
:1028A0000593C3F1200903EB481E694B5FFA89F9D0
:1028B00003EB8E0E5FEA990301F0158601331801D0
:1028C0006449654A0EEB000C0EF1100313ED024A49
:1028D00013ED035A13ED016A13ED047A51ED024A28
:1028E00051ED035A51ED016A51ED047A64EE244A28
:1028F00065EE255A66EE266A67EE277A10339C4508
:1029000042ED024A42ED035A42ED016A42ED047A79
:1029100001F1100102F11002D8D15049A0F11002CA
:10292000964401EB020C224419F0030309D0BEECDB
:10293000017AFCEC017A67EE277A013BE2EC017A3E
:10294000F5D1059B002B41F00382142F7DF42BABB6
:10295000F6F70CF9049BDFF82C81D4F8B061C01AAB
:10296000A8F80200FDF71FBBD4F8B4913C4A3D4BD8
:10297000DFED3D7AD3ED008A3C4B4FEAC9010A44B2
:10298000F8EE688A928809EE102A643AC82AA8BF2D
:10299000C82268EEA78AF8EE497A782AB8BF78226A
:1029A00068EEA78A07EE902A4944B0EE680A03EB66
:1029B0008108B8EEE78A21F0D3F9B8EEC99AF0EEB3
:1029C000409AB0EE680A21F02DF938EE097A79EED6
:1029D000487A28EE098A67EE877AB7EE006A88EEB1
:1029E000277A142FF8EE007A77EE076A60EE277ADE
:1029F00089EEA67A77EE065A36EE477AC6EE256A53
:102A000067EEA67A27EE267AC8ED006A88ED047A8A
:102A1000C8ED026AC8ED017AC8ED037A01F0D385EA
:102A2000134B144A09F1010983FB0938A8EBE97833
:102A300008EB48080136A9EB08081778C4F8B0611C
:102A4000C4F8B4812AE700BF30820020D4200020DF
:102A500038390020C83A0020E4200020B83A00208D
:102A6000383B00205C49002027D4D23678740020FF
:102A7000565555552C7E00205835002060380020D2
:102A800020390020307E0020DFF8FC93B9F800E008
:102A9000D9F804C04FEA5E084FEA880204EB8E06BC
:102AA0005FEADE0E04EB020300F0A08010320EF1AC
:102AB000010EED4803EB0E1E324410330CF11007EB
:102AC00006F1100151ED032A51ED043A10ED043ADC
:102AD00010ED032A51ED026A11ED016A10ED020AB0
:102AE00010ED018A12ED044A12ED035A53ED044A27
:102AF00053ED035A13ED027A53ED017A52ED020AB7
:102B000012ED011A73EE238A72EE221A40ED048A46
:102B100040ED031A70EE268A78EE061A40ED028A1E
:102B200040ED011A74EE848A75EE851A43ED048A2D
:102B300043ED031A77EE208A77EE811A43ED028A7D
:102B400043ED011A73EE633A75EE655A17ED035AB9
:102B500032EE623A74EE644A65EE631A17ED044A87
:102B600023EE052A64EE652AE3EE041A10339E452F
:102B700024EE843AA3EE842A00F1100007F1100736
:102B8000A5EE853A01F1100102F11002E4EE852A6A
:102B900041ED071A01ED082A02ED073A42ED082A35
:102BA00057ED055A17ED065A70EE666A38EE466A1A
:102BB00030EEC77A71EE677A26EE253A65EEE63A90
:102BC00025EE674A67EE054AE6EE053AA6EE853A37
:102BD000A7EE254AE7EEA54A01ED063A41ED053A92
:102BE00002ED064A42ED054A7FF46CAF1FFA88F801
:102BF000624641469D481BF023FC4146D9F804201B
:102C000030461BF01DFC9A4B1B78142B7FF440AE12
:102C100036E6DFF874929548D9F80820B9F80C1018
:102C200020F0E6F8924B1F78142F01F0DA84D4F8E4
:102C3000B0610136C4F8B061CCE5DFF8509299F884
:102C40000020900801F02285DFF844C200F101085D
:102C50004FEA48180CEB080E0CF12003ACF17001A0
:102C600013ED076A53ED056A13ED037A53ED017A0C
:102C700053ED025A13ED084A53ED064A13ED045A78
:102C800026EE066A66EEA66A27EE077A67EEA77A50
:102C9000A4EE046A20339E45E4EEA46A01F110011B
:102CA000A5EE057AE5EEA57AF1EEC65AB1EEE66A32
:102CB000F1EEC76AB1EEE77A41ED085A01ED076A15
:102CC00041ED066A01ED057ACAD1A8F12008C44495
:102CD00004EB001012F0030318BF0CF1080C0FD026
:102CE0005CED017A1CED027A67EEA77A013BE7EE14
:102CF000077A0CF1080CB1EEE77AA0EC017AEFD17B
:102D0000142F01F050840136C4F8B061FDF7B4B857
:102D1000F5F72CFF564B04901F78142F05BFDFF8F2
:102D20007481D4F8B061D4F8B061A8F80060FDF700
:102D300088B876EEC65AF0EE466AFFF744BB4D4AB5
:102D40004D49D2ED007A4D4A91ED007A1278C4EDEA
:102D50007E7A84ED7F7A002A01F0EC8277EE676A52
:102D60004749C4ED7C7AC4ED7B6AFF22D1ED006A4D
:102D7000DFED4A7A84F80022FDF7B0BB414FDFF85F
:102D8000189197ED004A97ED057AD7ED014A97ED36
:102D9000066AD7ED046A97ED035AD7ED025A67EE3B
:102DA000897A09EB8603A4EE277AA4EEA76A66EE79
:102DB000C76AA5EE476AE5EEA76A20EE070A87ED27
:102DC000056AC7ED066A83ED007A29EE088A20F0CD
:102DD0007BFF69EE288AD7ED0E5A97ED176A97EDBB
:102DE000091AD7ED121A97ED0F5A97ED187A97ED49
:102DF0000A2AD7ED132AD7ED0D6AD7ED167A97ED8B
:102E00000C3AD7ED0B3A97ED154AD7ED144AE1EE9F
:102E1000085A002209EB8603A8EEA16A00B2C4F8A2
:102E20009C21A2EE085AC4F8A021C4F8A421A8EE5F
:102E3000A27A66EEE56A67EEC67AA3EE655AE3EE1D
:102E4000886AA6EE447AE8EEA47A87ED0E5AC3EDBE
:102E5000205AC7ED0F6A83ED406A87ED177AC7EDF8
:102E6000187AFEF7CEBB00BFE4200020D42000205B
:102E70002C7E00206C600020DC35002040640020A7
:102E8000F0350020BC3B0020203900201A390020FA
:102E900054210020307E002038390020000000003E
:102EA000B5F93C306A6207EE903A0122F8EEE77A13
:102EB000EB66C5F888200023012FC5ED1F7AC5ED0C
:102EC0001E7AC5F8803001F05882B7427DF4F2AE28
:102ED000B5F93E302B6707EE903A00220123F8EE59
:102EE000E77AAA62C5F89C300023012FC5ED247A49
:102EF000C5ED237AC5F8943001F03B82B7427DF4EA
:102F000009AFB5F940306B6707EE903A0022012314
:102F1000F8EEE77AEA62C5F8B0300023012FC5ED7C
:102F2000297AC5ED287AC5F8A8307DF423AF1FEDC6
:102F3000258AB9F1030F2BD0BAF1000F09D007EEA3
:102F400090AAF8EEE77AF4EEC87AF1EE10FA01F101
:102F50002084C24A6B6F1268A8F80600002103EBB8
:102F6000560393FBF6F6EE6291621163D162FDF7B0
:102F700003BFBB4B9B7B002B3EF4D9A9FDF7DBBF06
:102F8000F7EE006AFEF793BCF7EE006AFEF730BD7D
:102F9000B0EE480A20F098FE00B2CDE7B4F84861E0
:102FA000013E36B2002EA4F848617EF7B2ABAD4ABE
:102FB000FEF72EB8B4F81A2102F57A7292B2FDF734
:102FC000D4BFA94BDFEDA97A93ED080AB4EEE70A66
:102FD000F1EE10FA40F21387049120F00BFFD4EDCC
:102FE000457A20EE270A20F06FFEB0F5617F049944
:102FF00001F3408007EE900AF8EEE76ADFED9C7A75
:1030000066EEA76A07EE906AB8EEE77AFDEEE67A1A
:1030100017EE903A2033402B41F2F4829FED950A4F
:10302000049120F051FE00B207EE900A0499B8EE28
:10303000E77A8C4AD2ED037A77EE877AC2ED037A8B
:10304000FDF781BF8C4F3A78013A0A2A1CD8DFE895
:1030500012F064018D01CB00AA009200760062009C
:10306000510040012B010B00844A854952680968D0
:10307000C8328A4203D319F07DF928B1B378032B03
:1030800001F0118401233B70F378002B3EF4ECAC8B
:103090007C4B1B78D80740F14981DFF8E481D4F8F4
:1030A0009821D8F800309A4200F24C813B78012BED
:1030B0003EF4DAAC94F89421002A3EF4D5AC0B2B04
:1030C0000DD801229A4040F6030112EA01060CD104
:1030D00012F4C06F03D0093B012B41F28684674B89
:1030E000D8F800205A600B233B70002384F89431F9
:1030F000FEF7BABC19F01CF915F0ECFF0028C3D09C
:1031000019F038F90028BFD05F4A604B12681A6086
:103110000A233B70B8E719F00BF95D4B002105203D
:103120008DE80300A3F108020291532016F0C4FCBD
:103130000028A9D1514A082310603B70A4E719F078
:10314000F7F8544A0292A2F10C034FF007080193DA
:10315000CDF80080A2F108030021143A472016F0B0
:10316000ABFC002890D1454B87F800804FF0FF3230
:1031700083E8050088E719F0DBF8474B00210220BF
:103180008DE80300A3F108020291482016F094FC98
:1031900000287FF479AF394B4FF0FF3106221860D9
:1031A00059603A7070E719F0C3F83C4A0292A2F1F4
:1031B0000C03282101930091A2F10A035021163A31
:1031C000492016F079FC00287FF45EAFDAF8003071
:1031D00013F0800301F05E83284B4FF0FF3105228E
:1031E000186059603A704FE7DFF8908019F0A0F846
:1031F000234AD8F80430126864339342BFF444AFD2
:10320000402019F079F800287FF43EAFD8F800305C
:103210002349DFF890B04FF0400A11E0049119F013
:10322000CDF8DBF80020D8F800300499013A0133DA
:10323000BAF1010ACBF80020C8F8003001F0BB83D6
:10324000CB5C1846002BE9D100234FF0FF32C8F8C1
:1032500000300423C8F804203B7015E79047002095
:1032600088620020F47E0020A04700208FC2753CB9
:10327000D06D393A000000007B830020EC61002013
:10328000E87600208D7D0020546000204C600020F6
:10329000746403082C640308106403083E62030886
:1032A000D8610308AC680020DE4B1B78002B01F0CE
:1032B000A4811A200AF0F4FD002841F09E8194F8C0
:1032C0009431002B41F0998109233B7015F0DAFE0F
:1032D000DAE61A200AF0E4FD0028F7D0D24B1B886A
:1032E000002BF3D1D14B4520D3F8008019F066F8BC
:1032F0000E2019F063F8404615F04CFBDDF82080F5
:10330000404615F047FBCA4ACA4B12681A6040464D
:103310000A233B7015F0A2FBD8E7C74B1B78DB07ED
:1033200001F19B82F378002B3EF49EAB09F0CAFCBE
:1033300000283FF4B2AEC14B1B6803F59C53083321
:10334000C4F898313B78012B7EF48EAB94F894311D
:10335000002B7EF489ABB378032B01F03B830BF099
:1033600037FD012384F89431FEF77EBBB34BB44A9A
:103370001B685360B3490023136003220B603A704B
:1033800082E6099B93F800E00EF0010EBEF1000FFB
:103390007DF483AEFDF73ABCAB4BDFEDAC7A1E6833
:1033A000C4ED707A16F0805640F0768310F48006F3
:1033B00000F0AD810026B6EE007A67EE877AF4EE73
:1033C000E75AF1EE10FA48BFF0EE675A40F1648315
:1033D000C4ED815AFDF7C1BAF5F7C8FB8146FDF788
:1033E00096BD74EE677AB7EE007AF4EEC77AF1EE26
:1033F00010FAC4ED707A40F3B18784EEA77A8DEDB0
:103400000C7AFDF7A0BABAF1000F00F07D8698EDB6
:10341000007ADDED0C6ADFF838C225EE877AA6EE79
:10342000867AF0EE676AE7EE056ABDEEE67A17EE99
:10343000106A17EE100A9E42A8BF1846B142C8BFD4
:10344000084607EE100AB8EEC77A012A8CED007A1A
:103450003DF423AE98ED047ADDED0D6A25EE877A12
:10346000A6EE867AF0EE676AE7EE056ABDEEE67ACA
:1034700017EE106A17EE100A9E42A8BF1846B14216
:10348000C8BF084607EE100AB8EEC77A022A8CEDCC
:10349000017A3DF402AE98ED087ADDED0E6A25EE74
:1034A000877AA6EE867AF0EE676AE7EE056ABDEEE9
:1034B000E67A17EE106A17EE100A9E42A8BF184669
:1034C000B142C8BF084607EE100AB8EEC77A032A11
:1034D0008CED027A3DF4E1AD98ED0C7ADDED0F6AEA
:1034E00025EE877AA6EE867AF0EE676AE7EE056A41
:1034F000BDEEE67A17EE106A17EE100A9E42A8BFDC
:103500001846B142C8BF084607EE100AB8EEC77A9F
:10351000042A8CED037A3DF4C0AD98ED107ADDED10
:10352000106A25EE877AA6EE867AF0EE676AE7EEF5
:10353000056ABDEEE67A17EE106A17EE100A9E4293
:10354000A8BF1846B142C8BF084607EE100AB8EE39
:10355000C77A052A8CED047A3DF49FAD98ED147A74
:10356000DDED116A25EE877AA6EE867AF0EE676ABF
:10357000E7EE056ABDEEE67A17EE106A17EE100A5E
:103580009E42A8BF1846B142C8BF084607EE100ABF
:10359000B8EEC77A062A8CED057A3DF47EAD98ED3B
:1035A000187ADDED126A25EE877AA6EE867AF0EEBD
:1035B000676AE7EE056ABDEEE67A17EE106A17EE67
:1035C000100A9E42A8BF1846B142C8BF084607EE7F
:1035D000100AB8EEC77A072A8CED067A3DF45DAD85
:1035E00098ED1C7ADDED136A65EE875AE6EE265AF1
:1035F000E5EE257AFDEEE77A17EE902A9342A8BF12
:1036000013468A42A8BF194607EE901AF8EEE77AE9
:10361000CCED077AFDF741BDD6003EF565ADFDF76F
:1036200097BC00BFDC3800204460002040600020D0
:10363000546000204C6000208D7D0020E876002042
:10364000EC610020AC680020CC610020000000800C
:1036500060380020012A40F3908607EE101AB8EE79
:10366000C77AC7EE876AB1EEE68AB9F1030F13D0C5
:10367000BAF1000F09D007EE90AAF8EEE77AF4EE5F
:10368000C87AF1EE10FA01F18480EB6E03EB560379
:1036900093FBF6F36B6218E4B0EE480A20F014FBDB
:1036A00000B2E5E7012A7FF742AC07EE101AB8EE48
:1036B000C77AC7EE876AB1EEE68A3AE4012A40F398
:1036C000588607EE101AB8EEC77AC7EE876AB1EED1
:1036D000E68AB9F1030F14D0BAF1000F09D007EE52
:1036E00090AAF8EEE77AF4EEC87AF1EE10FA01F15A
:1036F00050802B6F03EB560393FBF6F3AB62FFF79F
:10370000FDBBB0EE480A20F0DFFA00B2E4E7B6EE07
:10371000007AF4EEC75AF1EE10FA3FF74CAEFDF71F
:103720001CB9D8ED004A9DED0C4ADFF820C665EEC5
:10373000A44AFDEEC73AE4EE064AB0EE674AA4EEAC
:10374000854A13EE901AF4EEC46AF1EE10FAF0EE28
:10375000444A88BFF0EE474AFDEEE44A14EE900A70
:1037600014EE906A9842A8BF1E468142C8BF0E461A
:1037700004EE906AF8EEE44A012ACCED004A3DF4EA
:1037800041AAD8ED044A9DED0D4A65EEA44AE4EE47
:10379000064AB0EE674AA4EE854AF4EEC46AF1EE3A
:1037A00010FAF0EE444A88BFF0EE474AFDEEE44AD4
:1037B00014EE900A14EE906A9842A8BF1E46884202
:1037C000B8BF0E4604EE906AF8EEE44A022ACCED49
:1037D000014A3DF417AAD8ED084A9DED0E4A65EE60
:1037E000A44AE4EE064AB0EE674AA4EE854AF4EE37
:1037F000C46AF1EE10FAF0EE444A88BFF0EE474A90
:10380000FDEEE44A14EE900A14EE906A9842A8BFC6
:103810001E468842B8BF0E4604EE906AF8EEE44AAF
:10382000032ACCED024A3DF4EDA9D8ED0C4A9DEDFA
:103830000F4A65EEA44AE4EE064AB0EE674AA4EEEB
:10384000854AF4EEC46AF1EE10FAF0EE444A88BFFD
:10385000F0EE474AFDEEE44A14EE900A14EE906A48
:103860009842A8BF1E468842B8BF0E4604EE906A32
:10387000F8EEE44A042ACCED034A3DF4C3A9D8ED9E
:10388000104A9DED104A65EEA44AE4EE064AB0EEF9
:10389000674AA4EE854AF4EEC46AF1EE10FAF0EE3F
:1038A000444A88BFF0EE474AFDEEE44A14EE900A1F
:1038B00014EE906A9842A8BF1E468842B8BF0E46D2
:1038C00004EE906AF8EEE44A052ACCED044A3DF491
:1038D00099A9D8ED144A9DED114A65EEA44AE4EE8B
:1038E000064AB0EE674AA4EE854AF4EEC46AF1EEE9
:1038F00010FAF0EE444A88BFF0EE474AFDEEE44A83
:1039000014EE900A14EE906A9842A8BF1E468842B0
:10391000B8BF0E4604EE906AF8EEE44A062ACCEDF3
:10392000054A3DF46FA9D8ED184A9DED124A65EE9F
:10393000A44AE4EE064AB0EE674AA4EE854AF4EEE5
:10394000C46AF1EE10FAF0EE444A88BFF0EE474A3E
:10395000FDEEE44A14EE900A14EE906A9842A8BF75
:103960001E468842B8BF0E4604EE906AF8EEE44A5E
:10397000072ACCED064A3DF445A9D8ED1C4A9DED39
:10398000134A65EEA45AE6EE045AE5EE257AF4EE03
:10399000E76AF1EE10FAC8BFF0EE477AFEF7FBBE19
:1039A000E34BE44AB3F90430DFEDE37A82FB031220
:1039B000DB17C3EBA2031BB208EE103AB8EEC88ABD
:1039C00028EE278AB0EE480AF6F7C6FEF0EE408AE7
:1039D000B0EE480AF6F746FED84BD878002800F03B
:1039E0006383D749B4F98E31B1F9022044F25066AD
:1039F000D21AB24240F36F85A2F50C42A03A464279
:103A0000964200F3CC848242A8BF0246B1F900106E
:103A1000B4F98C711344CA1B44F250611BB28A4240
:103A2000A4F88E3140F3BE84A2F50C42A03A96422F
:103A300003DC9042A8BF10460646BA1912B207EE40
:103A4000902A07EE103AF8EEE77AF8EEC76A27EE0A
:103A5000E87A60EE277AA0EE267AA4F88C21E8EEC8
:103A6000A67ADFEDB86A27EE267A67EEA67ABDEE73
:103A7000C77AFDEEE77A17EE102A17EE903AA4F80F
:103A80009021A4F89231FDF7E7BF8223FCF777BAC3
:103A9000DFEDAD7AFCF73EBAB7EE007A77EE677AE3
:103AA000F4EEE75AF1EE10FA88BFF0EE675A8FE4B1
:103AB000D8ED004A9DED0C4ADFF890C265EEA44AAD
:103AC000FDEEC73AE4EE064AB0EE674AA4EE854A38
:103AD00013EE901AF4EEC46AF1EE10FAF0EE444AD6
:103AE00088BFF0EE474AFDEEE44A14EE900A14EE69
:103AF000906A9842A8BF1E468142C8BF0E4604EE97
:103B0000906AF8EEE44A012ACCED004A3DF4C0AADE
:103B1000D8ED044A9DED0D4A65EEA44AE4EE064A4E
:103B2000B0EE674AA4EE854AF4EEC46AF1EE10FAEC
:103B3000F0EE444A88BFF0EE474AFDEEE44A14EE48
:103B4000900A14EE906A9842A8BF1E468842B8BFF9
:103B50000E4604EE906AF8EEE44A022ACCED014AE1
:103B60003DF496AAD8ED084A9DED0E4A65EEA44AAA
:103B7000E4EE064AB0EE674AA4EE854AF4EEC46A63
:103B8000F1EE10FAF0EE444A88BFF0EE474AFDEE3F
:103B9000E44A14EE900A14EE906A9842A8BF1E46BA
:103BA0008842B8BF0E4604EE906AF8EEE44A032A53
:103BB000CCED024A3DF46CAAD8ED0C4A9DED0F4ABB
:103BC00065EEA44AE4EE064AB0EE674AA4EE854AE2
:103BD000F4EEC46AF1EE10FAF0EE444A88BFF0EE5B
:103BE000474AFDEEE44A14EE900A14EE906A9842B9
:103BF000A8BF1E468842B8BF0E4604EE906AF8EE93
:103C0000E44A042ACCED034A3DF442AAD8ED104A16
:103C10009DED104A65EEA44AE4EE064AB0EE674A0E
:103C2000A4EE854AF4EEC46AF1EE10FAF0EE444ACE
:103C300088BFF0EE474AFDEEE44A14EE900A14EE17
:103C4000906A9842A8BF1E468842B8BF0E4604EE4E
:103C5000906AF8EEE44A052ACCED044A3DF418AA2D
:103C6000D8ED144A9DED114A65EEA44AE4EE064AE9
:103C7000B0EE674AA4EE854AF4EEC46AF1EE10FA9B
:103C8000F0EE444A88BFF0EE474AFDEEE44A14EEF7
:103C9000900A14EE906A9842A8BF1E468842B8BFA8
:103CA0000E4604EE906AF8EEE44A062ACCED054A88
:103CB0003DF4EEA9D8ED184A9DED124A65EEA44AEE
:103CC000E4EE064AB0EE674AA4EE854AF4EEC46A12
:103CD000F1EE10FAF0EE444A88BFF0EE474AFDEEEE
:103CE000E44A14EE900A14EE906A9842A8BF1E4669
:103CF0008842B8BF0E4604EE906AF8EEE44A072AFE
:103D0000CCED064A3DF4C4A9D8ED1C4A9DED134AFA
:103D100065EEA45AE6EE045AE5EE257AF4EEE76A7B
:103D2000F1EE10FAC8BFF0EE477AFEF750B900BFC7
:103D3000EC4500206766666635FA8E3CE03F002061
:103D40003C400020CDCCCC3D000002436038002038
:103D5000E34B03EBC818059B4FEA890E5FEA930912
:103D600001EB0E0CA64400F0758509F101094FEA3C
:103D7000091908EB090008F110030CF110010EF10C
:103D8000100213ED024A13ED035A13ED016A13ED0D
:103D9000047A51ED024A51ED035A51ED016A51ED99
:103DA000047A64EE244A65EE255A66EE266A67EECA
:103DB000277A1033984242ED024A42ED035A42ED0F
:103DC000016A42ED047A01F1100102F11002D8D12A
:103DD000A9F11009059BC8440CEB0901CE4413F06E
:103DE00003033EF4B2ADB8EC017AF1EC017A67EE70
:103DF000277A013BEEEC017AF5D1FEF7A6BD9FEDE7
:103E0000B97AFFF716B9BAF1000F00F08683DFF830
:103E1000F0829DED0C4AD8ED004A65EEA44AE4EE2E
:103E2000064AB0EE674AA4EE854AF0EE444AB9F17C
:103E3000000F06D0F4EE446AF1EE10FAC8BFF0EEBF
:103E4000474ABDEEC77A17EE101ABDEEE47A04EECB
:103E5000901A17EE100A814200F3EC849842A8BF32
:103E6000184607EE100AB8EEC77ADFF898C2012AA2
:103E70008CED007A3DF411A998ED047A9DED0D4A80
:103E800025EE877AA4EE067AB0EE674AA7EE054AD9
:103E9000B0EE447AB9F1000F00F07084F4EEC46A19
:103EA000F1EE10FA40F36A8408469842A8BF18461B
:103EB00007EE100AB8EEC77A022A8CED017A3DF4BB
:103EC000ECA898ED087A9DED0E4A25EE877AA4EECF
:103ED000067AB0EE674AA7EE054AB0EE447AB9F129
:103EE000000F00F04084F4EEC46AF1EE10FA40F3E3
:103EF0003A8408469842A8BF184607EE100AB8EE62
:103F0000C77A032A8CED027A3DF4C7A898ED0C7AA3
:103F10009DED0F4A25EE877AA4EE067AB0EE674A49
:103F2000A7EE054AB0EE447AB9F1000F00F0108414
:103F3000F4EEC46AF1EE10FA40F30A84084698429F
:103F4000A8BF184607EE100AB8EEC77A042A8CED0F
:103F5000037A3DF4A2A898ED107A9DED104A25EE63
:103F6000877AA4EE067AB0EE674AA7EE054AB0EE6D
:103F7000447AB9F1000F00F0E183F4EEC46AF1EE87
:103F800010FA40F3DB8308469842A8BF184607EEB4
:103F9000100AB8EEC77A052A8CED047A3DF47DA8A4
:103FA00098ED147A9DED114A25EE877AA4EE067AF3
:103FB000B0EE674AA7EE054AB0EE447AB9F1000FB9
:103FC00000F0B283F4EEC46AF1EE10FA40F3AC8371
:103FD00008469842A8BF184607EE100AB8EEC77AFE
:103FE000062A8CED057A3DF458A898ED187A9DEDD7
:103FF000124A25EE877AA4EE067AB0EE674AA7EE5B
:10400000054AB0EE447AB9F1000F00F04C83F4EEAB
:10401000C46AF1EE10FA40F3468308469842A8BFFE
:10402000184607EE100AB8EEC77A072A8CED067A12
:104030003DF433A898ED1C7A9DED134A65EE875A3E
:10404000E4EE065AE5EE857AB9F1000F00F023831D
:10405000F4EEE67AF1EE10FA40F11D830A469A4238
:10406000A8BF1A4604EE902AF8EEE44ACCED074ABF
:10407000FDF713B807EE906ADFED1B6AB8EEE77A3A
:1040800066EEA65A9FED195A9FED196ADFED197A6F
:10409000A5EE856A26EEA55AE5EE867AE5EE276A54
:1040A00026EE870AFEF7BCBF134B9FED146AB3F9E7
:1040B0000020B3F9023007EE902A06EE903AF8EEAF
:1040C000E77AF8EEE66A27EEE87A60EE277AA0EE65
:1040D000267AE8EEA67A27EE067A67EE867AC6E4B6
:1040E000383900200000000084F9223F92E741B9EE
:1040F0009730083C15A82ABE3C400020CDCCCC3DD2
:104100005835002060380020D8ED006ADDED0C4AFB
:1041100065EEA66AE4EE866AF0EE674AE6EE854A48
:10412000FDEEE46A16EE90EA714500F3ED819E45DE
:10413000A8BF9E4606EE90EAF8EEE66A002E00F072
:104140006284DFF8A8C5012ACCED006A3CF4A5AF73
:10415000D8ED046ADDED0D4A65EEA66AE4EE866AE6
:10416000F0EE674AE6EE854AFDEEE46A16EE90EA66
:10417000714500F3C6819E45A8BF9E4606EE90EAB3
:10418000F8EEE66A002E00F09884022ACCED016A6F
:104190003CF483AFD8ED086ADDED0E4A65EEA66A01
:1041A000E4EE866AF0EE674AE6EE854AFDEEE46AE2
:1041B00016EE90EA714500F3A1819E45A8BF9E4688
:1041C00006EE90EAF8EEE66A002E00F06B84032A11
:1041D000CCED026A3CF461AFD8ED0C6ADDED0F4A1C
:1041E00065EEA66AE4EE866AF0EE674AE6EE854A78
:1041F000FDEEE46A16EE90EA714500F37C819E457F
:10420000A8BF9E4606EE90EAF8EEE66A002E00F0A1
:104210003E84042ACCED036A3CF43FAFD8ED106A2B
:10422000DDED104A65EEA66AE4EE866AF0EE674AB6
:10423000E6EE854AFDEEE46A16EE90EA714500F37B
:1042400069819E45A8BF9E4606EE90EAF8EEE66AB2
:10425000002E00F0ED83052ACCED046A3CF41DAF7E
:10426000D8ED146ADDED114A65EEA66AE4EE866AC1
:10427000F0EE674AE6EE854AFDEEE46A16EE90EA55
:10428000714500F344819E45A8BF9E4606EE90EA24
:10429000F8EEE66A002E00F0C183062ACCED056A2E
:1042A0003CF4FBAED8ED186ADDED124A65EEA66A65
:1042B000E4EE866AF0EE674AE6EE854AFDEEE46AD1
:1042C00016EE90EA714500F313819E45A8BF9E4605
:1042D00006EE90EAF8EEE66A002E00F0CE83072A9A
:1042E000CCED066A3CF4D9AED8ED1C6ADDED134A7C
:1042F00065EEA65AE4EE865AE5EE857AFDEEE77A9B
:1043000017EE902A914203DC9A42A8BF1A46114642
:1043100007EE901AF8EEE77A002E7FF479A9059B54
:10432000002B7FF475A9049B5B45B8BFF0EE477A7C
:10433000FFF76EB977EEC76AF0EE477AFEF710BD69
:10434000BA8E9FEDDE7A07EE902AF8EEE77ADC4A25
:1043500067EE877AC2ED007AFCF7FABDD94B1E688A
:1043600016F080567FF427A8FFF720B8D64AFCF74E
:1043700047BE9FEDD68AFFF7ACB99FEDD48AFFF711
:1043800074B99FEDD30ADFF8688325EE800A1FF029
:104390009BFCD4F8B061A8F80600FBF704BE3246D7
:1043A000FFF734BBCB498A42BCBF02F50C42A032B6
:1043B000FFF73DBB07EE906A9FEDC77ADFEDD36A4A
:1043C00084F88461F8EEE77A67EE877A37EEA67AAA
:1043D000BDEEC76A16EE103A2033402B40F2E28160
:1043E000DFEDBA6AB64BBDEEE77AC3ED016A17EEB0
:1043F000103A2033402B00F2D2819FEDC57AF4EEC3
:10440000C77AF1EE10FA40F36382DFEDBE5A9FEDFA
:10441000BC6A01E0F0EE477AF4EEC67AF1EE10FAEB
:1044200037EEE57AF6DCDFEDBF7AB4EEE77AF1EE4F
:1044300010FA40F14A82DFEDB35A9FEDB36A01E012
:10444000B0EE677AB4EEC67AF1EE10FA77EE257A1E
:10445000F6D49FEDAE7AF4EEC77AF1EE10FA40F39F
:10446000ED819FEDAB7A77EE677A67EEA75A9FED05
:10447000A95A9FEDA96A9FEDA97AA5EE856A27EE54
:10448000A55AA5EE867AE5EE077AC4ED627AFDF7C5
:10449000A7BE92ED000A059304921FF015FC8F4908
:1044A000DFF850E2D1F8EC10DFF84482049AA8F863
:1044B00000008EFB013EC917C1EBAE1107EE901A4A
:1044C000F8EEE77A059BFDEEE77A17EE901AA8F86A
:1044D0000210FCF79ABD7F4EB242BCBF02F50C42FF
:1044E000A032FFF78CBA7E497E4A8C46FEF71CBA92
:1044F00006EE901AEEE606EE901A85E606EE901AA3
:1045000060E606EE901A3BE606EE901A14E606EE1A
:10451000901ABDE606EE901A98E6FDEEC74A0DF138
:10452000300E9A46DFF8D0C1DFF8C08114EE901A41
:104530000EEB82024B4606E07245E8EC014A0CF1B4
:10454000100C3CF4AAADDCED004ABEEC014A65EE6D
:10455000A44AE6EE044AB0EE674AA5EE244AF0EE1D
:10456000444A33B1F4EE446AF1EE10FAC8BFF0EEFB
:10457000474AFDEEE44A14EE909A494504EE901A3B
:1045800004DCD145A8BFD14604EE909AF8EEE44A87
:10459000002ED1D105980028CED104985845B8BF37
:1045A000F0EE474AC8E7F4F7E1FA4F4BDFF84081F5
:1045B0001F78049B99F80020D4F8B061C01AA8F8BD
:1045C0000400FEF7A0BBF4F7D1FA049BDFF82081CA
:1045D000D4F8B491D4F8B061C01AA8F80200FEF77C
:1045E0001FBAF4F7C3FA404BDFF804811F78049B2D
:1045F000C01AA8F80200FEF71ABB089814F02EFAA9
:10460000FEF764BEDFED427AF4EEE76AF1EE10FAEF
:1046100040F3E881DFED3B5A9FED396A01E0F0EEAF
:10462000676AF4EEC66AF1EE10FA76EEE57AF6DC29
:10463000DFED3C6AF4EEE67AF1EE10FA40F1C78164
:10464000DFED305A9FED306A01E0F0EE667AF4EE6D
:10465000C67AF1EE10FA77EEA56AF6D4DFED2B7A82
:10466000F4EEE76AF1EE10FA04DDDFED297A77EE79
:10467000E66A05E5DFED2A7AF4EEE76AF1EE10FA74
:1046800044BFDFED287A77EEE66AF9E4154800F1D9
:10469000800CFEF71FBBFDEEE77A17EE902A8A42E8
:1046A000FFF6E2ACDBE4BDEEC77A17EE100A8842F3
:1046B000BFF6B4AC07EE101AB5E400BF6F12833A30
:1046C000A0000020CC610020F47E0020000000004B
:1046D0000000C842B0B9FFFF35FA8E3C5C010020F3
:1046E000B83A0020D42000202C7E00206038002022
:1046F000307E0020D34D62105835002000000000AD
:10470000E4CB1641DB0FC940E4CB16C1DB0FC93F38
:10471000DB0F494092E741B99730083C15A82ABE03
:10472000DB0FC9BFDB0F49C0BDEEC77A17EE100A19
:104730008842BFF64EAC07EE101A4FE4BDEEC77AC2
:1047400017EE100A8842BFF61FAC07EE101A20E4DD
:10475000BDEEC77A17EE100A8842BFF6F0AB07EE3F
:10476000101AFFF7F1BBBDEEC77A17EE100A8842A8
:10477000BFF6C0AB07EE101AFFF7C1BBBDEEC77A9C
:1047800017EE100A8842BFF690AB07EE101AFFF73B
:1047900091BBA8F80600A5F8B460FCF7F3BA5FED8A
:1047A000297A72E6F4EEE67AF1EE10FA40F3BE8072
:1047B0005FED2C5A1FED2E6A01E0B0EE667AB4EE82
:1047C000C67AF1EE10FA77EE656AF6DC1FED2B7A09
:1047D000F4EEC76AF1EE10FA40F1A5805FED375AAA
:1047E0001FED376A01E0F0EE476AF4EEC66AF1EEBB
:1047F00010FA36EEA57AF6D45FED3C6AB4EEE67AAE
:10480000F1EE10FA33DD5FED3E6A36EEC77A67EE01
:10481000075A1FED405A1FED406A5FED406AA5EE52
:10482000856A27EE255AE5EE866AA5EE267AF0EE31
:10483000476AD7E507EE101AFFF715BB1FED487A58
:10484000F4EEC77AF1EE10FA44BF1FED4A7A77EE24
:10485000677A0AE66146FFF7C2BA802012F0D2F802
:1048600008B11DF0EFFA0AF0B3FAFEF70DBC5FEDE8
:10487000546AB4EEE67AF1EE10FA44BF5FED576A7F
:1048800036EEC77AC3E794F8E031002B7BF4EDAD48
:10489000FBF7D9BD8E4A4FF0FF31136007235160FB
:1048A0003B70FEF7F1BBDFF87082D8F800001DF016
:1048B000A1FA884B1B780022022BC8F800207EF456
:1048C000E1AB1DF093F9FEF7DDBBF0EE477AC0E5F2
:1048D000B0EE677AA7E5DFED807AF4EEE7CAF1EE95
:1048E00010FA6EDCDFED7D7AF4EEE7CAF1EE10FA35
:1048F00067D47B4BD3ED007AB1EE677AB4EEC7CACA
:10490000F1EE10FA60D4B4EEE7CAF1EE10FA88BF07
:10491000B0EE67CA734BC7ED00AA1B689A427BF7DB
:10492000DDACFCF7B5BEB0EE667A65E7F0EE476A3F
:104930004CE76D4A6D4B10681B689847079B9BEDD1
:10494000007AD3ED007A6A4BD7ED006A93ED006AE6
:10495000684B83ED020A684B67EE277A2B4427EEFB
:104960008B7AD3ED007A67EE277AF0EE665AECEE9A
:10497000275AB1EE467AB4EEE57AF1EE10FA08DC89
:10498000B4EEE56AF1EE10FA8CBFB0EE657AB0EEE7
:10499000467A5A4B1B78012B02D0192B7BF4DBACE7
:1049A000DFED577AB4EEE7CAF1EE10FACCBF01237F
:1049B0000023FBF7DBBCCB5C002B7EF465ABFEF782
:1049C00043BC9FED50CAA5E7B0EE47CAA2E7F0EEA0
:1049D000676A43E6802012F015F800287DF444A8A9
:1049E000FEF7BDBCF0EE667A22E6452017F0E6FC45
:1049F000FF2017F0E3FC444817F0CCFC304617F0DA
:104A0000DDFCFEF76CBB059800287FF49AAB049898
:104A10005845B8BFF0EE476AFFF793BB05980028EA
:104A20007FF43BAC04985845B8BFF0EE476A34E4D5
:104A3000059800287FF40FAC04985845B8BFF0EEF5
:104A4000476A08E4132B05D1B0EE480A1FF03CF981
:104A50002E4B1880B0EE480AD5F878372C48984786
:104A60002C4B1B78132BB0EE408A7BF4DCAA1FF092
:104A70002BF9264B5880FBF7D6BA059800287FF40F
:104A80002EAC04985845B8BFF0EE476A27E4059865
:104A900000287FF4BEAB04985845B8BFF0EE476AD3
:104AA000FFF7B7BB059800287FF491AB04985845F1
:104AB000B8BFF0EE476AFFF78ABB059800287FF47D
:104AC00064AB04985845B8BFF0EE476AFFF75DBB8A
:104AD000EC6100208038002000C0F84400C0F8C419
:104AE00024350020083500209C340020B0340020FC
:104AF0002835002018380020C0340020EC2E00207B
:104B000000009642000000002C890308307E00203F
:104B1000787400202C7E0020B06800202DE9F04F32
:104B20002DED028B744B754A1C7893B000F59C41B7
:104B30002031814606911160002C00F0D886704A21
:104B40001268904240F2BE826E4A049212686E4928
:104B50006E4D6F4E0291013C1C7002F4805EBEF1FE
:104B6000000F40F0BC826B4B05931F7807F00107E4
:104B7000029B5B7D002B40F08F86049B1B68190411
:104B800001F14481644B9945B37800F24F85002BC5
:104B900040F04F85B5F90630049AD2F8009019F428
:104BA000805A40F00E86029AB2F81AB05B45B4BF44
:104BB0004FF0000B4FF0010B584B1B6813F0805364
:104BC00000F0C182002F00F0C2820299544A498C41
:104BD00092ED037A039207EE901AF8EEE77AB4EEBC
:104BE000E77AF1EE10FA81F29D81BBF1000F40F0FF
:104BF000B8824C4C94F8A020002A40F0B2824A4976
:104C00004A4A086890F82D000021116051609160B7
:104C1000002840F0A682464A1070002F40F0A7827C
:104C2000444B1A78002A50D10299B5F900E0488B1C
:104C3000898BB5F902407045B4BF8027002747F043
:104C400040037145D8BF3B469B0843F08007A04214
:104C5000B8BF3B4643F04007A142C8BF3B469B0854
:104C6000B5F90440B5F9067043F0800EA042B8BF14
:104C7000734643F0400EA142C8BF73469B0843F001
:104C8000800E284C8742C8BF734643F0400E94F80C
:104C9000A2C08F42B8BF73469C4501F05083A4F870
:104CA000A42084F8A620244984F8A2300F78002F8D
:104CB00001F09E825F2B01F0F3826F2B01F0958152
:104CC000059B1B78D80741F15981049B1B6803F0B1
:104CD0000403002B40F00B870DF14008174C002215
:104CE000C8F8042004F1500A109240F6330B4FF03C
:104CF000190940F2833726E01C6B002094690020DC
:104D0000186B00206C490020605B00207868002050
:104D1000E83800208D7D0020404B4C00CC61002005
:104D2000F47E0020E422002030820020243800207D
:104D3000B422002005680020E80000208C38002004
:104D40000434544520D0A278E3789A4219FB0271CA
:104D5000F6D26278043219FB037335F912205A45F2
:104D6000A8BF5A46B2F5617FB8BF4FF461728A425C
:104D7000E6DD9A42E4DC21782429E1D84046043477
:104D8000F5F7B0FD5445DED1BC4A98E8030013782E
:104D9000BB4A82E80300002B00F00286B94B069361
:104DA000B7480121F5F7AEFD002840F0BC82F3784A
:104DB000002B40F0B882B44CDFF80093B048B9F84B
:104DC000007027F00107BFB20221A9F80070F5F7C3
:104DD00099FD002800F0B282BB0741F11F81AB4B67
:104DE000AB4A197850680893BF0708BF81F00201E9
:104DF000C1F340010792F4F7EDFC2421A048F5F738
:104E000081FD30B9059A1378590744BF23F0040394
:104E10001370246814F00A0F40F0D882B9F80070BB
:104E2000A00600F100830C219548F5F76BFD0028E2
:104E300000F03983974B1B7847F48077082BA9F84B
:104E4000007000F03A830E2B00F03783049B1B6840
:104E5000580544D5904B1B79002B00F0B5811421E7
:104E60008748F5F74FFD002840F0B3810EF0E6F9D2
:104E700001200DF043FB90B3DFF844A200244FF073
:104E8000CC0B02E0DCB2022C29D80BFB04F8631C2B
:104E90005AF80870002FF5D1C378804A90F90200C3
:104EA00052F8233001970322009201213A460CF078
:104EB00017FB034604EB440000EB0010099353B1C9
:104EC00039460AEB8000CC2221F016F8099B4AF8FB
:104ED00008300134E4B219F095FE0028D3D1059BC7
:104EE0001C7814F0010400F0ED826D4B01221A7061
:104EF000069BB5F906101B686A485A89012791423A
:104F0000077080F27683684B4FF07E521A60674AD2
:104F1000029BB5F900E01F8B92F90430107892F8EB
:104F200001C0002BAEEB070383EAE378A8EBE3783C
:104F300014BF01224FF0FF32B8F5FA7FA8BF4FF43B
:104F4000FA78404580F25283A8EB000307EE903ACE
:104F5000F8EEE77A039BBE45C3ED007A03DAF1EE83
:104F6000677AC3ED007AB5F902E0AEEB070383EA96
:104F7000E378A8EBE378B8F5FA7FA8BF4FF4FA78A6
:104F8000404580F25083A8EB000307EE903AF8EE1C
:104F9000E77A039B7745C3ED017A03DDF1EE677A8B
:104FA000C3ED017AB5F90400C31B83EAE375A5EBF1
:104FB000E375B5F5FA7FA8BF4FF4FA756545CCBF28
:104FC000A5EB0C03002302FB03F307EE903A039AD0
:104FD000049BF8EEE77AB842C2ED027ABCBFF1EE6C
:104FE000677AC2ED027A1A6812F4805200F0DB820E
:104FF000B1F5FA6F2E4BA8BF4FF4FA61B1F57A7F85
:105000001878B8BF4FF47A71A1F57A71002840F092
:10501000E382284D284885FB013ECB17C3EB6E1376
:1050200003F1010E6FF0630C30F91EE030F913004C
:105030000CFB0313AEEB000103FB01F385FB03152F
:10504000DB17C3EB651303441BB207EE903A039BD7
:10505000B8EEE78A83ED038A002A40F01B85B9F891
:1050600000305A0600F1CB80002C40F04F811DF03B
:10507000DBFC13B0BDEC028BBDE8F08F373F0020A6
:10508000CC61002008480020084600204967002025
:105090004C67002088380020E47E0020087903084F
:1050A0008E7D0020EC210020902200201062002044
:1050B0009C8100201F85EB51D4360020A43F0020A6
:1050C000C45B0020A04B04931B68A04A029203F427
:1050D000805E9F4D9F4EBEF1000F3FF444AD002116
:1050E0009D48F5F70FFC00287FF43DAD9B4B0593E1
:1050F00019461B7813F001073FF43AAD984A9778A8
:1051000003F0FE030B70002F3FF432AD954C227874
:105110000B2A0DD80121914040F603070F4041F0C2
:10512000D98411F4C06F03D0093A012A41F2B9853C
:10513000DFF850B28C49DBF800204A600B2203F004
:105140000107227014E519F4800F7FF43BAD874C02
:10515000002284F8A020864A0392BBF1000F3FF49E
:105160004EAD844A01211170002F3FF459AD19F062
:10517000100F3FF455AD804A1278D2063FF550AD7E
:10518000BAF1000F7FF44CAD002B7FF449AD19F458
:10519000800F7FF445AD794B1B78002B01F0EB8439
:1051A000774B9B78BBF1000F41F08B853BB1754A83
:1051B000754B12681B689B1A002BC1F28E856B4CD5
:1051C000012384F8A1302BE5059B1B78D9077FF5D7
:1051D0004DAE3C2011F016FC00283FF480AE1CF0D0
:1051E00031FE3C2011F0BAFB00283FF478AE1CF0F1
:1051F00029FE3C2011F0B2FB0028F0D16FE6634B92
:10520000634AB3F904306349DFED636A09889FEDAF
:10521000637A82FB0302DB17C3EBA2035B1A1BB2A8
:1052200007EE903AF8EEE77A67EEA67A77EE876AAD
:10523000BDEEE66A16EE103A2033402B40F290871E
:10524000DFED576ABDEEE77A17EE103A2033402BB8
:1052500000F282879FED537AF4EEC77AF1EE10FAEE
:1052600041F32683DFED505A9FED506A01E0F0EEE6
:10527000477AF4EEC67AF1EE10FA37EEE57AF6DC0C
:10528000DFED4B7AB4EEE77AF1EE10FA41F11483D8
:10529000DFED455A9FED476A01E0B0EE677AB4EE64
:1052A000C67AF1EE10FA77EE257AF6D49FED3B7AC6
:1052B000F4EEC77AF1EE10FA40F34C869FED397A9E
:1052C00077EE677A67EEA75A9FED3B5A9FED3B6AF0
:1052D0009FED3B7AA5EE856A27EEA55AA5EE867A64
:1052E000E5EE077A039A92ED016AD2ED005A27EEB5
:1052F000C67A65EEA77AA5EEA67AE6EE267A82ED64
:10530000007AC2ED017A002C3FF4B1AE089B197807
:10531000079B01F001011868F4F75CFA13B0BDECCB
:10532000028BBDE8F08F274C23689A077FF544ADC8
:10533000DFF89490B9F8007047F0010727F00207F2
:10534000BFB2A9F800704AE56C490020605B0020FC
:1053500078680020E8380020CC6100208D7D002096
:105360007E8300207B830020EC610020E42200206B
:10537000F47E0020B42200200C460020E80000202B
:1053800034620020E8760020DC5F0020EC4500203D
:1053900067666666D85F002035FA8E3CDB0FC93F32
:1053A00000000000DB0F4940DB0FC940E4CB164191
:1053B000DB0F49C0E4CB16C192E741B99730083CF6
:1053C00015A82ABE08460020A43F00200521B948A0
:1053D000F5F798FAB9F80070002800F081857A078F
:1053E00040F1A3860621B348F5F78CFA002800F0B7
:1053F00070857B0640F1AA860721AE48F5F782FA50
:1054000000283FF40DADAC4BAC4AB3F90430AC49C5
:10541000B9F8007082FB0302DB17C3EBA203A006FE
:105420000B807FF500ADA74B1B78990706D5DFF8F9
:10543000F48298F81430042B00F2DB8717F0300F59
:105440003FF4F1AC10200DF0E5F820200DF0E2F86B
:105450009D4BB9F8007000221A709C499C4A9D48E7
:105460009D4C00230B609D4903604FF0000EC1F876
:1054700000E04B60C1F808E0C1F814E08B61C1F8AE
:105480001CE0236053609361C2F800E0C2F808E0BA
:10549000C2F814E0C2F81CE00C218648F5F732FA95
:1054A00000287FF4C7AC8E4B1B7827F48077BFB2FF
:1054B000082BA9F800707FF4C6AC27F04007A9F8C4
:1054C0000070C3E4874B1B780993002B7FF410AD69
:1054D000DFF854B2DFF854A21BF8030C9AF80080EE
:1054E0005946ABF1030708F0B1FC002800F0348402
:1054F000099BB8F1000F53D107F10801787908F042
:10550000A5FC002841F035827749B87A08F09EFC66
:10551000002800F03584B8F1020F41F02D82734964
:10552000F87B08F093FC002841F029827049387D0F
:1055300008F08CFC002800F03584B8F1040F41F02D
:1055400024826C49787E08F081FC002841F020829A
:105550006949B87F08F07AFC002800F03584B8F17A
:10556000060F41F00F82654997F8230008F06EFCA2
:10557000002840F0D987624997F8280008F066FCB7
:10558000002800F03584B8F1080F40F0BC875D4971
:1055900097F82D0008F05AFC00283FF4A9AC092325
:1055A0001A4600F0B2BF029B588B8142C0F2D283F0
:1055B000B1F5FA6FD4BFC0EB0101C0F5FA614FF449
:1055C0007A7303FB01F1504B1D78C0F5FA60B1FB13
:1055D000F0F1002D3FF41DAD5B784C4801FB03F367
:1055E00080FB0301DB17C3EB611112E5DFED487AA5
:1055F000B0E4B1F5FA6F80F2A783187A8B1A03FB37
:1056000000F3C2F5FA6293FBF2F3C3F1640307EE11
:10561000903AF8EEE77A9FED3F7A3F4B67EE877A54
:10562000C3ED007A73E4DFED3A7AB2E40BB90123FB
:10563000B3701B2008F034FCDFF8F49096F821805A
:1056400096F82030354C8246BB46052B00F21C8173
:10565000DFE813F09D0090000600EE000F01D3007C
:10566000B8F1010F04BF052386F82030BBF1000F0D
:1056700000F00181029B2A4FB3F91800D7F800E02F
:10568000B9F90030002160F30F0160F31F410022DF
:105690002960716960F30F0263F31F428E456A60EF
:1056A00000F2EB80B8F1010F41F0B78296F820309C
:1056B000CBE700BFCC610020EC4500206766666642
:1056C000D85F00200C460020483F00203C400020CE
:1056D000EC3F0020602200206422002014400020C3
:1056E000883800208E7D00200049002005490020D8
:1056F0000A4900200F4900201449002019490020C0
:105700001E490020234900209C8100201F85EB5169
:10571000000000000AD7233C9022002006680020E9
:10572000E876002010460020F6480020A80000205F
:105730003849002008F0E0FB012807D18D4FB9F867
:1057400002303A68642101FB03233361BAF1000F90
:1057500003D099F80630002B62D1B8F1010F00F0A8
:105760009380844F32693B689A42C0F038860123A7
:1057700086F82030B8F1010F3FD099F80730012B9F
:1057800000F0AB800FF0BAFA96F820305DE7BBF17D
:10579000000FCFD14FF48060BAF1000F00F0968374
:1057A0000CF040FF00223261049A059BD2F8009071
:1057B0001F78B5F9063019F4805A07F001073FF455
:1057C000F2A91D216C480393F5F79CF8039B002870
:1057D0007FF4E9A96949029AB1F806B0128BA2EBED
:1057E0000B018B4240F3F7855A449342B4BF4FF00C
:1057F000000B4FF0010BFFF7DFB95E4F3A68B9F8C5
:105800000230642101FB03234FF4806000223361E6
:1058100086F82020F2700CF0FDFE96F8203014E798
:105820000FF06CFA03224FF47A7386F82020F361AC
:10583000504F238843F00203238012F019F83A688E
:10584000F36913440422B36186F82020B8F1010FF4
:1058500040F0B7853B68B2699A4215D2484B187838
:1058600010B908F01DFB78B9238823F002032380C8
:10587000C4E7404FEAE73F4F3B6847F2305203230B
:10588000F26186F82030D4E7059B1F78B5F9063021
:1058900007F00107FFF780B9029A013BD27D35F985
:1058A0001330002A40F02383A3F57A73B3F57A7F8F
:1058B000A8BF4FF47A7323EAE37307EE903A9FEDA3
:1058C000317AF8EEE77A67EE877A2F4AFCEEE77ACC
:1058D00017EE903A1380FFF755B90FF00FFA032235
:1058E00040F6B83386F82020F361224FA1E7274F16
:1058F0003B78002B00F0E487254BDFF89880DFF839
:1059000098B0DFF898A0029345465E46039099460A
:105910000EE019F804109847032C28DC88B93B786E
:105920002AF8020F01349C4205F1040580F203813C
:10593000072CE1B23046DBF80430EADD984700B2CC
:10594000EDE738F824206B88801A4FF47A719B1A9F
:1059500001FB00F040F6CA0290FBF3F008449042CD
:1059600040F2EE23A8BF10469842B8BF184600B2D6
:10597000D5E700BFE8760020CC610020E0350020AC
:10598000E8000020AAF1823F4C380020706B002014
:10599000605B0020A46C002088690020E2220020C7
:1059A000DFF850B3DFF85093BF4C98460BF15A071D
:1059B0004FF0010A59461BF8010C08F047FAF8B1FC
:1059C0009BF804009BF802309BF803E000EB4001D9
:1059D00004EB8101013BD1F8B42003EB43034B44BA
:1059E00093420DD094F8E02081F8B0E00AFA00F07C
:1059F00022EA0000C1F8B430C1F8B88084F8E000B1
:105A00000BF1060BBB45D5D1A84B06931946A84A06
:105A1000A84BA94C09681B78D2F800B008910793ED
:105A2000A4F1B00A002763686BB393F80090B9F152
:105A3000000F28D0A168ABEB010100290ADB9AF81E
:105A4000E0100120B84021EA00010BF5FA708AF855
:105A5000E010A060079AB2B1217858780431C9B239
:105A6000002840F06582029A35F91110108B00F180
:105A7000C80E714540F37B849AF8E0109B78394159
:105A8000C80740F13E850137042F04F10C04CAD148
:105A9000FFF786B91D218948F4F734FF00283FF449
:105AA000DEAAF378002B7FF4DAAADFED857A854948
:105AB00038EE678AC7F5FA63FDEEC87A1BB2CDED02
:105AC000027ABDF90820120381FB0201D217C2EB52
:105AD000A11203FB02F343F30F333B4407EE903A6A
:105AE000039BF8EEE77AC3ED037AFFF7B8BA6E4C82
:105AF00094F8AA3053B1059B1B78DF0706D5029BAB
:105B0000B5F906205B8B9A4200F3ED8411216B48B6
:105B1000F4F7F8FE002800F0F38194F8AE302BB9CA
:105B200094F8A83013B93223A4F8AC30012384F8D8
:105B3000AE30FFF7D1B8DDF80C90634A04921146FD
:105B4000604A096842F2010AA2FB092B11EA0A0A1B
:105B50004FEA9B1B00F0D0815C4D5D48554C5D4A7F
:105B600095F800E0007884F800E01070BEF1000FB6
:105B700004D0584A92F800E08EF0010E4A4C0F20F3
:105B800084F82400002B00F04083534B0B931B78C8
:105B90000A931E463B78029F504AB7F824C0DFF8AC
:105BA0005C8109903D46FF8C08973746A2FB066250
:105BB00052082D8B0E9502EB420294F825500C955D
:105BC000BA1AD2B201F48051079204F128060BF5FB
:105BD00096726746424DCDF80CE0A4465446DDF877
:105BE00030A00F9100200592CDF834909E46039B83
:105BF000002B00F019823CF910101FFA81F9B94509
:105C00004FEA400203D3089B994540F24F8258F86F
:105C100020108B4580F01182A95E002C40F0258277
:105C200001307045A95206F10606E0DB09982D4ABD
:105C3000DDF834908CF824000F28644651460CBFE0
:105C400001210021734684F825A0117000F0E38241
:105C5000254EDFF85CB0254FDBF80000B1681C4A28
:105C60003C88F060401A01211170726844F004040D
:105C700090423C80174C88BF0022217088BF86F874
:105C80002120002B00F0DB82049A02981268184F42
:105C9000B0F82480B0F818C0114812F4805E3C4679
:105CA00040F0E08271463AE0E422002008480020FB
:105CB000E87600200C39002094230020CC610020DD
:105CC00000007A44D34D62106C49002064690020C2
:105CD000B8130020B91300201D6B0020ABAAAAAA9C
:105CE000786800200D390020E83800200668002080
:105CF000D86C00200D48002094640308206B00201D
:105D0000627802EB820202EB820202F2EE2292B28F
:105D100001318B4220F8022B04F102040ED017F857
:105D20001120002A00F0C681022AE9D00131028840
:105D300020F8022B8B4204F10204F0D10B9A137865
:105D400001331370FEF70BBF1B7AC3F1640307EE38
:105D5000903A5EE4114636E40BF10501787908F0DB
:105D600075F800283FF4D0ABB8F1010F40F0018680
:105D700007F10D01B87A08F069F8002840F0FC85B9
:105D8000D049F87B08F062F800283FF4CFABB8F1B7
:105D9000030F40F0F485CC49387D08F057F800280F
:105DA00040F0F385C949787E08F050F800283FF4A8
:105DB000CFABB8F1050F40F0EB85C549B87F08F0CF
:105DC00045F8002840F0DE85C24997F8230008F026
:105DD0003DF800283FF4CFABB8F1070F40F0A483A3
:105DE000BD4997F8280008F031F8002840F08B836F
:105DF000BA4997F82D0008F029F800283FF478A850
:105E0000B8F1090F3FF474A8FFF7C9BBB44CD4F83C
:105E10008830A9EB0303002BFEF6B4AEB14A94F828
:105E20008C30517C069AC4F888200133AE4A03F0C6
:105E30000F0332F8112084F88C3002992344897DB5
:105E400092B292FBF1F283F8902094F8901094F8BB
:105E5000912094F8923094F89C000A4494F893109E
:105E6000134494F89420194494F895300A4494F813
:105E70009610134494F89720194494F898300A44E3
:105E800094F89910134494F89A20194494F89B308C
:105E90000A44134494F89D1094F89F20184494F8F1
:105EA0009E3001440B441A44029942F30B12642AB7
:105EB000C97DA8BF642213B209B1C2F1640307EE21
:105EC000903A9FED8A7AF8EEE77AFCE40CF0A2FBB8
:105ED00068E427F04007BFB2A9F80070FFF78CBA5A
:105EE00027F00407BFB2A9F80070FFF77BBAC3F52B
:105EF0003B6308331BB2D7E47D4A92F800E035E6F5
:105F000094F8A830002B3EF4E7AE059B1B7813F005
:105F100001037EF4E1AE012284F8A83084F8A920C0
:105F2000FEF7DABE6E4C012284F8A020FFF719B903
:105F3000012800F071849AF8E0200123BB4001376A
:105F40001343042F8AF8E03004F10C047FF46BADA6
:105F5000FEF726BF9FED677AF4EEC77AF1EE10FAEE
:105F600044BF9FED657A77EE677AFFF7ABB9059B83
:105F7000624A1B781060DF0700F1988294F8A6103F
:105F800000297EF4A2AEB4F9A430322B7EF79DAE88
:105F900094F8A2200120572A84F8A60000F0B384C8
:105FA000049B1B6813F0040302D05A2A00F0D68524
:105FB0005D2A00F0F0845B2A00F086855E2A00F0FE
:105FC0008685562A00F0BE85972A00F0B185A72A5B
:105FD00040F0E9844A49049B0A781B6842F00402B5
:105FE0000A7003F00403FEF774BEB2F5FA7FFEF602
:105FF0006CAE94F8A620002A7EF467AE059B1B7851
:10600000012184F8A610DC0700F1008511F024F8C6
:10601000049B1B6803F00403FEF75BBE47F0020716
:10602000A9F80070FEF7DBBE002F3DD058F8201015
:106030008B454FEA4002FFF4EFAD324B995C03EB26
:106040000209002900F0008102296CD199F80110A1
:1060500001EB810101EB810101F2EE2189B20328FC
:1060600058DD09B2002C3FF4DBAD079B26F8131076
:10607000BAF1000F03D10A9B022B7FF6D1ADB6F81F
:1060800000A07188B6F804901F4B514489440FFA60
:1060900089F983FB09311D4BA1EBE97123F80290CB
:1060A00009B24FF0010ABBE539464200059B48F8AA
:1060B0002030B2E5CAB2022A2AD9032A7FF436AECA
:1060C000424625E6054900200A4900200F490020E4
:1060D00014490020194900201E49002023490020AE
:1060E000E4220020F07600200C77002014AE23413B
:1060F0000C390020DB0FC9BFDB0F49C0E05F002077
:106100000C460020D86C00205655555554230020CD
:106110006246FDE5012303FA00F9099B23EA09031E
:1061200009B2099379E5A95A99E7C54BC54AB3F96C
:106130000430C54982FB0302DB1747F00407C3EBB9
:10614000A203A9F800700B80FFF74CB947F0400795
:10615000A9F80070FFF750B9DFEDBC7AFFF7C2B8BD
:10616000F4EEC77AF1EE10FA40F3AE83DFEDB85AE1
:106170009FEDB86A01E0F0EE476AF4EEC66AF1EE10
:1061800010FA36EEE57AF6DCDFEDB36AB4EEE67AC5
:10619000F1EE10FA40F19B83DFEDAD5A9FEDAF6A4F
:1061A00001E0B0EE667AB4EEC67AF1EE10FA77EE60
:1061B000256AF6D49FEDAA7AF4EEC76AF1EE10FADA
:1061C00040F3B1809FEDA77A77EE666A66EEA65A35
:1061D0009FEDA55A9FEDA56A9FEDA57AA5EE856A6C
:1061E00026EEA55AA5EE867AE5EE076AFFF72AB8ED
:1061F0003946A048F4F786FB00283FF4B8AE84F88F
:10620000A77010F029FFFEF75BBD9B499B4A0B91DD
:106210009B4D012111701B2196480393F4F772FBEB
:10622000039B00287FF414AD964EDFF868B2F26845
:10623000DBF80030B3609B1AC82B00F24B83049B41
:106240001B6803F4805E79E5C1B2022940F2E28264
:1062500003297FF468AF0E9B19460F9B002B08BFE4
:106260003946FCE600210FE0627802EB820202EB85
:10627000820202F2EE2292B20131994220F8022B00
:1062800004F102043FF45AAD17F811201AB1022AA2
:10629000EAD00288F0E7CAB2032AFAD86246EBE7EE
:1062A000B2F5FA7FFEF611AD94F8A630002B7EF41D
:1062B0000CAD059F3B78012113EA010084F8A6107C
:1062C00000F01683704A927823F001033B70002A95
:1062D0003EF4FBAC6D4C23780B2B18D801FA03F27B
:1062E00040F603010A427EF4F0AC12F4C06F0ED007
:1062F000093B012B0BD8452016F060F8FF2016F063
:106300005DF8634816F046F8002016F057F861492A
:10631000049B614A1B68096851600B2203F0040367
:106320002270FEF7D6BC9FED5D7AF4EEC76AF1EEFF
:1063300010FA44BF9FED487A77EE666A46E7584AFE
:1063400058491068B4F9A420C76981FB0701891175
:10635000FF17781A00F5FF407F3082423EF7A3AC6A
:10636000C91B0A4412B2A4F8A420FEF79CBCC8388A
:10637000814258DA9AF8E0109B783941C9073FF515
:1063800082ABC3F1000809F1FF31162900F25481F4
:10639000DFE811F0D501E901BC013301FD0116026E
:1063A000A80194017F016A015501520133014401A2
:1063B0001602A80194011F010B01F7002A02E10057
:1063C000CD0005993A68F3690F781344B36107F07B
:1063D0000107FEF7DFBB4FF0010BFEF7EDBB0EF040
:1063E0008DFC032240F6B83386F82020F361FFF7D6
:1063F00020BA0A2007F054FD8246002800F04082AF
:10640000FA0640F10B83284C94F8F0A0BAF1000F83
:106410007EF409AD012384F8F030BAF1000F7FF467
:106420001CA8FEF700BD9AF8E0300122BA4023EA2A
:1064300002030BF5FA728AF8E030A260FFF723BB83
:10644000EC450020676666665C40002000000000A6
:10645000DB0FC940E4CB1641DB0F49C0E4CB16C1CA
:10646000DB0FC93FDB0F494092E741B99730083C49
:1064700015A82ABECC6100201D6B00200D3900201C
:1064800078680020E83800207E8300207B8300208D
:106490002C890308E8760020EC610020DB0FC9BFDF
:1064A00090470020D34D6210E4220020C04B1B789F
:1064B000002B3EF40AACF378002B7EF406AC94F883
:1064C000A7300133DBB2032B84F8A7307EF6FDAB97
:1064D000B84B5B781BB9BBF1000F7EF4F6AB11F043
:1064E000C7F9FEF7EDBB0021B348F4F70BFA00281B
:1064F0007FF40CAB322384F8AA00A4F8AC30FFF789
:1065000005BB98463FE708231A4602EB8202174470
:106510008AF80030B97878780AF046FF059B1C7835
:1065200004F00104FEF7E4BC07231A46EDE7DAF8AD
:10653000E400A24B90F836109A7841446429A8BF31
:10654000642121EAE17180F83610002A40F071835D
:1065500005F0CAFDEFE4DAF8E400984B90F8371044
:106560009A784144FE29A8BFFE2121EAE17180F812
:106570003710002AECD0162007F0F0FCDAF8E4001F
:10658000E6E7DAF8E40081788C4B4144C829A8BFDB
:10659000C82121EAE17181709B78002BD8D01420AA
:1065A00007F0DCFCDAF8E400D2E7DAF8E40041783E
:1065B000824B4144C829A8BFC82121EAE17141703A
:1065C0009B78002BC4D0132007F0C8FCDAF8E40055
:1065D000BEE7DAF8E4000178784B4144C829A8BF47
:1065E000C82121EAE17101709B78002BB0D0122004
:1065F00007F0B4FCDAF8E400AAE7089A6F4B917947
:10660000987841446429A8BF642121EAE17191711D
:10661000002840F02A83B9F10D0F0DD00898674B80
:1066200041799A7841446429A8BF642121EAE17143
:106630004171002A40F00D83DAF8E40088E7DAF8C7
:10664000E4005E4B017A9A784144C829A8BFC8216A
:1066500021EAE1710172002A3FF47AAF0B2007F0C2
:106660007DFCDAF8E40073E7DAF8E400534BC17913
:106670009A784144C829A8BFC82121EAE171C171B3
:10668000002A3FF465AF0A2007F068FCDAF8E4005E
:106690005EE7DAF8E400494B81799A784144C829E9
:1066A000A8BFC82121EAE1718171002A3FF450AFEF
:1066B000092007F053FCDAF8E40049E7DAF8E400CF
:1066C0003E4B41799B784144C829A8BFC82121EAA3
:1066D000E1714171002B40F0C282B9F1110F7FF4DA
:1066E00052AF35E7DAF8E400344B01799B78414446
:1066F000C829A8BFC82121EAE1710171002B40F02F
:10670000A282B9F1100F7FF452AF21E7089A1179F4
:106710008844B8F1640FA8BF4FF0640828EAE8780D
:1067200082F8048007F034FC244B9B78002B83D044
:106730000320414607F012FCDAF8E40008E7089A63
:106740001E4B11784144FA29A8BFFA2121EAE171D0
:1067500011709B78002B3FF46FAF012007F0FEFB18
:10676000DAF8E400F4E6089A144B9178414464297D
:10677000A8BF642121EAE17191709B78002B3FF45E
:106780005BAF022007F0EAFBDAF8E400E0E60898E5
:106790000A4BC1799A78414481F30801C171002AFA
:1067A0003FF44AAF052007F0D9FBDAF8E400CFE662
:1067B0000C39002034620020CC6100207E83002050
:1067C000DAF8E400C94BC1789B784144C829A8BFD6
:1067D000C82121EAE171C170002B40F02E82B9F18D
:1067E0000F0F7FF4F8AEB3E6089AC04B51784144DE
:1067F000B1F5967FA8BF4FF4967121EAE17151700F
:106800009B78002B3FF418AF152007F0A7FBDAF8B0
:10681000E4009DE60E9922E435F91110987840F6CF
:1068200033039942A8BF1946B1F5617FB8BF4FF451
:106830006171B9F10C0FA1F561714FF4966393FB8F
:10684000F0F391FBF3F100F08380B9F1180F7FF4BE
:1068500072ABDAF8E430C9B2C82993F817E00846F9
:10686000A8BFC82086453FF466ABA04AD875927889
:10687000002A3FF460AB484607F070FBFFF75BBBB4
:10688000FB0600F116810B2007F00AFB002840F000
:10689000DD80BC0600F12181954C94F8F030002B8E
:1068A0003FF4B8ADBAF1000F7EF4D7ADFEF7BBBA36
:1068B000B0EE677AFEF7E4BCF0EE477AFEF7F6BC7E
:1068C0008C4A0292FFF739B9B0EE667A5CE4F0EEDA
:1068D000476A6FE48849049B1A680B8823F0040315
:1068E0000B80012302F4805E86F82130FFF726BA80
:1068F000049B84F8A6001B68FA3AA4F8A42003F0CD
:106900000403FEF7E6B97D4B7D491A684FF47A73AC
:10691000B3FBF2F3C3EB431203EB8202049B1B684D
:10692000D200A1F8B42019067EF5D1A9754A1278D3
:1069300092077EF5CCA9744A127D042A7EF6C7A977
:1069400009F0FEFE049B1B6803F00403FEF7C1B9C7
:106950006E4B5B78C9B28B423FF4EDAA08460991B1
:1069600002F0FEFD614B09999B78002B3FF4E3AAEE
:1069700081E701231A46C8E502231A46C5E5032329
:106980001A46C2E506231A46BFE504231A46BCE5AB
:1069900005231A46B9E55E4A00215C4C5D4821702A
:1069A0000260FEF796B90021BB2A109100F0178112
:1069B000B72A00F01081BE2A00F00B81BD2A00F03A
:1069C000E9809E2A00F023819D2A00F01981AE2AD9
:1069D00000F00F81AD2A00F00581EF2A00F05B8105
:1069E000FD2A00F05281FB2A00F04981FE2A00F0C6
:1069F0004081F72A00F017817B2A7EF466A94FF4C4
:106A0000FA61022002F0D2FCFEF75FB9049B424912
:106A10001B680A6003F00403FEF75BB910200BF05B
:106A200001FE20200BF0F6FD3C49314C081F0AF016
:106A3000FDFB3B4B02221A7094F8F030B9F800705D
:106A4000002B7EF40AAD4FF0010AE3E4354B0399C5
:106A50005B8991ED007A07EE903AF8EEE77AB0EEB6
:106A6000C77AB4EEE77AF1EE10FA7FF512AF91ED46
:106A7000017AB0EEC77AF4EEC77AF1EE10FA7FF73A
:106A800008AFBB063FF508AF194C20200BF0CAFD3C
:106A90002146D8F80420D8F8003041F8EC2F04F152
:106AA000E800C4F8E8300AF0C1FB1D4B01221A705F
:106AB000C2E710200BF0AEFD194BB9F8007083F857
:106AC00000A04FF0010ADEE6174A012165E7174AE8
:106AD000022162E70746FEF74BB820200BF09AFD33
:106AE0000F4B034C00221A70A6E700BF7E830020E4
:106AF000E4220020605B0020066800205C49002042
:106B0000FC6C00200C460020104600201E82002055
:106B10003E82002030820020E05F0020403F0020C5
:106B2000483F0020E03F00208C820020DA820020D5
:106B3000049B714A1B684FF4C871118003F0040371
:106B4000FEF7C7B816F04AFDF4F7FDF816F02EFD73
:106B5000F5F712FD94F8A220FFF736BA94F8A820B2
:106B6000002A40F0C28094F8AA2082F0010284F842
:106B7000AA20FEF7AEB8BBF1000F3EF420AB5F4C8D
:106B800094F8A130002B3EF44BA8002384F8A130E8
:106B9000FEF746B84FF6FE73594A9789D0893B44B1
:106BA00001449381D18116F019FDF4F7CCF816F069
:106BB000FDFCF5F7E1FC049BB4F8A4201B68FA3A4D
:106BC0000021A4F8A42003F0040384F8A610FEF723
:106BD00080B80223E0E70B464FF6FE71DCE70B4678
:106BE0000221D9E7FF2100201CF0AAFE94F8A22080
:106BF000F3E6012100201CF0A3FE94F8A220E9E6B0
:106C00000021FF201CF09CFE94F8A220DFE601206A
:106C10001CF096FE94F8A220D6E6059A177807F0A5
:106C20000107FDF7B9BF0021042002F0BFFBFEF70A
:106C30004CB8172007F092F9FEE40F2007F08EF908
:106C4000DAF8E400CBE5102007F088F9DAF8E40080
:106C500057E50E2007F082F9DAF8E40078E4112015
:106C600007F07CF9DAF8E40037E50D2007F076F953
:106C7000D1E40021032002F099FBFEF726B80021A1
:106C8000022002F093FBFEF720B80021012002F061
:106C90008DFBFEF71AB80021084602F087FBFEF7CD
:106CA00014B8452015F08AFBFF2015F087FB154826
:106CB00015F070FB384615F081FB059B1B78FEF73D
:106CC00037BA002B3FF45BAF0F49104A09684FF405
:106CD0007A7000FB0313136051E7084C10F0C8FDF5
:106CE000002384F8A130FDF79BBF84F8A81084F836
:106CF000A900FDF7EEBF00BFE6840020E4220020DB
:106D0000186200202C890308E8760020DC5F002050
:106D10002DE9F047B0F908500D81EDB2382D8AB059
:106D20000C4600F0B78106462ED9802D00F0C980B0
:106D300077D8522D00F0B98040F26A81542D00F0CE
:106D4000D9816E2D40F03381B64B0A681B88B64D51
:106D5000FF2BA8BFFF23511C21601370A96881F38A
:106D6000100189B22046F3F787FAB04B2046198804
:106D7000F3F782FA296801F30F0189B22046012551
:106D8000F3F77AFA2B4647E0042D00F0A98140F290
:106D90002881202D00F0EF8040F26881242D00F042
:106DA000B581282D40F003810B68DFF8B882A04E32
:106DB000591C022221601A70236806275A1C22607F
:106DC0001F7023680A22591C21601A70236801254C
:106DD0005A1922601D70B8F800102046F3F74CFADB
:106DE000B8F802102046F3F747FA23685A192260D0
:106DF0001F7023685022591921601A7023680022DD
:106E0000591921601A7031882046F3F735FA7188D4
:106E10002046F3F731FA2B46284663810AB0BDE8D5
:106E2000F087822D7FD0C0F08581A02D00F0768183
:106E3000FE2D40F0BC807F4D05F1080635F8021BA1
:106E40002046F3F719FAAE42F8D101252B46284621
:106E500063810AB0BDE8F087762D40F0F181336898
:106E60005A1C32601B78002B01F04282102B07BFA6
:106E7000714A92E82200054629462268501C20608B
:106E800013702046F3F7E0F929462046F3F7DCF9C2
:106E90006A4B20461968F3F7D7F900212046F3F72B
:106EA000EBF900212046F3F7E7F922680021531C93
:106EB0000125236028462B46117063810AB0BDE886
:106EC000F0875F4B93F8009009F1020919F0FF0970
:106ED000BBD05C4B5C4F5D4EDFF88CA1994403F155
:106EE00001080A2516E0322D01F08181A5F13C0050
:106EF000C0B2132841F2828100232268511C216014
:106F000015702268C14502F10101216013709CD007
:106F100018F8015B0A2DE6D1BAF80030FF2BA8BFA4
:106F2000FF23DBB2E9E70B68494A3F4D1178494A34
:106F3000581C2060197011892046F3F79DF9394BD0
:106F400022681B88FF2B02F10101A8BFFF232160EB
:106F50001370A96881F3100189B22046F3F78CF908
:106F6000296801F30F0189B22046F3F785F93A4BFE
:106F7000226819789BE70B68364D591C6A782160A6
:106F80001A7023682A78591C21601A702368AA781D
:106F9000591C21601A7029892046F3F76DF923687E
:106FA0006A79591C21601A702268A9797FE7214605
:106FB0002846F4F7FBF900287FF447AF742D00F062
:106FC0001481772D7FF448AF336872689A421BBFF3
:106FD0005A1C326001461978204A204614F0F8FB0A
:106FE00033E7022D00F0F98000F2EC80012DDED1B4
:106FF0000B680022591C21601A7023685A1C2260F9
:107000001D7022682421531C23602B46117003E756
:10701000442DCCD1002A3FF418AF114B1360012549
:107020002B46F9E6DC7E00208C4500204C38002001
:1070300024810020307E0020CC230020D823002093
:10704000A85E0020DC640308676666663C81002059
:10705000F27E0020F4450020DC2D00207DAB0208EC
:10706000F1B200080862002064810020052D9ED145
:107070000B2264492046F3F7B7F8082262492046FC
:10708000F3F7B2F80125072260492046F3F7ACF880
:107090002B46C1E60A685E4B0125511C2160157024
:1070A0002268052150192060117022680A215019A8
:1070B0002060117022680021501920601170226830
:1070C0001978501920601170226859785019206081
:1070D000117022689978531923602B4611709BE632
:1070E00020462A464B49F3F77FF800212046F3F764
:1070F000C3F8DAE60B6800215A1C22601970226876
:107100000125531923602B46117085E6424B1968FF
:1071100020460125F3F798F82B4698E63F4B0846A2
:107120001968F3F791F83E4B20461968F3F78CF88D
:107130003C4BECE73C4B1E78033616F0FF063FF461
:1071400084AE3A4B3A4F1E4403F101094FF00A084E
:1071500020E0B8F1500F01F04780B8F1320F01F094
:107160006380A8F13C00C0B2132841F26180002581
:10717000294623685A1C2260204683F80080F3F7D2
:107180007BF829462046F3F777F8B1453FF45DAE2A
:1071900019F8018BB8F10A0FDBD1264B9D681968ED
:1071A00005EB85054FF6FF736D009D42A8BF1D4698
:1071B0009942A8BF194625EAE57521EAE171ADB209
:1071C00089B2D6E70B680322591C21601A70236824
:1071D0000222591C21601A7067E6042216492046D3
:1071E0000125F3F701F82B4616E6336872689A42D8
:1071F0001BBF5A1C326001461978104A204614F011
:10720000E7FA22E6688A0308748A0308808A03087A
:10721000198200202482002038620020107AFF1F8B
:10722000147AFF1F187AFF1FA85E0020EC64030881
:1072300034810020F0800020608A030881B60208B3
:10724000292D376801F01F80392D01F00A80212D8A
:1072500001F02E8072680B3DD31BEF2D00F2D48518
:1072600001A151F825F000BF9B7E0108097E0108AD
:10727000097E0108097E0108097E0108097E0108CE
:10728000097E0108097E0108097E0108097E0108BE
:10729000097E0108097E0108097E0108097E0108AE
:1072A000097E0108097E0108097E0108097E01089E
:1072B000097E0108097E0108097E0108097E01088E
:1072C000097E0108097E01084F7E0108097E010838
:1072D000357E0108097E0108137E0108097E010838
:1072E000097E0108097E0108477F0108097E01081F
:1072F000D17E0108097E0108097E0108097E010886
:10730000097E0108097E01084B7B0108097E0108FE
:10731000F77A0108097E0108C17D0108097E01088C
:10732000097E0108097E0108097E01084B6E0108EB
:10733000097E0108A57D0108097E0108097E010872
:107340008B7D0108097E0108317D0108097E010855
:10735000097E0108097E0108097E0108097E0108ED
:10736000097E0108097E0108097E0108B17C010837
:10737000097E0108257C0108097E0108097E0108B3
:10738000737C0108097E0108097E0108097E010855
:10739000097E0108097E0108097E0108097E0108AD
:1073A000597B0108097E01081F810108097E010837
:1073B00075800108097E0108977F0108097E010890
:1073C0006F7F0108CB810108097E0108097E010851
:1073D000097E0108097E0108097E0108097E01086D
:1073E000097E0108097E0108097E0108097E01085D
:1073F000097E0108097E0108097E0108097E01084D
:10740000097E0108097E0108097E0108097E01083C
:10741000097E0108097E0108097E0108097E01082C
:10742000097E0108097E0108097E0108097E01081C
:10743000097E0108097E0108097E0108097E01080C
:10744000097E0108097E0108097E0108097E0108FC
:10745000097E0108097E0108097E0108097E0108EC
:10746000097E0108097E0108097E0108097E0108DC
:10747000097E0108097E0108097E0108097E0108CC
:10748000097E0108097E0108097E0108097E0108BC
:10749000097E0108097E0108097E0108097E0108AC
:1074A000097E0108097E0108097E0108097E01089C
:1074B000097E0108097E0108097E0108097E01088C
:1074C000097E0108097E0108097E0108097E01087C
:1074D000097E0108097E0108097E0108097E01086C
:1074E000097E0108097E0108097E0108097E01085C
:1074F000097E0108097E0108097E0108097E01084C
:10750000097E0108097E0108097E0108097E01083B
:10751000097E0108097E0108A1810108097E010890
:10752000097E0108097E0108097E0108097E01081B
:10753000097E0108097E0108097E0108097E01080B
:10754000097E0108097E0108097E0108097E0108FB
:10755000097E0108097E0108097E01089B7A01085D
:10756000497A0108FD790108097E0108617901085D
:10757000F1780108D5780108097E01082F7A010801
:107580006F7801084778010835780108D777010836
:10759000097E0108A9770108097E0108097E010812
:1075A0008777010859770108457701081D77010899
:1075B000097E0108FB760108CF7601085D76010897
:1075C000097E0108097E0108097E0108097E01087B
:1075D000097E0108097E0108097E0108097E01086B
:1075E000097E0108097E0108097E0108097E01085B
:1075F000097E0108097E010843760108097E010819
:10760000097E010875760108097E0108097E0108D6
:10761000097E0108097E0108097E0108097E01082A
:10762000097E010829760108B84B1B78DB0700F1B9
:10763000EB830125F4F7EEFEF4F79EFF2B46FFF7F0
:10764000EBBB3046F2F7BEFDB14FF8813046F2F7A2
:10765000B9FD0125B8812B46FFF7DEBB3046F2F7B6
:10766000B1FDAC4A00EB80004300012513802B469E
:10767000FFF7D2BB7B1C33603B780F2B00F2C48337
:10768000BA1C3260C3EBC303A34A7978D154F91C06
:1076900031601344BA785A703A1D3260FA789A70A1
:1076A0007A1D32603A79DA70BA1D32607A791A71CD
:1076B000FA1D3260BA795A7107F108023260FA791C
:1076C0009A71012504F028F92B46FFF7A5BB3A462D
:1076D0007B1C3360914B12F8021B197032607A7870
:1076E0005A70FA1C3260BA789A703A1D3260FA7891
:1076F000DA7001252B46FFF78FBB3046F2F762FDAB
:10770000874F38823046F2F75DFD78823046F2F7D7
:1077100059FD0125B8822B46FFF77EBB3B467A1CFC
:107720003260804A13F8021B11703360784A7B780C
:107730009370FB1C3360774BBA789A7001252B4607
:10774000FFF76ABB784B794918684E2201251EF075
:10775000AEFB2B46FFF760BB3A467B1C3360744B95
:1077600012F8021B197032607A785A70FA1C326073
:10777000BA789A703046F2F725FD6E4B0125D88015
:107780002B46FFF749BB3046F2F71CFD694F3880A6
:107790003046F2F717FD78803046F2F713FD0125E9
